:020000040800F2
:1000000000060020B5050008F9300008753000082A
:10001000CD30000875300008A1300008B705000891
:10002000B7050008B7050008B70500082D4200080D
:10003000B7050008B7050008B7050008B7050008B0
:10004000B7050008B7050008B7050008B7050008A0
:10005000B7050008B7050008ED520008195300085D
:1000600045530008715300089D530008B705000868
:10007000B7050008B7050008B7050008B705000870
:10008000B7050008B7050008B7050008B52A00083D
:10009000A92B00082D2B0008212C0008C9530008AB
:1000A000B7050008B7050008B7050008B705000840
:1000B000B7050008B7050008B7050008B705000830
:1000C000B7050008B7050008B7050008B705000820
:1000D000B7050008B7050008B7050008B705000810
:1000E00041540008B7050008B7050008B705000827
:1000F000B7050008B7050008B7050008B7050008F0
:10010000B7050008B7050008C9540008B70500087E
:10011000B7050008B7050008B7050008B7050008CF
:10012000B7050008B7050008B7050008B7050008BF
:10013000B7050008B7050008B7050008B7050008AF
:10014000B7050008B7050008B7050008B70500089F
:10015000B7050008B7050008B7050008B70500088F
:10016000B7050008B7050008B7050008B70500087F
:10017000B7050008B7050008B7050008B70500086F
:10018000B7050008B7050008B7050008B70500085F
:10019000B7050008B7050008B7050008B70500084F
:1001A000B7050008B7050008B7050008B70500083F
:1001B000B7050008B7050008B7050008B70500082F
:1001C000B7050008B7050008B7050008B70500081F
:1001D000B7050008B7050008B7050008B70500080F
:1001E000B7050008B7050008B7050008B7050008FF
:1001F000B7050008B7050008B7050008B7050008EF
:10020000B7050008B7050008B7050008B7050008DE
:10021000B7050008B7050008B7050008B7050008CE
:10022000B7050008B7050008B7050008B7050008BE
:10023000B7050008B7050008B7050008B7050008AE
:10024000B7050008B7050008B7050008B70500089E
:10025000B7050008B7050008B7050008B70500088E
:10026000B7050008B7050008B7050008B70500087E
:10027000B7050008B7050008B7050008B70500086E
:10028000B7050008B7050008B7050008B70500085E
:10029000B7050008B7050008B7050008B70500084E
:1002A0002518000800000000000000000000000009
:1002B00053B94AB9002908BF00281CBF4FF0FF31CD
:1002C0004FF0FF3000F074B9ADF1080C6DE904CEC9
:1002D00000F006F8DDF804E0DDE9022304B0704721
:1002E0002DE9F047089D04468E46002B4DD18A42E9
:1002F000944669D9B2FA82F252B101FA02F3C2F11C
:10030000200120FA01F10CFA02FC41EA030E9440AC
:100310004FEA1C48210CBEFBF8F61FFA8CF708FBCD
:1003200016E341EA034306FB07F199420AD91CEBA5
:10033000030306F1FF3080F01F81994240F21C81D7
:10034000023E63445B1AA4B2B3FBF8F008FB10331F
:1003500044EA034400FB07F7A7420AD91CEB040454
:1003600000F1FF3380F00A81A74240F20781644424
:10037000023840EA0640E41B00261DB1D4400023A9
:10038000C5E900433146BDE8F0878B4209D9002D0D
:1003900000F0EF800026C5E9000130463146BDE897
:1003A000F087B3FA83F6002E4AD18B4202D3824201
:1003B00000F2F980841A61EB030301209E46002DB0
:1003C000E0D0C5E9004EDDE702B9FFDEB2FA82F205
:1003D000002A40F09280A1EB0C014FEA1C471FFA63
:1003E0008CFE0126200CB1FBF7F307FB131140EA4A
:1003F00001410EFB03F0884208D91CEB010103F117
:10040000FF3802D2884200F2CB804346091AA4B2D8
:10041000B1FBF7F007FB101144EA01440EFB00FEAC
:10042000A64508D91CEB040400F1FF3102D2A64511
:1004300000F2BB800846A4EB0E0440EA03409CE7B0
:10044000C6F12007B34022FA07FC4CEA030C20FA5D
:1004500007F401FA06F31C43F9404FEA1C4900FA7D
:1004600006F3B1FBF9F8200C1FFA8CFE09FB1811FA
:1004700040EA014108FB0EF0884202FA06F20BD96D
:100480001CEB010108F1FF3A80F08880884240F2BD
:100490008580A8F102086144091AA4B2B1FBF9F001
:1004A00009FB101144EA014100FB0EFE8E4508D9FC
:1004B0001CEB010100F1FF346CD28E456AD9023881
:1004C000614440EA0840A0FB0294A1EB0E01A14266
:1004D000C846A64656D353D05DB1B3EB080261EBD4
:1004E0000E0101FA07F722FA06F3F1401F43C5E9AE
:1004F000007100263146BDE8F087C2F12003D840E4
:100500000CFA02FC21FA03F3914001434FEA1C4725
:100510001FFA8CFEB3FBF7F007FB10360B0C43EA17
:10052000064300FB0EF69E4204FA02F408D91CEBC7
:10053000030300F1FF382FD29E422DD902386344C5
:100540009B1B89B2B3FBF7F607FB163341EA034165
:1005500006FB0EF38B4208D91CEB010106F1FF38B4
:1005600016D28B4214D9023E6144C91A46EA0046AB
:1005700038E72E46284605E70646E3E61846F8E63D
:100580004B45A9D2B9EB020864EB0C0E0138A3E786
:100590004646EAE7204694E74046D1E7D0467BE767
:1005A000023B614432E7304609E76444023842E7DF
:1005B000704700BF02E000F000F8FEE772B63A486C
:1005C00080F30888394880F3098839484EF6085185
:1005D000CEF20001086040F20000CCF200004EF6BE
:1005E0003471CEF200010860BFF34F8FBFF36F8FFD
:1005F00040F20000C0F2F0004EF68851CEF2000149
:100600000860BFF34F8FBFF36F8F4FF00000E1EE34
:10061000100A4EF63C71CEF200010860062080F30D
:100620001488BFF36F8F04F0D1FB04F073FB04F068
:1006300071FC4FF055301F491B4A91423CBF41F8B5
:10064000040BFAE71C49194A91423CBF41F8040BDC
:10065000FAE71A491A4A1B4B9A423EBF51F8040B5B
:1006600042F8040BF8E700201749184A91423CBFB2
:1006700041F8040BFAE704F08FFB04F061FC144C22
:10068000144DAC4203DA54F8041B8847F9E700F034
:1006900041F8114C114DAC4203DA54F8041B884761
:1006A000F9E704F077BB00000006002000220020DC
:1006B000000000080000002000060020F859000893
:1006C000002200208022002080220020C05F002025
:1006D000A0020008A4020008A4020008A402000866
:1006E0002DE9F04F2DED108AC1F80CD0D0F80CD0C8
:1006F000BDEC108ABDE8F08F002383F311882846F3
:10070000A047002003F06CFFFEE703F0C9FE00DF06
:10071000FEE700002DE9F04101F0FCF818B1324B82
:100720004FF440229A6004F087FA064604F0E8FA93
:100730000546A8B92D4B9E4220D001339E4220D0C1
:1007400026F0FF022A4B9A4203D0804641F28834B9
:1007500008E0F0B200F056FEA84642F2107401E044
:100760008046002400F0C4FF08B10024A04600F039
:100770004FFE074648B1CCB9474607E08046002403
:10078000F0E700244FF00108ECE70024194B9E42EB
:100790000CBF002505F001055DB9002004F058FAF2
:1007A00067B900F0C7FF01F045F819E04FF47A741B
:1007B000ECE704F09DFA00242746EEE700F07EF80F
:1007C000EFE701F005F84FF47A7003F011FF002C09
:1007D000F7D002F099FC401BA042F2D900F06EF86D
:1007E00002F092FC0546F2E700220020010007B06B
:1007F000000008B0263A09B010B584468E46BFF313
:100800004F8FBFF36F8F1F4B0022C3F88420BFF3BD
:100810004F8F5A6922F480325A61BFF34F8FD3F859
:100820008040C4F34E3000E01846C4F3C90243F6DA
:10083000E07303EA401343EA82731249C1F8743249
:100840001346013A002BF2D1431E0028ECD1BFF32E
:100850004F8FBFF36F8FBFF34F8FBFF36F8F4A6917
:1008600022F400324A610022C1F85022BFF34F8FB8
:10087000BFF36F8F202383F31188E5468CF308883C
:10088000704710BD00ED00E008B50A4B1870012854
:1008900007D0022801D040B108BD022001F03EF887
:1008A000FAE7022001F038F8F6E7034B00225A601D
:1008B000F2E700BF802200208422002008B5002338
:1008C000072B08D8234A52F82320B2F1FF3F0DD05E
:1008D0000133DBB2F4E71F4B5B681F4A934205D933
:1008E0001E4A91681B4A0A44934200D308BD04F093
:1008F000E5F9002000F0CAFF0220FFF7C5FF184B02
:10090000D3F8E8200022C3F8E820D3F81011C3F888
:100910001021D3F81011D3F8EC10C3F8EC20D3F861
:100920001411C3F81421D3F81411D3F8F010C3F83C
:10093000F020D3F81811C3F81821D3F8183172B683
:10094000044B4FF0E022C2F8083D59681868FFF7E1
:1009500053FFCBE700000408FFFF0308002200203C
:1009600000440258094A136899B21B0C49F2690005
:1009700000FB01331360064B186882B2000C44F28E
:10098000506101FB0200186080B2704718220020FD
:100990001422002010B50446FFF7E4FFB0FBF4F387
:1009A00004FB130080B210BD00B583B002F0ACFBB5
:1009B0000023ADF800308DF80230284B1B68C31AB5
:1009C000642B0BD9264B93F90030C3EB0313254A54
:1009D000118811FA83F31380204B1860214BB3F96F
:1009E0000030002B05DB962B06DD1E4B96221A806D
:1009F00002E01C4B00221A801B4B1B68C31AB3F584
:100A00007A7F05D9164A13785B421370164B18602B
:100A1000144BB3F90020154B83FB0213A3EBE273D5
:100A2000DBB28DF800308DF802308DF80130009B7C
:100A3000ADF804301B0C8DF8063000209DF8043012
:100A400063F307009DF8053063F30F209DF806302F
:100A500063F3174003B05DF804FB00BF145D002092
:100A6000102200201C5D0020185D002056555555B1
:100A70002DE9F04383B000EB800303EB830303F124
:100A8000320505F00705C5F13A05EDB23933DF0847
:100A90000020FFF789FF8DF80400C0F307238DF8CD
:100AA0000530C0F307408DF80600002631465BE0B4
:100AB0005FFA89F0FFF778FF8DF80400C0F3072391
:100AC0008DF80530C0F307408DF80600494630E048
:100AD0000022294B4FF4807058831046002A40D1E1
:100AE0004FF0007343EA4023234A93614FF480732D
:100AF00013830134E4B2072C35D804EBC6039D42BE
:100B0000E6D85A1B1D4BA3FB0203DB0803EB830350
:100B100003EB83039A4222D0184BA3FB0238A2EBCB
:100B2000D808174BA3FB08234FEA1319B1EB131F87
:100B3000BED1134BA3FB08231B0903EB4303A8EB14
:100B4000C30302AA02EBD30313F8040C08F0070254
:100B5000C2F1080240FA02F202F00102B9E70122F2
:100B6000B7E70023BEE70136BE4201D20024C2E748
:100B700003B0BDE8F08300BF000402581F85EB51AD
:100B8000ABAAAAAA70B50E4614461D4602F0E2FEB4
:100B900060B9022D08BF012C0CBF0120002004D138
:100BA00018A3D3E90023C6E9002370BD282C1FD069
:100BB0000CD8012C15D0052C06D114A3D3E90023A1
:100BC000C6E900230120F0E70020EEE7302C06D133
:100BD00010A3D3E90023C6E900230120E5E70020A4
:100BE000E3E70EA3D3E90023C6E900230120DCE7F5
:100BF0000CA3D3E90023C6E900230120D5E700BFF9
:100C0000AFF30080401DA12026812A0BF017304A47
:100C100039059E5678F6339F93CACD8D9E6AC421BE
:100C2000818A46EE26417272DF25D7B710B403469B
:100C30000022026042608260C260044C07CC1860EF
:100C400059609A605DF8044B704700BF00E8F11FDF
:100C5000F0B58DB007460E4602F056FA04464FF442
:100C6000C870FFF797FE044404F51674224B1C600D
:100C7000F37E0BB1002412E0204B00221A700DB05D
:100C8000F0BD651CEDB2E90008AB1C4400940023E4
:100C9000082201F0F801304602F052FF2C46B38AD8
:100CA000013B9C42EDD304A8FFF7C0FF224604A9F4
:100CB00008A804F06DFC48B90F2C0BD80F4B1C7022
:100CC0000D4A1368A3F516731360D8E70B4B002287
:100CD0001A70D4E700218DF80F100DF10F03009367
:100CE0000B460722304602F02BFF9DF80F103846C6
:100CF00002F028FEC3E700BFA03200209D32002092
:100D00002DE9F043FFB007460E4600241F9440F241
:100D10007512214620A800F017FE0CAD4FF04808D0
:100D200042462146284600F00FFE02F0EDF96C4BDA
:100D3000A3FB00239B096B4A136007CA85E80700E1
:100D400001232B746C740DF15200FFF76FFF042325
:100D500085F82030132385F821300DF11809CC4691
:100D6000DFF884E1BEE80F00ACE80F009EE8030066
:100D70004CF8040B8CF80010142385F83C30C5F8AF
:100D800040902B46202221461FA802F0D5FF2B7948
:100D9000032B28BF03232B710DAB022220211FA898
:100DA00002F0CAFF6B79072B28BF07236B710DF187
:100DB0003503032222211FA802F0BEFFAB79072BC7
:100DC00028BF0723AB710DF13603032225211FA88D
:100DD00002F0B2FF0EAB102228211FA802F0ACFFD8
:100DE00010AB082238211FA802F0A6FF0DF1410325
:100DF000082240211FA802F09FFF0DF142030822A4
:100E000041461FA802F098FF11AB202250211FA8D5
:100E100002F092FF0DEB0803402270211FA802F0A0
:100E20008BFF14AB0822B0211FA802F085FF0DF143
:100E300051030822B8211FA802F07EFFC02509E057
:100E40000DF152032344082229461FA802F074FF23
:100E5000083501340F2CF3D919AB082229461FA8F5
:100E600002F06AFF083500249DF86430A34209D9D6
:100E70001A9B2344082229461FA802F05DFF08356B
:100E80000134F1E700249DF86C30A34209D91C9B82
:100E90002344082229461FA802F04EFF08350134DA
:100EA000F1E7EB1DC3F3CF0305931FAB04930023BE
:100EB0000393B37E029306F1190301930123009378
:100EC00005A3D3E90023F17E384602F0A5FD7FB0EB
:100ED000BDE8F083AFF300809E6AC421818A46EEAC
:100EE000D34D62108C220020AC56000870B5BAB009
:100EF00002F00AF9214B9B68C31AF92B01D83AB0CA
:100F000070BD1E4CA06023462822002106A802F0D6
:100F100013FF04F10E0000F00DFDC6B200242825D9
:100F20000CE004F10802154B13440633082229464D
:100F300006A802F001FF08350134E4B2B442F0D350
:100F400007350E49C5F3CF05059506AB049301237C
:100F500003930823029301F10D03019330230093BF
:100F600004A3D3E90023097B054802F055FDC6E739
:100F7000AFF3008078F6339F93CACD8D305C0020AC
:100F8000A43200208B8A013B9BB2C92B68D8F0B5F4
:100F9000ABB007460E46354B1C7B5CB10024069473
:100FA0000794089406AB0822214609A802F0C4FE63
:100FB000082537E00C3300930023082219463046F9
:100FC00002F0BEFD0825B38A013B9C420FDA04F112
:100FD0000802264B134406330093002308222946B7
:100FE000304602F0ADFD08350134E4B2EBE71F4BAB
:100FF00000200021C3E9000100229A6083F8D72075
:10100000C3F8D8201B7B002BC8D1F27E174B1A7374
:10101000C4E7089B23440822294609A802F08CFE55
:10102000083501349DF81C30A342F2D80735C5F3CA
:10103000CF05059509AB049300230393B37E029378
:1010400006F1190301932823009306A3D3E9002393
:10105000F17E384602F0E0FCFFF748FF2BB0F0BD10
:10106000704700BF26417272DF25D7B7305C002081
:10107000F0B58FB000230A938DF834308DF83530F9
:101080000B930C930024274601E00134E4B2012CB9
:1010900040D801238DF80C3000238DF80D3041F23B
:1010A000B04204FB02F21D495518525896680020C0
:1010B0000021CDE900010DF10D0203A92846B0473A
:1010C0009DF80C60002EE0D0002306930793089350
:1010D000099341F2B04304FB03F3104AD3585F690C
:1010E0000DF10E0304AA0AA92846B84707AB0BAABC
:1010F00092E8030083E803009DF834308DF8243033
:101100000A9B0693DDE9042306A9054802F07AFE4E
:101110003746BAE7002FB5D10FB0F0BDD03200206E
:10112000A432002010B58CB0264802F013FC08B1A0
:101130000CB010BD01F0E8FF234B1B689842F7D3B9
:1011400001F0E2FF04464FF4C870FFF723FC0444AB
:1011500004F516741C4B1C6000238DF828301B4BC3
:101160001B7813B901238DF8283006A8FFF75EFD20
:10117000164B1978C1F11004E4B2062C00D90624EC
:10118000224606AB19440DF1290000F0C9FB0134D9
:1011900004940AAB0393182302930D4B019301238C
:1011A000009306A3D3E90023064802F0D5FB074BC2
:1011B00000221A70BCE700BFAFF30080401DA120E1
:1011C00026812A0BA4320020A03200209D3200206C
:1011D0009C320020012800D0704738B504464FF6F5
:1011E000FF73994200D038BD084D002C07DB28461C
:1011F00000F034FF05F5A5551035013CF5E7044A2C
:101200000449002004F0A6F9EDE700BFD032002029
:10121000605D00201912000838B5104C04E041F25E
:101220003000204401F0D2FD0D4B9C4214D0A4F5B7
:10123000A554103C0B4B236041F24403E218127991
:10124000002AECD1E558002DE9D0284601F0BEFD7A
:10125000284604F085F9E2E738BD00BF305C002085
:10126000D0320020B8570008F0B587B0254802F00A
:1012700021FC002839D00446002502958DF8145031
:101280008DF8155003950495027B8DF8142003AA60
:101290004068A16803C2226842F0004202922C46D4
:1012A00019E041F2B04304FB03F3174A9E189B5820
:1012B0001F6901F02DFF154A82184FF000030093BB
:1012C00041F1000302A93046B8470028C8BF45F0E5
:1012D00001050134E4B2012CE3D945B90C4B1B786C
:1012E000072B0BD801330A4A137007B0F0BD05482D
:1012F00002F0E4FB064B00221A70B7E7014802F047
:10130000DDFBF2E7A4320020D032002040420F0083
:101310001F5D002030B589B001F0F6FE274BA3FB1E
:1013200000308009264C206006AD23462022002193
:10133000284602F001FD2279032A28BF0322234612
:1013400003F8042F02222021284602F0F5FC6279DE
:10135000072A28BF0722234603F8052F032222214C
:10136000284602F0E9FCA279072A28BF0722234673
:1013700003F8062F03222521284602F0DDFC04F1A4
:10138000080310222821284602F0D6FC07230493E4
:101390000395182302930B4B019340F255130093CE
:1013A00004A3D3E90023084802F0D6FA09B030BDFF
:1013B000AFF30080F1C6A7C1D068080FD34D62100B
:1013C0008C2200201E5D0020A432002010B50246B1
:1013D0000B46094C204602F079FB204602F0BAFA8F
:1013E00038B1064B1B7B2BB10322054B5A71FFF71B
:1013F00091FF10BD0222F8E7A4320020305C0020EB
:101400008C220020014B1870704700BF98220020EA
:10141000374B1B7B23B1374B0E221A8100207047BC
:1014200070B584B0344B02AA93E8030082E803004D
:1014300008233249324804F0BBF8044678B3016906
:10144000B1F5E01F33D8438B40F21342934236D1BB
:101450002C4A024402F1100399423BD3891AA1F1AC
:1014600010052749002001F05BFE06462A4604F1DC
:101470001801002001F054FEA368B34202D1E368D2
:1014800083422FD01B4B0D221A81A168E268009085
:1014900033461D4801F002FC002004B070BD154B1E
:1014A0000A221A81194801F0F9FB0020F5E7114BD7
:1014B0000B221A81164801F0F1FB0020EDE70D4ADE
:1014C0000C21118140F213421946124801F0E6FB4B
:1014D0000020E2E7074B10221A810F4801F0DEFBE3
:1014E0000020DAE70D4801F0D9FB0120D5E700BF65
:1014F000305C00208C22002060570008DCFF1B00BD
:10150000000004080800FCF724570008C45600082F
:10151000D0560008E4560008045700085057000849
:101520002DE9F04784B002AFE9464B7E01335A42C1
:10153000DBB2D2B258BF53424D4A527B934205D1DF
:101540000D46CA7E4A4B1B7B9A4204D0CD460837D3
:10155000BD46BDE8F0870021F980BB1D0093012343
:101560001022284602F0ECFAAE8A023EB6B2F31C14
:101570009B109B00073323F00703ADEB030D0DF128
:10158000080800244FF0100AB4420DD208EB0403FF
:101590000093002308225146284602F0D1FA0AF1AE
:1015A000080A0134A4B2EFE7314C94F8D70000F0F8
:1015B0007BF90546D4F8D8303BB12D4BD3F8D83061
:1015C0003344AB4206D8002416E094F8D70000F06C
:1015D0007DF9F2E7264B93F8D700013000F076F959
:1015E000F1E7234B1868012208EB840100EB84002B
:1015F00000F0B4F90134A4B2B4EB960FF1D31C4B54
:101600001A685968921941F100011A605960D3F8BB
:10161000D8403444C3F8D84093F8D70000F044F9D8
:1016200084420AD3124B93F8D720013283F8D72093
:10163000D3F8D820521BC3F8D820FF2E0CD90C4A5F
:10164000136851689B0A43EA8153013309490B81AE
:1016500000239360CD467AE7054B00221A7300F011
:1016600047F9FFF7D5FE0028E9D0FFF727F9E6E7AD
:10167000305C00208C22002038B505460C4602F074
:1016800069F950B1E38A282B1CD014D8012B0FD153
:1016900021462846FFF734FB0CE0237E022B09D1BC
:1016A000E38A012B06D121462846FFF7D1FA01E053
:1016B000052B0CD038BD302BFCD121462846FFF736
:1016C0002FFFF7E721462846FFF75CFCF2E7BFF360
:1016D0004F8F0549CA6802F4E062044B1343CB60A4
:1016E000BFF34F8F00BFFDE700ED00E00400FA05F7
:1016F0004FF040531A680D4B9A4201D000207047BA
:1017000010B54FF04054607DFFF77CFE237D084804
:101710000373C92204F116010E3000F001F9E02232
:101720000021204600F010F9012010BD9AAD44C5FB
:10173000305C002030B583B01C4B02225A7100246B
:101740000CE041F2B04304FB03F319481A58556802
:10175000012218491844A8470134E4B2012CF0D9F9
:1017600000230193144B0093144B4FF480521449FF
:10177000144802F0CBF8144B197899B901F0C4FC65
:1017800004464FF4C870FFF705F9044404F51674D5
:101790000E4B1C6003F0B4FA10B1044B0F221A81F7
:1017A00003B030BD074802F0CDF8E7E78C220020F7
:1017B000D032002040420F00850B00087916000847
:1017C0009C220020A432002098220020A032002079
:1017D00008B509E0114B186001F09AFCFFF7F6FD1F
:1017E00010E00F4B1B7BBBB1FFF73EFDFFF740FC4A
:1017F000FFF798FC01F088FC084B1B68C31AB3F58F
:101800007A7FE7D20420FFF733F9054B1B7B002BCF
:10181000E7D0FFF76BFBE4E708BD00BF105D0020D9
:10182000305C002008B54FF6FF710120FFF7D2FCB5
:1018300008BD00BF38B503F0CBF8124B1880002468
:1018400006E003F0C1F804440F4A13680133136043
:10185000B4F5802F07D20B4B1B880B4A10688342CC
:10186000EFD8002500E00025B5F5802F09D2054C02
:101870002088013803F0A8F805442388013B238021
:10188000F2E738BD4C5D0020205D002008B503F074
:1018900015F908BD08B5034692000248184403F044
:1018A00009F908BD0000040808B5064B1B88064A64
:1018B00012689B1A834201D8002008BD104403F02F
:1018C00083F8FAE74C5D0020205D002010B5044647
:1018D000064B1868204403F07DF800B110BD034B9F
:1018E0001868204403F08EF8F8E700BF205D002060
:1018F00008B5074B93F824300BB9012008BD044903
:10190000002381F824300822086AFFF7C3FFF5E7B7
:10191000245D002000207047704700BF704700BF63
:10192000002304E011F803C000F803C00133934220
:10193000F8D370470346002000E0013013F9012B73
:10194000002AFAD1704700BF034602E003F8011BEA
:10195000624602F1FF3C002AF8D170472DE9F843B6
:10196000814688461546214B93F8243033B31F4AED
:10197000126A02EB8303834220D0FFF7B9FF0346CC
:10198000E0B930E0194E96F82400C0F10804AC42EA
:1019900028BF2C46E4B2A7003A46414606EB800039
:1019A000FFF7BEFFB944B8442D1BEDB296F82430C2
:1019B0001C44E4B286F82440082C0DD095B10B4BA2
:1019C00093F82430002BDDD10848C0F82090202265
:1019D000FF21FFF7B9FFD5E7FFF78AFF034600288D
:1019E000ECD100E001231846BDE8F883245D002017
:1019F00001207047704700BF704700BF10B5134605
:101A0000026814680022A04710BD00BF00F5805096
:101A100090F85904704700BF00F5805090F85204C8
:101A2000704700BF00F5805090F95804704700BF20
:101A30004E207047202383F3118862B600F5805250
:101A4000D2F89834D2F894041844D2F89034184458
:101A5000D2F878341844D2F888341844D2F8843450
:101A60001844002383F3118862B670472DE9F047CC
:101A700082B09846BDF828A000F5805393F8523400
:101A8000002B00F0D48005460C46914600F58052AC
:101A9000D2F874340133C2F874340B6813F0005F69
:101AA00048D10B7B082B02D94A7B002A42D00F2B4E
:101AB00040D8202383F3118862B6EB6AD3F8C420A0
:101AC00012F4001F40D1D3F8C470C7F304476A6A08
:101AD00007EBC706F10002EBC6062368002B3FDBCD
:101AE0009B045350236813F0804F03D0535843F0A6
:101AF00000535350227B3B0643EA02437360627BF0
:101B000092B343F44013736005F58052D2F8A434C5
:101B10000133C2F8A43405EB471241F268031344C1
:101B20001A7942F020021A71207B01F033F94FF04C
:101B3000000C31E005F58055D5F878340133C5F84F
:101B400078344FF0FF306FE005F58055D5F87C34E0
:101B50000133C5F87C34002080F3118862B663E05D
:101B600043F080435350BDE705EB471241F2680351
:101B700013441A796FF345121A71D5E7B3EBA20F2C
:101B80000FDA4FEA8C02083204EB83035B68B35030
:101B90000CF1010C5FFA8CFC6346C21CEED50332DB
:101BA000ECE7EA6A0123BB40C2F8D03005EB4712EC
:101BB00041F250031344C3F80090C3F8048041F28B
:101BC000580303EB4713E918D4F800C06668A0680F
:101BD00045F803C04E608860A3898B8141F268019B
:101BE000531818796AF300001871CAF34006C0B29E
:101BF00066F34100187157501A796FF382021A7117
:101C0000D2B242F010021A71D2B26FF3C3021A714B
:101C1000002383F3118862B6CDF800A04A464346FC
:101C20002146284601F078F802B0BDE8F0874FF071
:101C3000FF30F9E72DE9F84300F5805393F852544B
:101C4000002D40F008810446037C032B40F0048102
:101C500000231E469C4603E00CF1010C0133DBB26D
:101C600093420ADA01EBC30051F83370002FF3DB23
:101C700040680028F0DA0136F0E7202383F311886A
:101C800062B676B9E06AD0F8803043F00203C0F85B
:101C900080304E27002E52D0D4F814E000231E4688
:101CA00032E04D2E1AD8DFF8BCE1DEF80030370400
:101CB000E06A47EA8307C0F88470694818448000E6
:101CC00060613344CEF80030C6F14E07E06AD0F8C8
:101CD000803043F03003C0F88030DBE7E26A93697C
:101CE00023F00103936101F00FFA0646E36A9B6952
:101CF00013F0010F00F0AA8001F006FA801BFA2809
:101D0000F4D9A3E00133DBB29A4218DD01EBC3083A
:101D100051F833000028F5DBD8F80490B9F1000F32
:101D2000F0DA09F07F09DFF8488108EA004040EA6C
:101D3000090040F008404EF826000136E2E7BCF109
:101D4000000F0DD1E06AD0F8803043F00103C0F8F5
:101D50008030BCF1000F55D0A76900239E4644E0B7
:101D6000BCEB570F1AD2BCF1400F17D83D4F3B6860
:101D70004FEA0C40E66A40EA8300C6F8880038481B
:101D800018448000A06103EB4C033B60E06AD0F88C
:101D9000803043F00C03C0F88030DAE7E26A9369E0
:101DA00023F00103936101F0AFF90646E36A9B69F2
:101DB00013F0010F4AD001F0A7F9801BFA28F5D9DA
:101DC00044E020F06040DCF8046026F0604C4FEA0C
:101DD000CE0640F0005047F83E0004364CF000407C
:101DE000B8510EF1010E0133DBB29A420ADD01EB6C
:101DF000C30C51F833000028E3DBDCF80460002E4C
:101E0000DFDAF0E7174B1A68154B13449B00A36207
:101E1000154A934212D8E26A936923F00103936151
:101E200001F072F90646E36A9B6913F0010F08D0CE
:101E300001F06AF9801BFA28F5D907E00B4801F098
:101E40005DF904F58054012584F85254002383F38E
:101E5000118862B600E000252846BDE8F88300BF7F
:101E6000002B00105C5D0020FCB500406C570008A2
:101E70000000FF0708B5202383F3118862B600F540
:101E80008050406C00F0C8FF002383F3118862B6D5
:101E900008BD00BF70B504460D4641F244068059A6
:101EA00000F0C6FF1F2801D8002070BD202229465F
:101EB000A05901F039F8202814BF00200120F4E7D0
:101EC0002DE9F04188B005460E4617469846202376
:101ED00083F3118862B600220023CDE90023002499
:101EE000ADF8084003948DF818408DF8194004941B
:101EF000059441F24404005900F072FF1F280DD8E8
:101F0000002020B105F5805393F8523483B90020A6
:101F100080F3118862B608B0BDE8F08120226946DE
:101F2000285901F09BF8202814BF00200120E8E781
:101F300003AB07CB30607160B2601B88B381DDE911
:101F40000023C7E90023BDF80830A8F800300023BB
:101F500083F3118862B643463A463146284600F07C
:101F6000B3FED8E710B5394B0360002343608360AC
:101F70000446374B44F8303B23464FF07F0C0DE0CE
:101F80009FED307B83ED007B00221A81DA601A76A8
:101F90005A761A615A6120330CF1FF3CBCF1000FF4
:101FA000EEDA41F23002024400F580531C634FF434
:101FB00080545C6300249C63DC63012483F840400C
:101FC0005A6483F8484041F2500303444FF01F0E17
:101FD000BEF1000F11DB9C469FED1A7BACEC027B3F
:101FE00000229A608CF80C208CF80D20DA601A61BF
:101FF0009A6120330EF1FF3EEAE700F5805383F843
:1020000058140022A3F85A24A3F85C2483F85E2411
:1020100083F85F2483F86024A3F86224A3F864247F
:1020200083F8662483F8672483F86824012904D898
:10203000084B53F82130C36210BD074801F05EF829
:10204000AFF300800000000000000000045800080A
:10205000B8570008A85700089057000810B5044664
:10206000034B19784A1C1A70FFF77CFF204610BDFD
:10207000595D002000F58050012380F859347047E5
:1020800000297AD070B582B00C46434B994211D9E1
:102090000A234249B1FBF4FC013BDBB29E46581CCB
:1020A000BCFBF0F100FB11C131B1022B67D9013B40
:1020B000DBB2F3E71123ECE7BCFBF0F0411EB1F516
:1020C000806F5FD2C3EBC30E1EF1030150D4C1F386
:1020D000C70C8DF800C0A3EB0C05EDB28DF80150D4
:1020E0000CF101064FF47A710CFB0111354491FBA0
:1020F000F5F189B2ADF80210B1F5617F18D9BEF1E2
:10210000010E37D4CEF3C70E8DF804E0A3EB0E0317
:10211000DBB28DF805300EF101054FF47A710EFB3C
:1021200001112B4491FBF3F3ADF80630019B0093B2
:102130009DF800104B1C9DF80160334400FB03F335
:10214000164DB5FBF3F3A3421ED10139C9B20F29D5
:102150001CD8EEB1082E1DD8BDF80230138001380E
:102160005080002313715171013E9671012007E0E8
:102170000731ACE70EF1070EC4E7002070470020DE
:1021800002B070BD0020FBE70020F9E70020F7E770
:102190000020F5E70020F3E73F420F0000B4C4043D
:1021A00070B5C36A40F27772C3F8BC20C36A0722D5
:1021B000C3F8C820114C23689A00C16A42F4C022B7
:1021C000C1F8A0200E495A189200C26103F16C02B6
:1021D0002260950045F0E065C66AC6F8C0500A4422
:1021E00092004262EA3323600B449B008362054AFB
:1021F000934200D870BD044800F080FF5C5D002071
:10220000002B0010FCB500406C5700082DE9F0438E
:1022100089B0984600F5805393F85834022B00F2A9
:10222000768106460F469146BB4A52F82320002A83
:102230005CD0F76086F81080B84B1B78EBB9202390
:1022400083F3118862B6B64BD3F8EC2042F4807267
:10225000C3F8EC20D3F8942042F48072C3F89420A1
:10226000D3F8942022F48072C3F89420AB4B01225F
:102270001A70002383F3118862B606F5805393F831
:102280005134ABB9202383F3118862B606F580532D
:1022900093F85834A34AD35C63B3012B33D006F5CB
:1022A0008053012283F85124002383F3118862B6FE
:1022B000202383F3118862B6F26A936923F0100336
:1022C000936100F021FF0546F36A9C6914F008044D
:1022D00022D000F019FF401BFA28F5D9002484F31E
:1022E000118862B6204609B0BDE8F0838A4A42F8F8
:1022F00023009EE70221132001F0FCFF022115209C
:1023000001F0F8FFCBE70221142001F0F3FF0221D6
:10231000162001F0EFFFC2E79A6942F001029A61CC
:1023200000F0F2FE0546F36A9A6912F0010F05D13A
:1023300000F0EAFE401BFA28F5D9CFE79A6942F08F
:1023400002029A61F26A0023536583F3118862B630
:1023500006F58053586C00F05FFD1F2C2BD820220F
:1023600000216846FFF7F0FA002502958DF8145019
:102370008DF8155003950495069541F2500505EB2F
:10238000441506EB050EEC46BCE80F007051CEF884
:102390000410CEF80820CEF80C30BCE80700CEF8C8
:1023A0001000CEF81410CEF818209CF800308EF8EB
:1023B0001C300134D1E706F58053002283F8502405
:1023C00083F8532441F25A42324439463046FFF7EB
:1023D00057FE044600286CD006F58052C2F86C7493
:1023E00092F85E1492F85F341B0243EA416392F85C
:1023F00060140B43B2F85C14F26A43EA0143D36100
:10240000B9F1000F1AD041F26242324449463046D7
:10241000FFF736FE054600285FD006F58052C2F869
:10242000709492F8671492F868341B0143EA012310
:10243000B2F86414F26A43EA0143D360F36A0025F8
:10244000C3F8BC503046FFF7ABFE06F5805383F867
:102450005954F36A6FF040421A65F36A324A5A657A
:10246000F36A4FF002229A65F36A4FF0FF32C3F825
:10247000E020F36A0322DA65F26A936943F4407359
:102480009361B8F1030F3FF42DAFF26A936923F023
:102490000103936100F038FE0546F36A9B6913F06F
:1024A000010F2ED000F030FE401BFA28F5D9002491
:1024B00018E7F26A936923F00103936100F024FEA8
:1024C0000546F36A9B6913F0010F3FF40BAF00F070
:1024D0001BFE401BFA28F4D904E7F26A936923F043
:1024E0000103936100F010FE0446F36A9B6913F048
:1024F000010F0ED000F008FE001BFA28F5D92C467B
:10250000F0E606F58056012386F85234EAE6002408
:10251000E8E62C46E6E600BF505D0020585D00204E
:1025200000440258A457000855020002F0B589B0D3
:10253000054617461E4600240DE005F58053D3F8E6
:10254000543433B105F58052D2F89C340133C2F8CB
:102550009C340134E4B21F2C61D8EB6AD3F8D81054
:102560002046E14011F0010FF3D005EB441241F297
:102570006C039B5C13F0080FEBD105F58052D2F889
:1025800080340133C2F8803405EB441241F26C030D
:102590009B5C13F0200F06D005F58052D2F8A834CA
:1025A0000133C2F8A83405EB401341F26801194425
:1025B0000B7943F008030B71DBB213F0010FBCD0B1
:1025C00005F5805393F85334002BB6D00022002336
:1025D000CDE900230023ADF8083003938DF81830BF
:1025E0008DF819300493059341F2580303EB401022
:1025F00005EB000C03AB2858DCF80410DCF80820CD
:1026000007C3BCF80C201A80009701960123ADF88F
:1026100008302B681B6C6946284698478DE709B03F
:10262000F0BD00BF2DE9F0478CB005460E4600F026
:102630006FFD81468846002E5AD1EB6AD3F8A02060
:1026400012F4FE0F00F0BB80D3F8A42012F0007F3C
:1026500006D005F58051D1F894240132C1F89424B4
:10266000D3F8A42012F07F0F00F0AB80D3F8A43091
:10267000C3F3052AEF690AEBCA0307EBC30700237C
:1026800008938DF82C308DF82D3009930A933B6810
:1026900013F0804F4FD1C3F38A42089213F0005FCA
:1026A00003D0089B43F0804308937B6813F4001F1A
:1026B00048D001238DF82D3005F58052D2F8AC3486
:1026C0000133C2F8AC34FB8803F00F038DF82C30D3
:1026D00000249DF82C0000F05DFBA04236D93B1988
:1026E0001A7A0CAB234403F80C2C0134E4B2F0E763
:1026F000012E68D1EB6AD3F8B02012F4FE0F66D039
:10270000D3F8B42012F0007F06D005F58051D1F83F
:1027100094240132C1F89424D3F8B42012F07F0F2E
:1027200057D0D3F8B430C3F3052A2F6A0AEBCA0393
:1027300007EBC307A3E723F06042089242F0004290
:102740000892ABE700238DF82D30BCE746BBEB6A5F
:10275000C3F8A8A000220023CDE900230023ADF890
:10276000083003938DF818308DF8193004930593D1
:1027700003AC0CAB13E90F0007C42380CDF8009025
:10278000CDF804802B681B6C69462846984768B1D1
:1027900005F58055D5F88C340133C5F88C3413E039
:1027A000012ED7D1EB6AC3F8B8A0D3E705F5805561
:1027B000D5F890340133C5F89034012004E00020AE
:1027C00002E0002000E000200CB0BDE8F08700200F
:1027D000FAE70020F8E700BF38B504460D4604E0EC
:1027E00004F58053012283F8532429462046FFF73D
:1027F00019FF0028F4D104F58053D3F8543433B1D1
:1028000004F58054D4F89C340133C4F89C3438BDAA
:10281000C36A1A6C12F47F0F3BD01A6C00F5805318
:10282000C3F8A02400231F2B33DC10B402E00133D3
:102830001F2B2BDC00EB431141F26C02525C12F0B7
:10284000020FF4D041F26C02525C12F0040FEED190
:102850000A4641F26801515801228A40C16AD1F802
:10286000CC402242E3D0C1F8D42000EB431141F226
:1028700068020A44117941F00401117100F5805198
:10288000D1F888240132C1F88824D0E75DF8044BE0
:102890007047704708B5202383F3118862B6FFF7AD
:1028A000B7FF002383F3118862B608BDC36AD3F86B
:1028B000C02012F07C5F06D0D3F8C43013F4001FA0
:1028C00003D101207047002070470020704700BFEF
:1028D00008B5202383F3118862B600F58050406C60
:1028E00000F07EFA002383F3118862B61F288CBFA4
:1028F0000020012008BD00BF00F5805393F8593433
:1029000073B1C26A936923F00103936100F58050AB
:10291000D0F898340133C0F89834002380F8593443
:10292000704700BFF0B51C46202383F3118862B6C0
:10293000002100E001311F2936DC00EB411E41F28D
:102940006C0C1CF80EC01CF0040FF3D141F26C0C9F
:102950001CF80E3013F0100FECD0F44641F268036F
:102960005EF803500123AB40C56AD5F8CC60334212
:10297000E0D041F25006B6445CF80670DEF8046020
:102980009742A641D6D2C5F8D43041F268036344D9
:102990001D7945F004051D7100F58055D5F8843486
:1029A0000133C5F88434C5E7002383F3118862B688
:1029B000F0BD00BFF8B507460E4614461D4600237D
:1029C0001370FFF785FF80F0010333701DB13846A7
:1029D000FFF76CFF2070F8BD2DE9F04F83B0804603
:1029E0000F4691469B460C9EDDF834A00B78009371
:1029F0001378019300F08CFB04460D463B781BB91D
:102A000099F8000000284DD022462B464046FFF79B
:102A100089FF4046FFF73EFF4046FFF76DFF5B46EC
:102A20004A4639464046FFF7C5FF3B7813B1009B45
:102A3000002B32D199F8003033B1019B7BBB224689
:102A40001C462B46009D0CE02246019C2B46009D17
:102A500007E099F8003003B14CBB00F059FB024687
:102A60000B46B24273EB0A011BD208F58051D1F834
:102A70005404D0B10168C968B21A6AEB03038847ED
:102A80005B464A4639464046FFF794FF3B78002BA9
:102A9000DFD0002DDDD0009804E0009802E001981E
:102AA00000E0002003B0BDE8F08F0020FAE70198B5
:102AB000F8E700BF08B51B4B1B6853B31A4B1B6DDF
:102AC00013F0010F04D1184B1B6D13F0040F07D046
:102AD000154B05221A650021124B1868FFF77CFE82
:102AE000114B1B6D13F0100F04D10F4B1B6D13F026
:102AF000400F07D00C4B50221A650121094B186872
:102B0000FFF76AFE074B1868FFF782FE01F0C6FB6D
:102B100008BD054B01221A6510221A654FF4805238
:102B20001A65F3E7505D002000A0004008B51C4B7B
:102B30001B6883B11B4B1B6D13F4007F14D1194B21
:102B40001B6D13F0007F22D1154B1868FFF760FE54
:102B500001F0A4FB08BD134B01221A6510221A656F
:102B60004FF480521A65F3E70E4B4FF400721A656A
:102B700000F0CEFA02460B4652EA030102D0013AB7
:102B800043F1FF3306490868FFF7D0FCD7E7054B50
:102B90004FF000721A65024B1868FFF76BFAD3E723
:102BA000505D002000A0004008B51B4B5B6853B38C
:102BB0001A4B1B6D13F0010F04D1184B1B6D13F052
:102BC000040F07D0154B05221A650021124B5868D7
:102BD000FFF702FE114B1B6D13F0100F04D10F4BCA
:102BE0001B6D13F0400F07D00C4B50221A650121CA
:102BF000094B5868FFF7F0FD074B5868FFF708FED0
:102C000001F04CFB08BD054B01221A6510221A6524
:102C10004FF480521A65F3E7505D002000A4004095
:102C200008B51C4B5B6883B11B4B1B6D13F4007F15
:102C300014D1194B1B6D13F0007F22D1154B58682E
:102C4000FFF7E6FD01F02AFB08BD134B01221A65D0
:102C500010221A654FF480521A65F3E70E4B4FF4B9
:102C600000721A6500F054FA02460B4652EA03015C
:102C700002D0013A43F1FF3306494868FFF756FC9A
:102C8000D7E7054B4FF000721A65024B5868FFF703
:102C9000F1F9D3E7505D002000A400400FB40020FC
:102CA00004B0704710B5026854681A46A04710BDBA
:102CB00000207047002070470020704700207047B8
:102CC00000207047704700BF30B583B084460D4682
:102CD000043003C802AA02E9030069B10C461B884C
:102CE00013F0040F08D1DCF80030DB6B6046984726
:102CF0002A46C1B20098A047012003B030BD00BFF2
:102D000082B0EC468CE80600031D9CE8030083E8D3
:102D10000500012002B0704770B58AB004460E4627
:102D2000031D93E803000AAB03E9030069B10D46F4
:102D3000BDF8383013F0040F0AD12368DB6B20464E
:102D400098473246C1B20898A84701200AB070BD22
:102D500000220023CDE900230023ADF808300393BF
:102D60008DF818308DF819300493059303AB306853
:102D70007168B26807C3B2891A8000F0CDF9CDE955
:102D800000010423ADF8083023681B6C6946204617
:102D90009847DAE7082818D909280BD00A280BD059
:102DA0000B280BD00C280BD00D280BD00E280BD0E5
:102DB000402070470C207047102070471420704747
:102DC00018207047202070473020704710B5044607
:102DD000037C0BB1204610BD006802F0D1FBF9E77F
:102DE000BFF35B8FC368BFF35B8FBFF35B8F8268FA
:102DF000BFF35B8F9A4208D94268BFF35B8F80684C
:102E0000BFF35B8F101A18447047BFF35B8F806865
:102E1000BFF35B8F181A7047BFF35B8F0023C3604B
:102E2000BFF35B8FBFF35B8F8360BFF35B8F704734
:102E30000346406800B97047BFF35B8F9A68BFF3E1
:102E40005B8FBFF35B8FD968BFF35B8F914209D370
:102E50005868BFF35B8FDB68BFF35B8FD21A013A10
:102E60001044E8E70020F4E738B505460C46FFF7C4
:102E7000B7FFA04201D2002038BDBFF35B8FA96825
:102E8000BFF35B8F0C446968B4FBF1F301FB13449F
:102E9000BFF35B8FAC60BFF35B8F0120ECE700BF3B
:102EA00070B504460E461546FFF7C2FFA84200D390
:102EB000284608B9002070BD2368BFF35B8FE26825
:102EC000BFF35B8F134433606268BFF35B8FE368CB
:102ED000BFF35B8FD11A884207D971602168B16056
:102EE0009B1A1844F0600220E5E770600120E2E7D9
:102EF00038B505460C46FFF79BFFA04201D20020E3
:102F000038BDBFF35B8FE968BFF35B8F0C44696822
:102F1000B4FBF1F301FB1344BFF35B8FEC60BFF331
:102F20005B8F0120ECE700BF2DE9F04385B08146BF
:102F300088466946FFF7B4FF0746002425460EE0A1
:102F400004AB03EBC40656F80C2C08EB050156F84D
:102F5000100CFEF7E5FC56F80C3C1D440134A7426A
:102F6000EEDC29464846FFF7C3FF284605B0BDE81A
:102F7000F08300BFBFF35B8FC368BFF35B8FBFF30A
:102F80005B8F8268BFF35B8F9A4210D94368BFF3AF
:102F90005B8F8268BFF35B8F9B1A0B6073B1036812
:102FA000BFF35B8F8068BFF35B8F18447047BFF33C
:102FB0005B8F8268BFF35B8F9B1AEEE70020704740
:102FC000F0B583B007460E461546FFF709FF0446E5
:102FD0000190A84200D32C4614B9002003B0F0BDE4
:102FE00001A93846FFF7C6FF019B6BB1A34200D988
:102FF0000194306001987060A0420DD23B68B360CC
:10300000241AF4600220E9E73B683360746000230F
:10301000B360F3600120E1E70120DFE72DE9F04133
:1030200084B088466946FFF7CBFF07460024254653
:103030000EE004AB03EBC40656F80C2C56F8101C3B
:1030400008EB0500FEF76CFC56F80C3C1D440134FF
:10305000A742EEDC284604B0BDE8F08138B505464D
:10306000FFF7DCFF044601462846FFF7FDFE204639
:1030700038BD00BF00B59BB0EFF3098168226846F8
:10308000FEF74EFCEFF30583044B9A6BDA6A9A6AFB
:103090009A6A9A6A9A6A9A6A9B6AFEE700ED00E069
:1030A00000B59BB0EFF3098168226846FEF738FC53
:1030B000EFF30583044B9A6B9A6A9A6A9A6A9A6A42
:1030C0009A6A9B6AFEE700BF00ED00E000B59BB086
:1030D000EFF3098168226846FEF722FCEFF30583CF
:1030E000034B5A6B9A6A9A6A9A6A9A6A9B6AFEE7D3
:1030F00000ED00E0FEE700BFFEE700BF0FB408B53B
:10310000029801F003FAFEE708B501F02FFD08BDB3
:1031100008B501F005FD08BD08B5FFF7F9FF08BDCA
:1031200000B58E460AE040F3000C09490CEA0101A3
:1031300081EA50000133DBB2072BF4D91346013A80
:1031400023B11EF8013B58400023F5E75DF804FB6E
:103150002083B8ED401A83B2002800DB704703F1EA
:10316000200000B2FAE700BF03780133DBB203703E
:103170001F2B01D900230370704700BF082818D9FE
:1031800009280BD00A280BD00B280BD00C280BD009
:103190000D280BD00E280BD0402070470C20704714
:1031A0001020704714207047182070472020704767
:1031B00030207047082818D90C280BD910280BD9B3
:1031C00014280BD918280BD920280BD930280BD953
:1031D0000F207047092070470A2070470B20704766
:1031E0000C2070470D2070470E207047034621F0D9
:1031F000604C20F06042C00FB0EBD17F0FD00029AF
:1032000008DB002B09DB944519D094452CBF002026
:10321000012070474FEA9C4CF3E7920CF3E7C1F3AF
:103220008071C3F38070944514BF00230123814251
:1032300008BF00231BB994452CBF00200120704714
:103240002DE9F04107460D46D0F81C80B8F1000F7B
:103250000CD046464446A4B169686068FFF7C6FFD3
:1032600030B9236826465BB11C46F4E7F96108E0F3
:10327000A04502D035602C6003E02C60FD6100E0C9
:103280002560BDE8F08100BFC37DC3F38402013235
:1032900062F38603C375C38A6FF30903C382C37DD8
:1032A0006FF3C713C375704710F0800F04D010F48C
:1032B000004F03D001207047022070470020704764
:1032C00010B50446FFF7F0FF022802D0C4F3074010
:1032D00010BDC4F30F2014F07F0FF9D100F00300EC
:1032E000F6E700BF00E0006810B103698B42FAD135
:1032F000704700BF2DE9F043079CCE0803EBD405CF
:1033000001F0070304F007041A442AE003F0070859
:1033100004F00707C646B84538BFBE46CEF1080ED2
:10332000D11A8E4528BF8E464FF47F4C2CFA0EFCE6
:103330005FFA8CFC4CFA07FCD90800EB060919F877
:10334000011001FA08F1F940C9B24FEAD40815F8A2
:10335000087079400CEA01014F4005F80870734489
:1033600074449342D2D1BDE8F08300BF2DE9F04F01
:1033700087B004900E4605920393838AB1EBC30F86
:1033800080F088801146DA0031448A4204D2D2B2F9
:10339000F3B2D21AD3B20593049BDB683BB3272E5A
:1033A00036D8C6F12803059A9A422ED35FFA86FBD7
:1033B000CBF1280B5FFA8BFB00230093039B5A464B
:1033C000314604988068FFF795FF5E44059BA3EBA8
:1033D0000B04E4B204998A8A2F4B13444FEAC309C1
:1033E000D1F80C80282133464646984628E0049BB5
:1033F0001B69002BD3D100230093039B059A314610
:1034000004988068FFF776FF37E0DDF814B0D3E763
:10341000059C4FF0000BDDE72546CDF800B0039B7F
:103420002A46A8EB0101301DFFF764FFA844AB4416
:103430005FFA8BFB641BE4B2A9EB0A0936683946D4
:10344000002E18BF002C13D0CA46B9F1E00F28BFD8
:103450004FF0E00A0AEB0107B845EDD2A7EB0803ED
:103460009C42D9D3FDB25FFA88F3ED1AEDB2D4E7EE
:103470004646049B186900B124B9BDF9140007B091
:10348000BDE8F08FCDF800B0039B2246711AFFF71C
:1034900031FFF2E70020F2E7FBFFFF1F002070473B
:1034A0000139002307E0C25C10F801C000F803C036
:1034B0004254013301398B42F5D3704780EA012031
:1034C000002303E0400080B20133DBB2072B08D8B1
:1034D00010F4004FF6D0400081B241F22100484084
:1034E000F2E7704770B516461D46002411E0C4F19E
:1034F0002003A4F1200C26FA04F105FA03F3194382
:1035000025FA0CFC41EA0C01C9B2FFF7D7FF0834D9
:10351000A4B23F2CEBD970BD38B50C4604E014F8CA
:10352000011BFFF7CBFF2A46551E002AF7D138BDF5
:1035300007290BD938B505460C464FF6FF70FFF743
:10354000D1FF22462946FFF7E7FF38BD4FF6FF704F
:10355000704700BF10B48446002305E001EB43141C
:10356000CCF80040A44601339A42F7D80023CCF8A7
:1035700000308280C38003815DF8044B704700BF38
:103580000346006848B102681A60DA88013292B2D4
:10359000DA8019898A4200D91A81704708B5FFF785
:1035A000EFFF08B10023036008BD00BF2DE9F0471D
:1035B0008246894616461F46CB8AC3F30903052B6C
:1035C0002FD01846002407E0315D09EB0302D176C5
:1035D00001339BB20134A4B2042B02D8BAB2A24286
:1035E000F2D8BBB2A34213D9B9F81610C1F309013E
:1035F0004A1F93083B48A0FB0303C3EBC303A2EBA2
:1036000083031FFA83F8D9F8045065B1012318E049
:103610000344B9F8162063F30902A9F81620012023
:1036200054E00024E0E75046FFF7B8FF0546C9F82C
:10363000040000284CD04FF000082FE001339BB26B
:1036400015462A68002AF9D17A18053A92082549C0
:10365000A1FB021292B2013292B293422CBF00231C
:103660000123B8F1000F18BF0023BBB15046FFF78C
:1036700095FF286078B3054610E0325D05EB0C033A
:103680001A710CF1010C1FFA8CFC0134A4B2BCF1CC
:103690001B0F01D8A142F0D8A14204D8B9B2A1426F
:1036A0000AD9C446F3E75046FFF778FF2860A8B16F
:1036B00005464FF00008F1E7B9F81630C3F30902E8
:1036C000114461F30903A9F816300120BDE8F08721
:1036D0006FF00200FAE76FF00200F7E76FF0020008
:1036E000F4E700BF2549922403680B600160C3889A
:1036F000013BC380704700BF70B506460C4605E02D
:103700000D6806F10C00FFF7EFFF656061680029A6
:10371000F6D1E38A6FF30903E3820020002170BD34
:1037200008B5FFF72DFF034628B100220260426072
:103730008260C2600261184608BD00BF2DE9F04FEB
:1037400085B0019103930E9FBDF83C600292002A60
:1037500000F086808246331E18BF0123002F18BF59
:103760000023002B7FD1072E06D94FF0800B4FF09E
:1037700000094C46C8465FE00C30FFF7D1FF044615
:10378000002873D0324639460830FEF7C9F8701C5D
:10379000C0B2FFF70FFDFFF7F1FC83B2013B2074CD
:1037A000029A127802F01F0242F0C00214FA83F368
:1037B0001A72019B43F00043636021465046FFF7B5
:1037C0003FFD4FF00108404605B0BDE8F08F3A5D7F
:1037D0002B441A720130C0B20134A4B20346062849
:1037E00001D8B442F3D3B44237D00130C0B2FFF7AE
:1037F000E1FCFFF7C3FC421E4FEA4913DBB243EA88
:103800000B0B029B1B7803F01F034BEA030B55FACB
:1038100082F383F808B0019B43F000436B60287487
:1038200029465046FFF70CFD08F101080FFA88F809
:1038300089F001094FF0000BB442C4D00AF10C002A
:10384000FFF76EFF0546A0B12CB9039B03721B0A5C
:1038500043720220C2E70020C0E74FF0400BC4E7EC
:103860006FF00108AFE76FF00108ACE76FF00208F6
:10387000A9E76FF00208A6E730B589B004460D4607
:10388000202200216846FEF75FF804952046FFF7E6
:1038900077FE8646A0B1EC46BCE80F00CEF80000EB
:1038A000CEF80410CEF80820CEF80C30BCE80F009B
:1038B000CEF81000CEF81410CEF81820CEF81C3038
:1038C000704609B030BD00BF10B504460C30FFF79C
:1038D000D3FF034610B1A2690260A061184610BD73
:1038E00038B504460D46806918B1FFF7FBFC40B1BE
:1038F00038BD04F10C00FFF7BFFF0028F8D0A0612D
:10390000F6E729462046FFF7DFFFF1E7F8B5044662
:103910000E4615461F4628220021FEF715F8A7601F
:10392000069B6360079B23626A09B5F5001F01D3FC
:103930004FF6FF7292B2314604F10C00FFF70AFE17
:10394000F8BD00BF03781BB94BB2002B00DD01703E
:10395000704700BF007870472DE9F04F83B09A465A
:10396000BDF830409DF838900F9FBDF84060B7FA21
:1039700087F35B09002E08BF0023002B3FD10546CB
:103980009046B9F11F0F3DD8FFF7E4FF8346D8B941
:10399000072E3AD834F003033AD1324639464FF66F
:1039A000FF70FFF7B9FD20F001004004400C400219
:1039B00040EA0969240204F4407449EA040949EA26
:1039C0000B0B4FF6FF730BE0240244EA096949EA46
:1039D000000B4246534631463846FFF7A9FD0346E1
:1039E000019600970D9A59462846FFF7A7FE044610
:1039F0000D98FFF7B9FB204603B0BDE8F08F6FF0DC
:103A00000104F8E76FF00104F5E76FF00304F2E753
:103A10006FF00104EFE700BF2DE9F04F83B01E46C1
:103A20009DF838409DF83CA0DDF84080BDF84490FA
:103A3000B8FA88F35B09B9F1000F08BF00237BBB1C
:103A400005468B4617461F2C2DD8FFF783FF68B31A
:103A50009DF830301B0443EA046444EACA3444EA63
:103A60000B24044344F080043A463346494640461A
:103A7000FFF75EFD0346CDF80490CDF800800D9A67
:103A800021462846FFF75AFE0446BAF1010F03D03B
:103A9000204603B0BDE8F08F0D98FFF765FBF7E710
:103AA0006FF00104F4E76FF00104F1E76FF0030435
:103AB000EEE700BFC06900B10430704708B5C169C6
:103AC0000B68C3610C30FFF70FFE08BD2DE9F04114
:103AD00005461646984687693C4610E0214628462A
:103AE000FFF70AFEAB691B68AB61214605F10C00CC
:103AF000FFF7FAFDAC69274601E027462468DCB1F0
:103B0000A168E368711A68EB03030C4A8A424FF01C
:103B1000000272EB0303F0D2AB69A342DED0214670
:103B20002846FFF7E9FD23683B60214605F10C00BC
:103B3000FFF7DAFD3C68E2E7BDE8F08180841E0013
:103B40002DE9F04182B0089E002E18BF002800F039
:103B5000DE8014461D46531EDBB23F2B00F2DA8096
:103B6000012A14BF002305F00103002B40F0D5808B
:103B7000009301936B46FFF7F9FB071E3BDD14F042
:103B8000070F0AD002AB03EBD40111F8083C6242E4
:103B900002F00702134101F8083C012C0BD0082C5D
:103BA0002DD9102C2ED9202C2FD9402C00F2B880E2
:103BB0004FF0080800E0A046FFF770FC40BB9DB145
:103BC000B4EBC80F10D0082C27D89DF80020631E36
:103BD00022FA03F313F0010F06D00123A3405B4246
:103BE000DBB213438DF80030002D72D0082C5ED864
:103BF0009DF900303370384602B0BDE8F0814FF0D7
:103C00000108D9E74FF00208D6E74FF00408D3E7E0
:103C100041466846FFF744FCD1E7102C0FD8BDF8A9
:103C20000020631E22FA03F313F0010FDCD00123FE
:103C3000A3405B429BB21343ADF80030D4E7202C85
:103C40000CD8009A631E22FA03F313F0010FCBD0B5
:103C50000123A3405B421A430092C5E73F2C62D880
:103C60000098019A631EC4F1210CA4F1210120FAED
:103C700003F302FA0CFC43EA0C0322FA01F10B43B2
:103C800013F0010FB0D00123A4F12001C4F1200CE6
:103C900003FA01F123FA0CFC41EA0C01A3405B4258
:103CA00061EB410103430A43009301929CE7102C0E
:103CB00003D8BDF9003033809DE7202C02D8009B4B
:103CC000336098E7402C31D8DDE90023C6E90023B2
:103CD00091E7012C05D0082C07D89DF800303370EF
:103CE00089E79DF80030337085E7102C03D8BDF8C4
:103CF000003033807FE7202C02D8009B33607AE7C6
:103D0000402C16D8DDE90023C6E9002373E76FF0E5
:103D1000010770E76FF001076DE76FF001076AE7D1
:103D20006FF0080767E76FF0080764E76FF00807B0
:103D300061E76FF008075EE7F0B585B005460E460F
:103D4000402A03D8144612B9012400E0402400227E
:103D500002920392012C06D0082C22D81B788DF8F1
:103D60000830012703E01B788DF808302746FFF75D
:103D700095FB68BB14F0070F0AD004AB03EBD4012A
:103D800011F8083C624202F00702934001F8083C37
:103D900000962B462246002102A8FFF7ABFA05B099
:103DA000F0BD102C04D81B88ADF808300227DEE7E0
:103DB000202C03D81B6802930427D8E7402C05D891
:103DC000D3E90023CDE902230827D0E70027CEE777
:103DD000394602A8FFF764FBCCE700BF70B5064682
:103DE0000C4605E00D6806F10C00FFF77DFCE56070
:103DF000E1680029F6D10023E360A3602361A38278
:103E000070BD00BF2DE9F04F99B006460D460592F2
:103E100004930F683846FFF747FA8346022800F0FC
:103E20008880C7F30628002F80F2E08117F0C04F8A
:103E300040F0DF812C7B002C00F0DE81BBF1020F13
:103E400005D03046FFF786FD404540F0D881C7F3E6
:103E500004630B9307F07F0106913846FFF730FAB1
:103E60000C9040EA0B47069947EA814747EA4867C2
:103E7000013C2C4494F8049000220023CDE9162341
:103E80005FEAD913029357D0746800915B460246EB
:103E900016A93046A047002800F0B48139463046C4
:103EA000FFF71EFD0446002800F0AF81A768E36815
:103EB00057EA03020CBF0122002207920599CF1B8B
:103EC000049961EB0308904B9F4278F100032CBFEB
:103ED0000123002308936A7BA37E9A4214BF00202B
:103EE00001200A90029B099394F817A0CAF3840A50
:103EF00009F01F0CCDF80CC061465046FFF72AF9B7
:103F00000D90824B9F4278F100072CBF01270027BC
:103F100051460398FFF71EF9079A089911431CD1DF
:103F20000A9A099B1A4211D00D9B012B0EDD012329
:103F300014E04FF0000876E73946B069FFF7D2F990
:103F400004460028B2D16FF00C0062E1099B3B42AD
:103F500055D00F2855DD002300E00123002B52D15E
:103F60006A7BA37E9A4240F05381029B13B119F001
:103F7000400F63D1C9F34013E27DB3EBD21F40F091
:103F80004B81C2F38403039A9A4240F04881029B1A
:103F9000002B00F08C8019F0400F40F088802B7BC4
:103FA000032B40F23F81059BA360049BE360AF1DA0
:103FB0002B7B033BDBB23A46214606F10C00FFF7B0
:103FC000F5FA00286ADB2B796A7943EA0223238316
:103FD000DDE916234FF6FF70FFF784FAA0822A7BF3
:103FE000033AD2B23946FFF797FAA082E37DDA436B
:103FF000C2F3C01262F3C713E375002009E1002386
:10400000ACE70123AAE7E37D69F38603E375DBB23E
:104010006FF3C713E37521463046FFF76DFB6B7BEB
:10402000A376029B002B9BD1E37DC3F38402013274
:1040300062F38603E3756FF00C00EAE0059FA7606A
:10404000049BE360202200210EA8FDF77DFC0E9763
:10405000049B0F932B1D10932B7B013BDBB2ADF820
:104060004C300C9BADF84E308DF850B0039B8DF862
:1040700051300B9B8DF85230069B8DF8533096F8DB
:10408000243083F001038DF85430B3680EA9304614
:1040900098472046FFF7F8F80020BAE0214630465E
:1040A000FFF72AFB2046FFF7EFF80320B1E0029B61
:1040B00013B919F0400F09D0297B0139C9B2E28A3E
:1040C000C2F30902042A6FD8002328E02F1D2B7B9E
:1040D000013BDBB23A46214606F10C00FFF766FAD7
:1040E000002808DB2A7B013AD2B23946A08AFFF7C2
:1040F00013FAA0827AE721463046FFF7FDFA204600
:10410000FFF7C2F8032084E081841E0041420F00C3
:10411000E8180779A018C77601320133DBB2042A08
:1041200098BF8B42F4D3059A0E92049A0F9204F131
:104130001B021092626811928B424ED22B440433C0
:104140001293E38AC3F309031944ADF84C100C9B96
:10415000ADF84E308DF850B0039B8DF851300B9B6D
:104160008DF85230069B8DF8533096F8243083F04A
:1041700001038DF85430002363602A7B013A291D26
:10418000A08AFFF7C9F9A082238B984227D00EA9F5
:104190003046FFF723FE2046FFF776F8A28A238BEE
:1041A0009A4221D0112034E0606828B105270368C5
:1041B00023B11C371846FAE70023B4E7D21B1B2AA9
:1041C00098BF8B42AFD2EF1897F804C0871887F8D2
:1041D00004C001320133DBB2F1E70023B0E7B3687A
:1041E0000EA930469847D2E7002012E06FF0090090
:1041F0000FE06FF009000CE06FF0090009E06FF0CC
:104200000A0006E06FF00B0003E06FF0020000E030
:10421000002019B0BDE8F08F6FF00D00F9E76FF0E6
:104220000E00F6E76FF00F00F3E700BFEFF309832E
:10423000683305494A6B22F001024A6383F3098817
:10424000002383F31188704700EF00E0202080F303
:10425000118862B60D4BD96821F4E0610904090C9C
:104260000B4A0A43DA60D3F8FC2042F08072C3F8AC
:10427000FC20084A0849C2F8B01F116841F001014A
:1042800011601022DA7783F82200704700ED00E019
:104290000003FA05001000E055CEACC5202383F3DF
:1042A0001188104B5B6813F4006F03D1002383F374
:1042B0001188704710B5F1EE103AEFF30984683CAD
:1042C0004FF08073E361084BDB6B236684F309884E
:1042D00000F0B8F810B1054BA36110BD044BA36109
:1042E000FBE700BF00ED00E000EF00E00B07000877
:1042F0000E0700080901C9B2074A131883F8001312
:1043000000F01F01400901238B4000F1600142F8D9
:10431000213042F82030704700E100E0024B1B6082
:104320005B6000229A607047645D00200023037484
:10433000054B1B68996882689142FAD203605A68FB
:104340004260106058607047645D002008B520230B
:1043500083F31188037C032B0ED0042B10D043B1C0
:104360004FF0FF334361FFF7E1FF002383F3118830
:1043700008BD83F31188FBE7436900221A60EFE769
:1043800042680368136042685A60E9E700230374D7
:10439000054B1B68996882689142FAD803605A6895
:1043A0004260106058607047645D002008B5074B9C
:1043B000196908741A681068186043601A6101204E
:1043C00010741869FCF78CF908BD00BF645D00200B
:1043D00010B586B00446B1F1FF3F12D00A4B1B69FD
:1043E0000A4A01A800F054F92046FFF7DFFF049BBA
:1043F00013B101A800F05CF9034B1B69586906B0C2
:1044000010BDFFF7D3FFF7E7645D00204D430008C0
:1044100010B504460A4B18696161A26883689A4224
:1044200003D82046FFF782FF10BDFFF7AFFF01461C
:10443000034B1C61012323742046FCF751F9F3E779
:10444000645D0020044B1A6890681B699B68984261
:1044500094BF002001207047645D002010B5084C17
:10446000206923681A6822605460236101221A744B
:10447000FFF78CFF01462069FCF732F910BD00BF41
:10448000645D002008B5054B1A6892681B699B683B
:104490009A4200D808BDFFF7E1FFFBE7645D00200A
:1044A00010B5084C206923681A68226054602361A3
:1044B00001221A74FFF76AFF01462069FCF710F920
:1044C00010BD00BF645D0020FEE700BF10B5FFF720
:1044D00025FF00F0CFF80A4C80220A49204600F060
:1044E00047F844F8180C01230374FFF7AFFE0023CC
:1044F00083F3118862B6044800F058F810BD00BF7D
:104500008C5D0020485800085858000808B572B65D
:10451000034B586200F0ECFA00F0CEFBFEE700BF60
:10452000645D002008B500F003F908BDEFF31180C9
:1045300058B9EFF30583C3F308031BB1202383F3BA
:1045400011887047202383F31188704778B908B524
:10455000EFF30583C3F308031BB1002383F3118832
:1045600008BDFFF78FFF002383F31188F8E770473A
:1045700082600222027400224274704710B584687F
:10458000A4F17C0344F80C3C026944F83C2C4269D9
:1045900044F8382C044A44F81C2CC2680168A4F181
:1045A0001800FFF7E5FF10BDF906000810B520233D
:1045B00083F31188FFF7E2FF04460021FFF728FF8D
:1045C000002383F31188204610BD00BF08B5034BBC
:1045D0001B6958610F20FFF7E9FE08BD645D0020EC
:1045E00008B5202383F31188FFF7F0FF08BD00BF53
:1045F00008B50146202383F311880820FFF7E8FE61
:10460000002383F3118808BD70B505460E461C468D
:104610000368984209D0C068121AA21800D2144642
:104620009B68A34210D82A6814E0C2608C60706056
:1046300003680B6059602960092C00D80A24E868D7
:10464000204400F0C9FB14E0204400F0D5FBEAE769
:10465000E41A126893689C42FAD8B46032605368D6
:1046600073601E60566093681B1B93604FF0FF33AE
:10467000AB6070BD054B03F114025A619A614FF0B3
:10468000FF32DA6100221A62704700BF645D0020C9
:1046900038B504460D460361C26000F0B3FB024624
:1046A0002B4621460148FFF7AFFF38BD785D00205B
:1046B00038B51E4B5B69984210D04268036813609E
:1046C00042685A600023C3600268816893680B44A3
:1046D0009360164B4FF0FF32DA6138BD1968134A08
:1046E000134643F8141F4B600021C16052699A427F
:1046F00018D0816893680B4493600C4D2C6A00F0CD
:1047000081FB021B6B699B689342E6D9241A1C4407
:10471000092C01D802F10A03044A106A184400F077
:104720006BFBDAE700F062FBD7E700BF645D0020B7
:1047300038B507E0002383F311882069A8472023B8
:1047400083F31188144D6C6900F05CFB2B6AC21A6C
:10475000A168914211D819442B46296261682268E8
:104760000A6061685160E5680022E26053F8142F26
:104770009A42DFD100F03AFBDCE7074A52F8144FC7
:10478000944207D01A1A0A44092A00D80A2210446F
:1047900000F032FB38BD00BF645D00200020704790
:1047A000FEE700BF704700BF4FF0FF30704700BF0B
:1047B000BFF34F8F054B1B6913F0070FFAD1034B63
:1047C000D3F8103113F0070FF4D1704700200052D6
:1047D000034B4FF0FF325A61C3F81421704700BFFA
:1047E0000020005208B5104B1B7803B108BDFFF73D
:1047F000DFFF0E4BDB6813F0010F05D00B4B0C4AAB
:104800005A6002F188325A60084BD3F80C3113F029
:10481000010FEBD0054B064AC3F8042102F18832A0
:10482000C3F80421E2E700BF205F0020002000520F
:1048300023016745002301E0043001338B4205D298
:104840000268B2F1FF3FF7D00020704701207047A7
:104850002DE9F04105460E4600F17843B3F5801F7F
:104860000FD2184CDFF86C80174FFFF7A1FF4FF005
:10487000FF33C8F800303B6843F002033B6000227E
:104880000EE0124CDFF85080114FEEE7236813F072
:10489000050FFBD156F8043B45F8043B0132D2B278
:1048A000072AF3D9BFF34F8FFFF782FF4FF0FF3393
:1048B000C8F800303B6823F002033B600120BDE8EC
:1048C000F08100BF102000520C2000521021005235
:1048D0000C210052142000521421005208B5144B30
:1048E0001B781BBB134B1B6913F0040F04D0114A38
:1048F000D36843F04003D3600E4BD3F8103113F06C
:10490000040F06D00B4AD2F80C3143F04003C2F832
:104910000C31FFF74DFF074BDA6842F00102DA6015
:10492000D3F80C2142F00102C3F80C2108BD00BFEE
:10493000205F0020002000522DE9F84312F01F0FE5
:1049400035D104460D46164610F01F0F01D0002742
:104950002EE0FFF747FF02E02034203E20351F2ED7
:1049600021D920222146284600F012FE0028F3D04B
:1049700008212046FFF75EFF0746C8B1FFF7D6FDC6
:10498000814629462046FFF763FF07464846FFF762
:10499000DDFD4FB120222946204600F0F9FD002818
:1049A000DAD0002700E00127FFF798FF00E000279A
:1049B0003846BDE8F88300BF0F2803D800F58060B3
:1049C00040047047002070474FF40030704700BF2C
:1049D000102070470F2811D838B50546FFF7ECFFB7
:1049E00004462846FFF7F0FF30B12368B3F1FF3FDC
:1049F00006D104380434F7E7012038BD00207047A1
:104A00000020FAE70F2801D90020704770B504464E
:104A1000FFF78CFD0546FFF7CBFEFFF7E3FEFFF740
:104A2000D7FE072C28D8224E4FF0FF333361FFF713
:104A3000BFFE230243F02403F360F36843F08003D6
:104A4000F3601B4B1B6913F0040FFAD1FFF7B0FEA4
:104A50002046FFF7B1FF06462046FFF7B5FF0146A7
:104A6000304600F005F9FFF739FF2846FFF76EFDE5
:104A70002046FFF7AFFF70BD0D4E4FF0FF33C6F875
:104A80001031FFF795FEA4F108031B0243F0240345
:104A9000C6F80C31D6F80C3143F08003C6F80C315F
:104AA000034BD3F8103113F0040FF9D1CEE700BF58
:104AB0000020005208B5FFF73FFF08BD08B50346C8
:104AC00010B10A4A127822B113B9084B1B7833B9D6
:104AD00008BDFFF787FE054B01221A70F8E7034B6C
:104AE00000221A70FFF7FAFEF2E700BF205F0020F5
:104AF00010B500240BE0074804EB44039A0013466A
:104B000003445968805800F0C5F80134E4B2052C1C
:104B1000F1D910BD7058000808B500F073F908BD50
:104B200070B5104E82B0FFF701FD0546FFF7F4FFA8
:104B30003268034690420ED30B49D1E900411C195B
:104B40002846336041F100010191FFF7FFFC204648
:104B5000019902B070BD044A516814680131516076
:104B6000EDE700BF245F0020285F002070B5124EE3
:104B700082B0FFF7DBFC0546FFF7CEFF3268034645
:104B8000904213D30D49D1E900411C1928463360E6
:104B900041F100010191FFF7D9FC4FF47A72002333
:104BA00020460199FBF784FB02B070BD034A5168AF
:104BB000146801315160E8E7245F0020285F00207D
:104BC00009E000F1010C064A52F8202041F8042BBC
:104BD0001A465FFA8CF0531EDBB2002AF1D17047FF
:104BE0005040005810B4114B1B6F13F4004F06D106
:104BF0000E4B1C6F1C671C6F44F400441C670C4C6C
:104C0000236843F48073236009E000F1010C51F83C
:104C1000044B084A42F820401A465FFA8CF0531EB3
:104C2000DBB2002AF1D15DF8044B70470044025812
:104C3000004802585040005800B583B0012201A935
:104C40000020FFF7BDFF019803B05DF804FB00BF33
:104C500010B582B00446FFF7EFFFA04201D102B0C9
:104C600010BD0194012201A90020FFF7BBFFF6E768
:104C70000144BFF34F8F03E0054BC3F85C022030C3
:104C80008842F9D3BFF34F8FBFF36F8F704700BFD8
:104C900000ED00E00144BFF34F8F03E0054BC3F884
:104CA000700220308842F9D3BFF34F8FBFF36F8F6C
:104CB000704700BF00ED00E0704700BF034B1B785A
:104CC0001BB1034B4AF6AA221A607047345F0020DA
:104CD00000480058044B1B6823B9044BD3F8D02478
:104CE000014B1A60704700BF305F0020004002583F
:104CF000024B4FF48032C3F8D02470470040025872
:104D000008B5FFF7E7FF024B1868C0F3806008BDE5
:104D1000305F002010B4BFF34F8FBFF36F8F1C4B79
:104D20000021C3F85012BFF34F8FBFF36F8F5A6942
:104D300042F400325A61BFF34F8FBFF36F8FC3F855
:104D40008410BFF34F8FD3F88040C4F34E3000E09F
:104D50001846C4F3C90243F6E07303EA401343EA7A
:104D600082730B49C1F860321346013A002BF2D12D
:104D7000431E0028ECD1BFF34F8F4B6943F48033BF
:104D80004B61BFF34F8FBFF36F8F5DF8044B7047DC
:104D900000ED00E0FEE700BF084B094903E051F8D1
:104DA000042B43F8042B074A9342F8D302E0002275
:104DB00043F8042B044A9342F9D37047C05F0020A4
:104DC000785A0008C05F0020C05F0020704700BF15
:104DD00008B500F0DBF808BD034B586300221A61E8
:104DE0000222DA60704700BF000C0040014B002235
:104DF000DA607047000C0040014B5863704700BFF9
:104E0000000C0040014B586A704700BF000C004086
:104E10004B6843608B688360CB68C3600B694361F8
:104E20004B6903628B6943620B680360704700BF84
:104E300010B52A4BD3F8882040F2FF710A43C3F81B
:104E40008820D3F88800264A0240C3F88820D3F887
:104E50008820D3F8E0200A43C3F8E020D3F80821E3
:104E60000A43C3F80821D3F808311E4C21461E48D6
:104E7000FFF7CEFF04F11C011C48FFF7C9FF04F146
:104E800038011B48FFF7C4FF04F154011948FFF72C
:104E9000BFFF04F170011848FFF7BAFF04F18C015D
:104EA0001648FFF7B5FF04F1A8011548FFF7B0FF5A
:104EB00004F1C4011348FFF7ABFF04F1E00112480D
:104EC000FFF7A6FF04F1FC011048FFF7A1FF04F56E
:104ED0008C710F48FFF79CFF10BD00BF00440258C3
:104EE00000F8FFFFB85800080000025800040258FC
:104EF00000080258000C0258001002580014025812
:104F000000180258001C02580020025800240258C1
:104F10000028025808B5FFF78BFF00F0EFF8064BAA
:104F20000522C3F898204FF06052C3F89C20034A32
:104F3000C3F8A02008BD00BF00ED00E01F0008037B
:104F400008B500F0EDFAFFF7C1FA0D4BD3F8DC20FD
:104F500042F04002C3F8DC20D3F8042122F04002E2
:104F6000C3F80421D3F80431064B1A6842F0080252
:104F70001A601A6842F004021A60FFF7ABFE08BD1F
:104F80000044025800180248704700BF114BD3F884
:104F9000E82042F00802C3F8E820D3F8102142F0DC
:104FA0000802C3F81021D3F810310B4AD36B43F039
:104FB0000803D363094BC7229A624FF0FF32DA62CB
:104FC00000229A615A63DA605A6001225A611A60BB
:104FD000704700BF004402580010005C000C004005
:104FE00008B50A4A1369D168C9B20B40D9431161A7
:104FF00013F0020F00D108BD202383F31188FFF7BF
:1050000091FA002383F31188F5E700BF000C0040FC
:1050100010B5384BD3F880204FF0FF31C3F8801023
:10502000D3F880200022C3F88020D3F88000D3F882
:105030008400C3F88410D3F88400C3F88420D3F824
:105040008400D86F40F0FF4040F4FF0040F43F5030
:1050500040F03F00D867D86F20F0FF4020F4FF00F9
:1050600020F43F5020F03F00D867D86FD3F8884035
:1050700021482043C3F88800D3F88800C0F30A0011
:10508000C3F88800D3F88800D3F89000C3F89010D4
:10509000D3F89000C3F89020D3F89000D3F8940090
:1050A000C3F89410D3F89400C3F89420D3F8940074
:1050B000D3F89800C3F89810D3F89800C3F8982054
:1050C000D3F89800D3F88C00C3F88C10D3F88C0078
:1050D000C3F88C20D3F88C00D3F89C00C3F89C1044
:1050E000D3F89C10C3F89C20D3F89C3000F0F2F960
:1050F00010BD00BF0044025800F8FFFF6B4B0122B7
:10510000C3F808216A4BD3F8F42042F00202C3F836
:10511000F420D3F81C2142F00202C3F81C21D3F87A
:105120001C31644B0422DA60624B5B6813F4005F4D
:10513000FAD0604B604A1A6001229A605F4ADA60D6
:1051400000221A614FF440429A615A4B9B6913F452
:10515000005FFAD0574A136843F480731360544BCE
:105160001B6F13F4407F05D0514B4FF480321A6708
:1051700000221A674E4A136843F0010313604C4B38
:105180001B6813F0040FFAD0494B00221A61484BF8
:105190001B6913F0380FFAD1454B01221A604FF00A
:1051A00080425A6000225A67454ADA62454A1A61CB
:1051B0001A6842F480321A603D4B1B6813F4003FBA
:1051C000FAD03B4A136843F480531360384B1B6892
:1051D00013F4005FFAD0364B3B4A9A6200225A63BE
:1051E0003A491963DA633A4999635A64394A1A6445
:1051F000394ADA621A6842F0A8521A602C4B1B68CE
:1052000003F02853B3F1285FF8D1294B48229A6163
:105210004FF48862DA6140221A62304ADA644FF051
:1052200080521A652E4A5A652E4A9A652E4B3222B2
:105230001A602D4B1B6803F00F03022BF9D11C4A97
:10524000136943F003031361194B1B6903F038031F
:10525000182BF9D1164BD3F8DC2042F00052C3F8DA
:10526000DC20D3F8042142F00052C3F80421D3F823
:105270000421D3F8DC2042F08042C3F8DC20D3F8CC
:10528000042142F08042C3F80421D3F80421D3F86A
:10529000DC2042F00042C3F8DC20D3F8042142F0C5
:1052A0000042C3F80421D3F8043170470080005154
:1052B000004402580048025800C000F004000001F9
:1052C0000000FF010088900832206000630209019D
:1052D0001D02040047040508FD0BFF01200000200B
:1052E0000010E000000101000020005208B54FF05E
:1052F000B042D2F8883003F00103C2F888302BB1F5
:10530000044B1B6813B1034A50689847FEF7C6FF69
:1053100008BD00BF385F002008B54FF0B042D2F89A
:10532000883003F00203C2F888302BB1044B9B682D
:1053300013B1034AD0689847FEF7B0FF08BD00BF1D
:10534000385F002008B54FF0B042D2F8883003F043
:105350000403C2F888302BB1044B1B6913B1034A14
:1053600050699847FEF79AFF08BD00BF385F0020DC
:1053700008B54FF0B042D2F8883003F00803C2F805
:1053800088302BB1044B9B6913B1034AD06998470D
:10539000FEF784FF08BD00BF385F002008B54FF05E
:1053A000B042D2F8883003F01003C2F888302BB135
:1053B000044B1B6A13B1034A506A9847FEF76EFF0D
:1053C00008BD00BF385F002010B54FF0B043D3F8E0
:1053D000884004F47872C3F8882014F0200F05D0B8
:1053E000164B9B6A13B1154AD06A984714F0400FC8
:1053F00005D0124B1B6B13B1104A506B984714F039
:10540000800F05D00D4B9B6B13B10C4AD06B9847A6
:1054100014F4807F05D0094B1B6C13B1074A506C04
:10542000984714F4007F05D0044B9B6C13B1034ADA
:10543000D06C9847FEF732FF10BD00BF385F0020E8
:1054400010B54FF0B043D3F8884004F47C42C3F861
:10545000882014F4806F05D01A4B1B6D13B1194AC4
:10546000506D984714F4006F05D0164B9B6D13B127
:10547000144AD06D984714F4805F05D0114B1B6E11
:1054800013B1104A506E984714F4005F05D00D4BCD
:105490009B6E13B10B4AD06E984714F4804F05D021
:1054A000084B1B6F13B1074A506F984714F4004F15
:1054B00005D0044B9B6F13B1024AD06F9847FEF79B
:1054C000EDFE10BD385F002008B5FFF789FDFEF73F
:1054D000E5FE08BD08B506210846FEF70BFF0621CC
:1054E0000720FEF707FF06210820FEF703FF06212D
:1054F0000920FEF7FFFE06210A20FEF7FBFE06212B
:105500001720FEF7F7FE06212820FEF7F3FE0921FB
:105510007A20FEF7EFFE07213220FEF7EBFE08BDF2
:1055200008B5FFF775FD00F005F8FFF72DFDFFF753
:105530004FFC08BD002307E0054A002142F8331064
:1055400002EBC302516001330F2BF5D9704700BF46
:10555000385F00200B460146184600F003B80000F3
:1055600000F00EB810B5054C13462CB10A460146A2
:105570000220AFF3008010BD2046FCE700000000D1
:10558000024B0146186800F035B800BF1C2200200D
:1055900010B501390244904201D1002005E00378A2
:1055A00011F8014FA34201D0181B10BD0130F2E7E2
:1055B0002DE9F041A3B1C91A17780144044603F15B
:1055C000FF3C8C42204601D9002009E00578BD420D
:1055D00004F10104F5D10CEB0405D618A54201D164
:1055E000BDE8F08115F8018D16F801EDF045F5D014
:1055F000E7E7000037B5002944D051F8043C01909A
:10560000002BA1F10404B8BFE41800F03FF81E4AD3
:105610000198136833B96360146003B0BDE830408B
:1056200000F03AB8A34208D9256861198B4201BF3E
:1056300019685B6849192160EDE71A465B680BB190
:10564000A342FAD911685518A5420BD12468214408
:105650005418A3421160E0D11C685B685360214478
:105660001160DAE702D90C230360D6E725686119D7
:105670008B4204BF19685B68636004BF49192160ED
:105680005460CAE703B030BDB85F0020014800F0A5
:1056900009B800BFBC5F0020014800F005B800BF9A
:1056A000BC5F00207047000070470000636F6D2EE4
:1056B0006375626570696C6F742E68657265332BF3
:1056C000000000004E6F20617070207369670A004F
:1056D000426164206677206C656E6774682025756A
:1056E0000A00000042616420626F6172645F696455
:1056F0002025752073686F756C64206265202575A0
:105700000A0000004261642066772064657363725A
:105710006970746F72206C656E6774682025750AF5
:1057200000000000426164206170702043524320F9
:105730003078253038783A3078253038782030780D
:10574000253038783A3078253038780A0000000063
:10575000476F6F64206669726D776172650A000039
:1057600040A2E4F1646891060000000043414E4607
:105770004449666163653A204D65737361676520CE
:1057800052414D204F766572666C6F7721000000A4
:105790004261642043414E496661636520696E64DD
:1057A00065782E000001000000A0004000A4004029
:1057B00000000000000000000D220008FD19000894
:1057C000D9290008F11900086D1A0008C11E000847
:1057D000351C0008311A0008351A0008F5190008B0
:1057E0000D1A0008F9190008751E0008191A00089A
:1057F000012D0008251A0008951E00080000000071
:1058000000000000A52C0008F5300008B12C0008AD
:10581000F1190008192D0008C92C0008B52C000842
:10582000B92C0008BD2C0008F5190008C12C00088F
:10583000F9190008C52C0008F5300008012D0008F2
:10584000F5300008F53000086D61696E0000000059
:1058500069646C650000000050580008A85D0020D5
:10586000205F002001000000C94400080000000083
:1058700000000020000002000200000000010030D3
:1058800000000000000000000000002400000800EC
:10589000040000000004000000FC00000200000002
:1058A000000004300080000000000000000000380C
:1058B00000000100010000000000002800000000BE
:1058C000AAAAAAAA00000024FFFF0000000000000E
:1058D000000000000000550A00000000AAAA9AAAD1
:1058E00000000000FFF2000000000000000099002E
:1058F0000000000000000000AAAAAAAA0000000000
:10590000FFFF000000000000000000005A0000003F
:10591000000000009AAAAAAA00000000F3FF0000FD
:1059200099000000000000000000000000000000DE
:10593000AAAAAAAA00000000FFFF000000000000C1
:10594000000000000000000000000000AAAAAAAAAF
:1059500000000000FFFF0000000000000000000049
:105960000000000000000000AAAAAAAA000000008F
:10597000FFFF000000000000000000000000000029
:1059800000000000AAAAAAAA00000000FFFF000071
:105990000000000000000000000000000000000007
:1059A000AAAAAAAA00000000FFFF00000000000051
:1059B000000000000000000000000000AAAAAAAA3F
:1059C00000000000FFFF00000000000000000000D9
:1059D0000000000000000000AAAAAAAA000000001F
:1059E000FFFF00000000000000000000F4A8FF7F9F
:1059F000010000000000000013040000000000008F
:105A0000000018000000000001000000FE2A010054
:105A1000D20400002022002000000000000000004E
:105A20000000000000000000000000000000000076
:105A30000000000000000000000000000000000066
:105A40000000000000000000000000000000000056
:105A50000000000000000000000000000000000046
:105A60000000000000000000000000000000000036
:105A70000000000000000000FFFFFFFFFFFFFFFF2E
:105A8000FFFFFFFFFFFFFFFFFFFFFFFFFFFFFFFF26
:105A9000FFFFFFFFFFFFFFFFFFFFFFFFFFFFFFFF16
:105AA000FFFFFFFFFFFFFFFFFFFFFFFFFFFFFFFF06
:105AB000FFFFFFFFFFFFFFFFFFFFFFFFFFFFFFFFF6
:020000040803EF
:020000040804EE
:10000000000700306109040851320508F5020408B0
:10001000D5310508C5310508CD3105086309040847
:10002000630904086309040863090408BDBD0508E1
:1000300063090408630904086309040863090408E0
:1000400063090408630904086309040863090408D0
:100050006309040863090408E1FB05080DFC0508B1
:1000600039FC050865FC050891FC050855C2050822
:100070007DC20508A9C20508D5C2050801C3050847
:1000800029C3050855C305086309040831FE04089F
:1000900025FF0408A9FE04089DFF0408BDFC05080F
:1000A0006309040863090408630904086309040870
:1000B0006309040863090408F9FD050863090408D5
:1000C00063090408593F04086309040899C905082D
:1000D00063090408BDFD0508D1FD0508630904088E
:1000E00035FD050863090408630904086309040869
:1000F00063090408630904086309040881C3050847
:1001000063090408630904080DFE0508ADC9050864
:1001100063090408630904086309040863090408FF
:10012000ADC30508D5C3050801C405082DC40508DD
:1001300059C405086309040863090408630904082D
:1001400063090408630904086309040863090408CF
:1001500081C40508ADC40508D9C40508E5FD050836
:1001600063090408630904086309040863090408AF
:10017000630904086309040863090408630904089F
:10018000630904086309040863090408630904088F
:10019000630904086309040863090408630904087F
:1001A000630904086309040863090408630904086F
:1001B000630904086309040863090408630904085F
:1001C000630904086309040863090408630904084F
:1001D000630904086309040863090408630904083F
:1001E000630904086309040863090408630904082F
:1001F000630904086309040863090408630904081F
:10020000630904086309040863090408630904080E
:1002100063090408630904086309040863090408FE
:1002200063090408630904086309040863090408EE
:1002300063090408630904086309040863090408DE
:1002400063090408630904086309040863090408CE
:1002500063090408630904086309040863090408BE
:1002600063090408630904086309040863090408AE
:10027000630904086309040863090408630904089E
:10028000630904086309040863090408630904088E
:10029000630904086309040863090408630904087E
:1002A00081220408753B04081574040845C4040839
:1002B00019000508050A0508712D0508013405080F
:1002C0009D620508CD8D0508B19405080000000069
:1002D00040A2E4F164689106349B4A0C4BFBDF2496
:1002E00010E50200C17D3DB400001304FFFFFFFFD5
:1002F000FFFFFFFFEFF30383EFF30982EFF30881C2
:10030000DFF814D02DE9FE4F684601F07DF8BDE816
:10031000FE4F8D4670470000C4290030F1EE101AE0
:10032000A0EC200A01607047A0EC108A704700BF63
:1003300080F0004002E000BF81F0004142001FBF9A
:100340005FEA410392EA030F7FEA226C7FEA236CA3
:100350006AD04FEA1262D2EB1363C1BFD218414098
:1003600048404140B8BF5B42192B88BF704710F02E
:10037000004F40F4000020F07F4018BF404211F0D1
:10038000004F41F4000121F07F4118BF494292EA39
:10039000030F3FD0A2F1010241FA03FC10EB0C0065
:1003A000C3F1200301FA03F100F0004302D54942F2
:1003B00060EB4000B0F5000F13D3B0F1807F06D39F
:1003C00040084FEA310102F10102FE2A51D2B1F197
:1003D000004F40EBC25008BF20F0010040EA03008C
:1003E0007047490040EB0000013A28BFB0F5000F0C
:1003F000EDD2B0FA80FCACF1080CB2EB0C0200FAC2
:100400000CF0AABF00EBC25052421843BCBFD04010
:100410001843704792F0000F81F4000106BF80F48A
:1004200000000132013BB5E74FEA41037FEA226C4D
:1004300018BF7FEA236C21D092EA030F04D092F018
:10044000000F08BF0846704790EA010F1CBF00204C
:10045000704712F07F4F04D1400028BF40F00040A9
:10046000704712F100723CBF00F50000704700F0C9
:10047000004343F0FE4040F4000070477FEA2262F0
:1004800016BF08467FEA23630146420206BF5FEAC1
:10049000412390EA010F40F4800070474FF00003C1
:1004A00004E000BF10F0004348BF40425FEA000C88
:1004B00008BF704743F0964301464FF000001CE030
:1004C00050EA010208BF70474FF000030AE000BF86
:1004D00050EA010208BF704711F0004302D54042C4
:1004E00061EB41015FEA010C02BF84460146002036
:1004F00043F0B64308BFA3F18053A3F50003BCFA51
:100500008CF2083AA3EBC25310DB01FA02FC6344FD
:1005100000FA02FCC2F12002BCF1004F20FA02F204
:1005200043EB020008BF20F00100704702F12002F7
:1005300001FA02FCC2F1200250EA4C0021FA02F258
:1005400043EB020008BF20EADC7070477BB972B948
:100550000029BEBF00204FF0004106E008BF002880
:100560001CBF6FF000414FF0FF3000F0F7B9ADF164
:10057000080C6DE904CE002909DB002B1ADB00F022
:1005800085F8DDF804E0DDE9022304B0704740425D
:1005900061EB4101002B1BDB00F078F8DDF804E093
:1005A000DDE9022304B0404261EB4101524263EBBA
:1005B00043037047524263EB430300F067F8DDF8F2
:1005C00004E0DDE9022304B0404261EB41017047E1
:1005D000524263EB430300F059F8DDF804E0DDE933
:1005E000022304B0524263EB4303704753B94AB944
:1005F000002908BF00281CBF4FF0FF314FF0FF302B
:1006000000F0ACB9ADF1080C6DE904CE00F03EF895
:10061000DDF804E0DDE9022304B0704708B50246C6
:100620000B4643EC172BB5EEC07BF1EE10FA03D46A
:10063000BDE8084000F00AB8B1EE477B51EC170B5B
:1006400000F004F8404261EB410108BD9FED0B6BE7
:1006500041EC170B9FED0B5B27EE066BBCEEC66BF8
:10066000B8EE464BA4EE457BFCEEC77B16EE101AA7
:1006700017EE900A704700BFAFF300800000000043
:100680000000F03D000000000000F0412DE9F047BF
:10069000089D04468E46002B4DD18A42944669D966
:1006A000B2FA82F252B101FA02F3C2F1200120FA49
:1006B00001F10CFA02FC41EA030E94404FEA1C4897
:1006C000210CBEFBF8F61FFA8CF708FB16E341EA93
:1006D000034306FB07F199420AD91CEB030306F119
:1006E000FF3080F01F81994240F21C81023E63443A
:1006F0005B1AA4B2B3FBF8F008FB103344EA0344DE
:1007000000FB07F7A7420AD91CEB040400F1FF33F2
:1007100080F00A81A74240F207816444023840EA2F
:100720000640E41B00261DB1D4400023C5E9004368
:100730003146BDE8F0878B4209D9002D00F0EF80EB
:100740000026C5E9000130463146BDE8F087B3FA1E
:1007500083F6002E4AD18B4202D3824200F2F98006
:10076000841A61EB030301209E46002DE0D0C5E909
:10077000004EDDE702B9FFDEB2FA82F2002A40F055
:100780009280A1EB0C014FEA1C471FFA8CFE012658
:10079000200CB1FBF7F307FB131140EA01410EFBFC
:1007A00003F0884208D91CEB010103F1FF3802D2A3
:1007B000884200F2CB804346091AA4B2B1FBF7F09D
:1007C00007FB101144EA01440EFB00FEA64508D9C0
:1007D0001CEB040400F1FF3102D2A64500F2BB80FD
:1007E0000846A4EB0E0440EA03409CE7C6F120074C
:1007F000B34022FA07FC4CEA030C20FA07F401FA92
:1008000006F31C43F9404FEA1C4900FA06F3B1FB1A
:10081000F9F8200C1FFA8CFE09FB181140EA01417F
:1008200008FB0EF0884202FA06F20BD91CEB01011C
:1008300008F1FF3A80F08880884240F28580A8F174
:1008400002086144091AA4B2B1FBF9F009FB1011C6
:1008500044EA014100FB0EFE8E4508D91CEB010164
:1008600000F1FF346CD28E456AD90238614440EA07
:100870000840A0FB0294A1EB0E01A142C846A64687
:1008800056D353D05DB1B3EB080261EB0E0101FA10
:1008900007F722FA06F3F1401F43C5E9007100266D
:1008A0003146BDE8F087C2F12003D8400CFA02FCC3
:1008B00021FA03F3914001434FEA1C471FFA8CFED3
:1008C000B3FBF7F007FB10360B0C43EA064300FBC3
:1008D0000EF69E4204FA02F408D91CEB030300F161
:1008E000FF382FD29E422DD9023863449B1B89B218
:1008F000B3FBF7F607FB163341EA034106FB0EF3A1
:100900008B4208D91CEB010106F1FF3816D28B424D
:1009100014D9023E6144C91A46EA004638E72E4619
:10092000284605E70646E3E61846F8E64B45A9D211
:10093000B9EB020864EB0C0E0138A3E74646EAE780
:10094000204694E74046D1E7D0467BE7023B61442E
:1009500032E7304609E76444023842E7704700BF97
:1009600002E000F000F8FEE772B63A4880F308882B
:10097000394880F3098839484EF60851CEF2000113
:10098000086040F20000CCF200004EF63471CEF266
:1009900000010860BFF34F8FBFF36F8F40F200007C
:1009A000C0F2F0004EF68851CEF200010860BFF3AD
:1009B0004F8FBFF36F8F4FF00000E1EE100A4EF63D
:1009C0003C71CEF200010860062080F31488BFF36A
:1009D0006F8F1EF00FFE1EF0B1FD1EF00FFF4FF0E7
:1009E00055301F491B4A91423CBF41F8040BFAE7BE
:1009F0001C49194A91423CBF41F8040BFAE71A49D5
:100A00001A4A1B4B9A423EBF51F8040B42F8040BA2
:100A1000F8E700201749184A91423CBF41F8040BFF
:100A2000FAE71EF0CDFD1EF0FFFE144C144DAC4253
:100A300003DA54F8041B8847F9E701F011FC114C64
:100A4000114DAC4203DA54F8041B8847F9E71EF055
:100A5000B5BD00000007003000230030000004088E
:100A6000000100300007003040E00608002300309D
:100A7000D0270030D0270030C0020130A002040887
:100A8000CC020408CC020408CC0204082DE9F04F83
:100A90002DED108AC1F80CD0D0F80CD0BDEC108A26
:100AA000BDE8F08F002383F311882846A04700207B
:100AB0001DF07EFDFEE71DF007FC00DFFEE70000F5
:100AC00070B54FF0FF0C4CF4E06C1CEA11541DBFE4
:100AD0001CEA135594EA0C0F95EA0C0F00F0DEF8AF
:100AE0002C4481EA030621EA4C5123EA4C5350EA94
:100AF000013518BF52EA033541F4801143F48013E5
:100B000038D0A0FB02CE4FF00005E1FB02E506F075
:100B10000042E0FB03E54FF00006E1FB03569CF0CA
:100B2000000F18BF4EF0010EA4F1FF04B6F5007FD0
:100B300064F5407404D25FEA4E0E6D4146EB060642
:100B400042EAC62141EA55514FEAC52040EA5E50CB
:100B50004FEACE2EB4F1FD0C88BFBCF5E06F1ED875
:100B6000BEF1004F08BF5FEA500E50F1000041EBAC
:100B7000045170BD06F0004646EA010140EA020059
:100B800081EA0301B4EB5C04C2BFD4EB0C0541EA7B
:100B9000045170BD41F480114FF0000E013C00F390
:100BA000AB8014F1360FDEBF002001F0004170BDB4
:100BB000C4F10004203C35DA0C341BDC04F11404CD
:100BC000C4F1200500FA05F320FA04F001FA05F259
:100BD00040EA020001F0004221F0004110EBD37026
:100BE00021FA04F642EB06015EEA430E08BF20EA52
:100BF000D37070BDC4F10C04C4F1200500FA04F3F5
:100C000020FA05F001FA04F240EA020001F0004186
:100C100010EBD37041F100015EEA430E08BF20EAF9
:100C2000D37070BDC4F1200500FA05F24EEA020E41
:100C300020FA04F301FA05F243EA020321FA04F070
:100C400001F0004121FA04F220EA020000EBD37027
:100C50005EEA430E08BF20EAD37070BD94F0000F27
:100C60000FD101F00046400041EB010111F4801F5B
:100C700008BF013CF7D041EA060195F0000F18BF0C
:100C8000704703F00046520043EB030313F4801F48
:100C900008BF013DF7D043EA0603704794EA0C0F02
:100CA0000CEA135518BF95EA0C0F0CD050EA410618
:100CB00018BF52EA4306D1D181EA030101F0004195
:100CC0004FF0000070BD50EA410606BF10461946BD
:100CD00052EA430619D094EA0C0F02D150EA0136C9
:100CE00013D195EA0C0F05D152EA03361CBF10460A
:100CF00019460AD181EA030101F0004141F0FE41A9
:100D000041F470014FF0000070BD41F0FE4141F42C
:100D1000780170BD81F0004102E000BF83F0004324
:100D200030B54FEA41044FEA430594EA050F08BF86
:100D300090EA020F1FBF54EA000C55EA020C7FEA4A
:100D4000645C7FEA655C00F0E2804FEA5454D4EBC7
:100D50005555B8BF6D420CDD2C4480EA020281EA91
:100D6000030382EA000083EA010180EA020281EAC9
:100D70000303362D88BF30BD11F0004F4FEA01311B
:100D80004FF4801C4CEA113102D0404261EB41012A
:100D900013F0004F4FEA03334CEA133302D05242B0
:100DA00063EB430394EA050F00F0A780A4F101046C
:100DB000D5F1200E0DDB02FA0EFC22FA05F28018A6
:100DC00041F1000103FA0EF2801843FA05F359418C
:100DD0000EE0A5F120050EF1200E012A03FA0EFC0B
:100DE00028BF4CF0020C43FA05F3C01851EBE37135
:100DF00001F0004507D54FF0000EDCF1000C7EEB52
:100E000000006EEB0101B1F5801F1BD3B1F5001F8F
:100E10000CD349085FEA30004FEA3C0C04F10104AE
:100E20004FEA445212F5800F80F09A80BCF1004FD7
:100E300008BF5FEA500C50F1000041EB045141EA59
:100E4000050130BD5FEA4C0C404141EB0101013C22
:100E500028BFB1F5801FE9D291F0000F04BF014611
:100E60000020B1FA81F308BF2033A3F10B03B3F1E3
:100E700020020CDA0C3208DD02F1140CC2F10C0273
:100E800001FA0CF021FA02F10CE002F11402D8BFD1
:100E9000C2F1200C01FA02F120FA0CFCDCBF41EA9D
:100EA0000C019040E41AA2BF01EB0451294330BD6C
:100EB0006FEA04041F3C1CDA0C340EDC04F1140449
:100EC000C4F1200220FA04F001FA02F340EA030020
:100ED00021FA04F345EA030130BDC4F10C04C4F166
:100EE000200220FA02F001FA04F340EA0300294646
:100EF00030BD21FA04F0294630BD94F0000F83F490
:100F0000801306BF81F480110134013D4EE77FEA72
:100F1000645C18BF7FEA655C29D094EA050F08BFBE
:100F200090EA020F05D054EA000C04BF194610469F
:100F300030BD91EA030F1EBF0021002030BD5FEAE3
:100F4000545C05D14000494128BF41F0004130BD0B
:100F500014F580043CBF01F5801130BD01F000455F
:100F600045F0FE4141F470014FF0000030BD7FEAD2
:100F7000645C1ABF194610467FEA655C1CBF0B46CD
:100F8000024650EA013406BF52EA033591EA030FE4
:100F900041F4002130BD00BF90F0000F04BF0021DC
:100FA000704730B54FF4806404F132044FF000050F
:100FB0004FF0000150E700BF90F0000F04BF002188
:100FC000704730B54FF4806404F1320410F00045EE
:100FD00048BF40424FF000013EE700BF42004FEAE9
:100FE000E2014FEA31014FEA02701FBF12F07F4366
:100FF00093F07F4F81F06051704732F07F4208BF1D
:10100000704793F07F4F04BF41F40021704730B523
:101010004FF4607401F0004521F000411CE700BF6F
:1010200050EA010208BF704730B54FF000050AE0F2
:1010300050EA010208BF704730B511F0004502D5F3
:10104000404261EB41014FF4806404F132045FEAF5
:10105000915C3FF4D8AE4FF003025FEADC0C18BF9E
:1010600003325FEADC0C18BF033202EBDC02C2F190
:10107000200300FA03FC20FA02F001FA03FE40EA22
:101080000E0021FA02F11444BDE600BF4FEA41020E
:1010900012F5001215D211D56FF47873B3EB6252CA
:1010A00012D94FEAC12343F0004343EA505311F0F1
:1010B000004F23FA02F018BF404270474FF0000083
:1010C000704750EA013005D111F0004008BF6FF0C1
:1010D000004070474FF00000704700BF4FEA4102E8
:1010E000B2F1E04324BFB3F5001CDCF1FE5C0DD986
:1010F00001F0004C4FEAC0024CEA5070B2F1004FD0
:1011000040EB830008BF20F00100704711F0804FD2
:1011100021D113F13872BCBF01F00040704741F497
:1011200080114FEA5252C2F11802C2F1200C10FA9B
:101130000CF320FA02F018BF40F001004FEAC1237F
:101140004FEAD32303FA0CFC40EA0C0023FA02F323
:101150004FEA4303CCE77FEA625307D150EA0133F9
:101160001EBF4FF0FE4040F44000704701F00040C9
:1011700040F0FE4040F40000704700BF10F8012B23
:1011800011F8013B012A28BF9A42F7D0D01A7047C4
:10119000034613F8012B002AFBD1181A01387047B7
:1011A000C36A13F0040F01D04068704700687047AD
:1011B000704700BF10B5044608462160FFF7F0FFF6
:1011C000E060FFF7F5FF60600023A360204610BDDC
:1011D0000368DB6A13F0100F0CBF0120002070477A
:1011E00038B50446C5682035C560FFF7F1FF08B182
:1011F0004835E5606368DB69DB0903F00403E268F6
:101200001343E36038BD00BF4FF0E023D3F8880DEF
:1012100000F4A000B0F5A00F14BF0020012070471B
:1012200010B50446FFF7F0FF18B1A36843F00103BF
:10123000A36010BD00F47F40B0F53E4F14BF002006
:101240000120704710B5044643689869FFF7B0FF66
:101250000088FFF7EFFF206110BD00BF014B024A7D
:101260001A607047D0270030ED55CEAC4FF0E02328
:10127000D3F8000D00F47020B0F5402F14BF00200B
:101280000120704703691BB142689369023393617F
:10129000704700BF08B504220121024800F034FC69
:1012A00008BD00BF803D060808B5042201210830B2
:1012B00000F02AFC08BD00BF08B5102201214068DB
:1012C00000F022FC08BD00BF08B500682022012103
:1012D0000C3000F019FC08BD08B54068042201215B
:1012E000103000F011FC08BD08B5042201210C30BB
:1012F00000F00AFC08BD00BF08B540680C220121BF
:10130000143000F001FC08BD08B50C220121006872
:1013100000F0FAFB08BD00BF38B5044610E0082213
:101320000121204600F0F0FB25682846FFF740FF2A
:10133000217A6268521BB2FBF1F200F0E5FB0C343B
:101340001CB12368B3F1FF3FE9D138BD00B587B0C8
:10135000094B00931433019304238DF808304FF0A8
:10136000FF330393049301238DF814306846FFF78D
:10137000D3FF07B05DF804FB28ED00E0094B1A68C5
:10138000094B9A4200D1704700B583B0074B0193D7
:10139000042201210DEB020000F0B6FB03B05DF862
:1013A00004FB00BFD0270030ED55CEACACCE55EDE0
:1013B00070B5A2B00446FFF70BFF08B311A8FEF703
:1013C000B3FF666806F1200C01AD6036AE46DCF86E
:1013D0000000DCF80410DCF80820DCF80C30AEE883
:1013E0000F000CF1100C7546B445EFD163681B6E0D
:1013F00021938422012101A800F086FB22B070BD58
:1014000001A8FEF78BFFF4E700B587B0014601A8FD
:10141000FFF7D0FE01A8FFF7E3FE01A8FFF700FFEA
:1014200001A8FFF70FFF08E001A8FFF7C1FF24E0C4
:10143000FFF7A4FF00F0D6FB50BBFFF70FFF04A897
:1014400000F0A2FBFFF726FF01A8FFF72DFF01A880
:10145000FFF732FF01A8FFF737FF01A8FFF73CFFB6
:1014600001A8FFF741FF01A8FFF746FF01A8FFF71A
:101470004BFF039B13F0010FD6D100F083F9FFF768
:101480004BFFFFF7F3FE0028D2D1FFF75FFFCFE756
:1014900001A8FFF7F7FE07B05DF804FB08B52520AB
:1014A0001CF03AF8144BD3F8982042F01002C3F81D
:1014B0009820D3F8982022F01002C3F89820D3F88F
:1014C0009820D3F8F02042F01002C3F8F020D3F8AF
:1014D000182142F01002C3F81821D3F81831074B35
:1014E0006D22DA604FF0FF321A620D221A60044B4F
:1014F00001221A7008BD00BF0044025800100140CC
:10150000FC2900300148024BC01A7047000018083F
:1015100020E506080048704720E5060838B50E4B60
:101520001B78202B00D038BDFFF7F4FF0B4D0C4C7F
:1015300023682022294618441DF066FB23682033C7
:1015400023600021044B1970202228461FF074FAF2
:101550001DF0B8FFE7E700BFC4290030C8290030FC
:10156000EC2900302DE9F84307460D469046002649
:101570001AE0254B4FF0FF32DA61244B20221A701B
:10158000BDE8F883214C23785A1C22703A78DFF8A2
:10159000789009F80320FFF7C1FF23785A1C2270C6
:1015A000002209F8032001364645E9D2174B1C7882
:1015B000174B1B681C440434FFF7A4FF8442D8D2A5
:1015C000FFF7ACFF022DDDD0042D1AD0012DEBD199
:1015D0000E4A1378591C1170B95D0B4AD15401366B
:1015E000E2E73B78E200D34008490A78501C0870D3
:1015F00005498B54FFF792FF0134032CF1D90136D2
:10160000D2E70024F9E700BFC8290030C429003020
:10161000EC29003070B5294B1E68294B1D783544E4
:101620000435FFF76FFF044685422FD2244B1B7809
:1016300003B306F12002944206D81F2B04D8214B95
:10164000DE611F4B20221A70FFF764FF1D4D202220
:10165000294630441DF0D8FA1849194A1378086809
:1016600003440B6000211170202228461FF0E4F98A
:101670001DF028FF114B1B689C420FD800201DF065
:10168000C7FA114B5B68B3B1012070BD0D4B4FF031
:10169000FF32DA610A4B20221A70C7E7094DEB616D
:1016A000FFF738FF20442022294620381DF0ACFAED
:1016B0001DF008FFE2E70020E7E700BFEC2900305B
:1016C000C4290030C8290030F429003010B50024A6
:1016D00000E00434FFF716FFA04209D9FFF71AFF14
:1016E00024F003031B58B3F1FF3FF2D0002000E0C9
:1016F000012010BD10B504681CB91D4B00221A70E2
:1017000010BD20461DF0F6FB0028F6D020461DF047
:101710001FFC00F21450A04218D8A4F21453154A2A
:10172000136020461DF03EFC04F5E053834213D8BD
:10173000114A13600023114A1360114A1370FFF716
:10174000C5FF78B90A4B00221A70D9E720461DF070
:10175000FFFB084B1860E4E720461DF023FC064B16
:101760001860E7E71DF0AEFE01201DF051FAC7E753
:1017700000230030F0290030E8290030EC29003047
:10178000C42900302DE9F0416F4B1B786F4A126875
:10179000134443F698271F441CF078FC05460224A6
:1017A00032E06B4EF61A3BE06A4B04EB440203EB6B
:1017B00082014FF0010C81F808C043F8225004EB7D
:1017C0000C02D2B205F1380004EB440103EB8101B5
:1017D000486002EB420103EB810080F808C0E86931
:1017E00043F82100E9690234E4B2314402EB4202D9
:1017F00003EB820359603744FFF784FEB8425CD99B
:1018000028461CF053FC05462B1E18BF01233A2C1A
:1018100088BF002313B3EE694F4B9E42C1D0AE1B6D
:10182000A8690028C0D01DF065FB0028BCD0224666
:10183000484B04EB440103EB81004FF0010C80F8AE
:1018400008C0A86943F82100A9696444E4B20D31D5
:1018500002EB420203EB82035960A5E7DFF8148133
:101860003E4EA8EB0605FFF74DFEC31B25D49D4257
:1018700040DD384A04EB440502EB85074FF0010CCC
:1018800087F808C042F825606444E4B233447B60C2
:101890000746334A334BD11AC01B0ED481423ADD7E
:1018A0002C4A04EB440502EB85060127377242F807
:1018B00025303C44E4B2184470603B2C38D8254BAA
:1018C00004EB440103EB8102012010724FF0FF3260
:1018D00043F8212003EB81046260234B1B7833B172
:1018E000224B1A681B4B1A60214A12685A60194829
:1018F000BDE8F081174B04EB440103EB810C4FF082
:10190000010E8CF808E043F821607444E4B2CCF88E
:1019100004802F44BDE70F4904EB440501EB850625
:101920000127377241F825303C44E4B27260C4E7C5
:10193000084B012283F8CC224FF0FF32C3F8C422B7
:10194000C3F8C822C9E700BFC4290030EC29003021
:10195000002300300423003000070030D02700307F
:1019600000000430C002013000230030F0290030B4
:10197000E8290030C002013008B50D4B1B78A3B137
:1019800000210A460B4BDB6913F0200FFAD0094BFC
:101990005B6ADBB20849505C00219842F1D1013208
:1019A000D1B20E29EDD1002008BDFFF777FDE7E7A2
:1019B000FC29003000100140843D060808B5FFF7FF
:1019C000DBFF08BD10B50446084B1B781BB1E4B221
:1019D000074B9C6204E0FFF761FDF8E71DF072FD24
:1019E000034BDB6913F0400FF8D010BDFC29003029
:1019F0000010014008B5024B185CFFF7E3FF08BD7B
:101A0000083E060810B504460009FFF7F3FF04F08E
:101A10000F00FFF7EFFF10BD10B5044602E00134E0
:101A2000FFF7D0FF20780028F9D110BD70B504462B
:101A30000E46002504E014F8010BFFF7E3FF013523
:101A4000B54208D2002DF6D015F00F0FF3D10248A1
:101A5000FFF7E2FFEFE770BD6846060870B582B099
:101A600004460E46002505E002210DF10600FFF7B1
:101A7000DDFF0135B5420CD234F8023BADF806303B
:101A8000002DF1D015F0070FEED10348FFF7C4FF8A
:101A9000EAE702B070BD00BF6846060870B582B0C4
:101AA00004460E46002505E004210DEB0100FFF77A
:101AB000BDFF0135B5420BD254F8043B0193002D14
:101AC000F2D015F0030FEFD10248FFF7A5FFEBE7C7
:101AD00002B070BD6846060808B50B461146022BD9
:101AE0000AD0042B0BD0012B03D00648FFF794FF3C
:101AF00008BDFFF79BFFF8E7FFF7B0FFF5E7FFF73B
:101B0000CDFFF2E76846060870B504460D46164656
:101B1000074B1B781BB9074B1B781BB970BDFFF730
:101B2000DBFFF8E7324629462046FFF71BFDF5E7C5
:101B3000C52900300023003010B504460C4BD0E915
:101B4000000183E803000B48FFF766FF63685BB1A1
:101B50000948FFF761FF0948FFF75EFFFFF72EFF17
:101B60000748FFF759FF10BD0648FFF755FFF2E79A
:101B7000F4290030943D06089C3D0608B03D060857
:101B800068460608A83D060810B504460268EFF34B
:101B900005815369C9B2D92011F020FB074B1B788E
:101BA0001BB9074B1B7823B910BD2046FFF7C4FFB4
:101BB000F7E72046FFF79EFDF6E700BFC529003096
:101BC0000023003008B50548FFF726FF044B5B688B
:101BD0000BB1012008BD0020FCE700BFF83D06085E
:101BE000F429003008B5094B1B784BB9084B1B781A
:101BF0004BB90020064B1870044B01221A7008BD27
:101C0000FFF7E0FFFBE7FFF705FDF8E7C529003028
:101C10000023003008B503681B680021984708BD01
:101C200008B503681B68984708BD00BF084AC0F89C
:101C300004240849C0F81014074AC0F81024C0F85A
:101C40004813C0F84823C0F88010C0F880207047BF
:101C5000D844060878830608D43E060810B5044622
:101C60000123002B01DB013BFBE70123002B01DB00
:101C7000013BFBE70123002B01DB013BFBE704F108
:101C8000280009F06BFC04F1500005F0C5FCFF23AF
:101C900084F8C03104F5E27009F076FF04F5447071
:101CA0000AF0FCFA04F559700AF0DEFB0122002369
:101CB000C4E9EE23002384F8C83304F574701C4A89
:101CC0001C49116001E001339BB203EB4302194947
:101CD00011F83220002AF6D1174A1380174B1B68DF
:101CE00003BB164B1860164BC4F8043404F582602D
:101CF0000EF018FA134BC4F82834134BC4F82834E8
:101D000004F22C43C4F82C3464224FF4FA7104F525
:101D1000876009F0D7FE0D4B1B6833B90B4B1C6075
:101D2000204610BD0A4811F097FA0A4811F094FABB
:101D3000003F003028400608FC3E0030C03E003026
:101D4000D8440608F43E060864830608042A0030D6
:101D50001C3E0608383E0608012800D070474FF6A2
:101D6000FF739942FAD110B5094C2046FFF776FF70
:101D7000084A094920461EF095F80EF02FFE074B41
:101D80001860074A0749084802F01AFA10BD00BF58
:101D9000302A00303CCD00302D1C04082C2A0030A5
:101DA00051220408551F0408202A003008B50829CC
:101DB00002D00A2908D008BD074B1B68586C03687D
:101DC0001B6909219847F6E7034B1B68586C0368A9
:101DD0001B6907219847EEE72C2A003008B5FFF76A
:101DE000E5FF08BD2DE9F04188B004461DF06AFB0F
:101DF000534D0021286802F0F1F90368DE6A2023C0
:101E00001A464FF4E131B0470321286802F0E6F9A1
:101E10000368DE6A4FF4807380224FF4E131B047EB
:101E2000204600F035FA1DF04DFB204601F028FA5F
:101E300004F12806304609F0B1FC1DF043FB0021F7
:101E40000291019100910B460A463E480EF0ECF9D2
:101E50002B68586D03685B689847002865D194F932
:101E600050301BB194F92430002B62D0344D2B68D4
:101E7000586C03685B6A0022082198472B68586CED
:101E800003685B6A0122072198472B68586C036836
:101E90005B6A00220A2198472B68586C03685B6ACA
:101EA0000122092198472B68586C0368D3F82C80CD
:101EB0000494254F05970326009604AB0CCB08210C
:101EC000C0472B68586C0368DD6A06940797009634
:101ED00008AB13E90C000A21A84704F2044504F5F5
:101EE0008561284602F050F90121284602F024F9C4
:101EF000204601F047FE04F5E27009F04FFF104D57
:101F00002B68D86C03681B6898472B68D86C0368EB
:101F10001B6D984704F559700AF0F2FB11F0D8F9DF
:101F20000A4B186008B0BDE8F08109480EF07CF952
:101F300095E7314604F1500005F0DCFBCDE700BF2A
:101F40002C2A0030583E0608DD1D0408002A003007
:101F5000803E060808B50248FFF744FF08BD00BFF1
:101F6000302A003090F8C83303B1704770B58AB09A
:101F700011F0AEF90646294B1B68C31A632B4BD9E7
:101F800004AC274D0FCD0FC495E8030084E803008F
:101F9000224B1E60002439E0224B1B78234403F0BF
:101FA000070303EB43030AAA134413F8182C07EEA4
:101FB000902AF8EEE77A9FED1C6A67EE867A13F8AE
:101FC000172C07EE102AB8EEC77A27EE067A13F818
:101FD000163C06EE903AF8EEE66A66EE866AFCEE8D
:101FE000E66ACDED016ABCEEC77A8DED027AFCEEB1
:101FF000E77ACDED037A00239DF804209DF80810C0
:102000009DF80C000AF0ACFB0134E4B2032CC3D9F8
:10201000044A1378013313700AB070BD082A0030E7
:102020007C3C06080C2A00309A99993E70B51248FB
:10203000124C241A1DF058F901462246104801F0AE
:102040005FFC1CF023F804460DE0251AA6691DF07C
:102050004BF902462B4631460A4801F051FC204616
:102060001CF024F8044634B1E069074B9842ECD1E7
:10207000064DED1AEAE770BD0001003000070030A0
:10208000A03E0608AC3E06080007003000230030E2
:1020900008B590F8603303B908BD002380F86033B9
:1020A0000AF02AF90AF0A0F909F066FF0AF0A6F989
:1020B000F2E700BF10B504F06BFA074C2368186D07
:1020C0000368DB690522002198472368186D0368BF
:1020D0005B682821984710BD2C2A003070B5044653
:1020E00011F0F6F80546524B1B68C31AB3F57A7F18
:1020F0007AD809F0DBFE4F4B1B68EB1A41F28832AD
:10210000934202D90168002973D194F91030012B50
:1021100076D0494B1B68EB1A132B7ED8204601F072
:10212000B9FC94F8003463B3444B1B784BB3444D73
:102130002B68186D03681B696421984794F9243053
:10214000013B07EE903AF8EEE77AF0EEE77A9FED82
:102150003D7AF4EEC77AF1EE10FA4FF0010384F8FD
:1021600024304CBF1946002104F1240004F0AEF9DC
:102170002046FFF79FFF2B68186D03689B6B0021BB
:1021800098472E4B1B785BBB94F9243043B32C4EFD
:102190003368186D03681B696421984794F92430EB
:1021A00007EE903AF8EEE77AF0EEE77A9FED257ABF
:1021B000F4EEC77AF1EE10FA4FF0000584F82450DF
:1021C0004CBF0121294604F1240004F07FF9204688
:1021D000FFF770FF3368186D03689B6B29469847BB
:1021E00094F9243003B370BD114B186009F0A6FFB9
:1021F0007FE7104B1D600289134801F081FB84E7E3
:10220000124B1B68EB1A41F28832934281D90F4B73
:102210001D602046FFF70AFF7BE7074B1D6004F5B2
:1022200059700AF081FA79E72046FFF79BFEDAE75A
:10223000102A0030182A00301C2A0030D425003023
:102240002C2A003000000034BC3E0608142A00305E
:1022500008B50248FFF742FF08BD00BF302A003032
:1022600010B584460A46044B186803681C68034B83
:102270006146A047002010BD2C2A0030202A0030E3
:1022800008B54FF6FF710120FFF766FD08BD00BFDE
:1022900010B5044604F00CFF03F0CCFD30B320462B
:1022A00004F054FE18B1B4F90030022B1BD005F035
:1022B000B9F803F08BFEB4F90030023B07EE903A18
:1022C000F8EEE77AF0EEE77A9FED0D7AF4EEC77A52
:1022D000F1EE10FA4FF0020323804CBF01210021E0
:1022E000204604F0F3F804F0AFFD10BD054B1B6869
:1022F000186C03681B6804499847044810F0ACFF49
:10230000000000342C2A0030003F0608183F060861
:10231000BFF34F8F0549CA6802F4E062044B1343D0
:10232000CB60BFF34F8F00BFFDE700BF00ED00E0C3
:102330000400FA05012800D070474FF6FF73994258
:10234000FAD1024B012283F8D22FF5E7982E003004
:1023500070B50E4614461D4618F0B4F968B9022D42
:1023600008BF012C0CBF0120002040F0828042A356
:10237000D3E90023C6E900237BE0282C1BD823B235
:10238000002B73D0013C272C72D8DFE804F03771A2
:1023900071614571717171534C71717171717171AC
:1023A000717171717171717171717171717171711D
:1023B00071717171713E40F24C439C4241D00AD917
:1023C00044F627639C4217D12DA3D3E90023C6E925
:1023D000002301204DE040F226439C423FD040F2D2
:1023E00039439C4206D128A3D3E90023C6E9002340
:1023F00001203EE000203CE000203AE024A3D3E9A5
:102400000023C6E90023012033E023A3D3E90023FE
:10241000C6E9002301202CE021A3D3E90023C6E96B
:102420000023012025E020A3D3E90023C6E90023EF
:1024300001201EE01EA3D3E90023C6E900230120EA
:1024400017E01DA3D3E90023C6E90023012010E013
:102450001BA3D3E90023C6E90023012009E01AA346
:10246000D3E90023C6E90023012002E0002000E0B8
:10247000002070BDAFF30080401DA12026812A0BF3
:10248000ECFD51169C2A1F63C41EDD8B3CD9312004
:102490009E6AC421818A46EE26417272DF25D7B733
:1024A000F017304A39059E56D5A4D139F922B6A77E
:1024B000CDD269EBC51A133B03806A5575F30087CB
:1024C000DBC293A716112720011517CB0E03561F49
:1024D00010B5044602F05EFDB0FBF4F304FB1300FC
:1024E00080B210BD00B583B0014610238DF80730CF
:1024F0000023036043608360C360054B1B68586D15
:1025000003685B6B0DF10702984703B05DF804FBAD
:102510002C2A003070B58AB006460D4610F0D8FE61
:1025200004464FF4C870FFF7D3FF044404F5167453
:10253000214BC3F8CC4FEB7EFBB105A9284619F01F
:1025400007FA01A8FFF7CEFF9DF81640224601A921
:102550000DF117001EF052FAC0B90F2C1ED8164B01
:1025600083F8D04FD3F8CC2FA2F51672C3F8CC2F36
:10257000214612480DF058FE06E011480DF054FEB9
:102580000D4B002283F8D02F0AB070BD0D480DF01E
:102590004BFE094B002283F8D02FF5E79DF814106D
:1025A000304618F087F89DF81420034B93F8D21F9B
:1025B00005480DF039FEE7E7982E0030584206082E
:1025C000084206083442060890420608F0B5ADF508
:1025D0004B7D06460D4600276B9740F27512394633
:1025E0006CA81EF029FA08AC4FF4C4723946204694
:1025F0001EF022FA10F06CFE03463E48A0FB0323B7
:102600009B093D4A136007CA84E8070001F0AEFC4D
:10261000037C237401F0AAFC437C63740323A3743A
:10262000364B5A6962619A68A261DB68E3610DF119
:102630004200FFF757FF042384F82030132384F867
:1026400021302F4B5B69BB423EDD2E4A1268506D34
:1026500001932D4B00932D4B50220DF2531101F09D
:10266000FFFE50210DF253101EF06EFD8DF8520149
:10267000234F97F918206BAC013A18BF012221466D
:1026800008A819F03FF880B297F91830012B14BF51
:102690000023012307930723069305900494002346
:1026A0000393AB7E029305F1190301930123009379
:1026B0000EA3D3E90023E97E304618F06DF8011E21
:1026C0000EDD0DF54B7DF0BD0E4B1B68586D0E4BAE
:1026D00000930F4B50220DF2531101F0C1FEC0E7E1
:1026E0000C480DF0A1FDECE7AFF300809E6AC42119
:1026F000818A46EED34D62108C2E0030D002040841
:10270000302A00302C2A0030B4420608AC420608B9
:10271000C4D50608CC4206082DE9F041ADF5866D1A
:1027200005460C461CF0CEFECEA9204619F0A6F9AF
:10273000002840F0C9804FF4D072002166A81EF036
:102740007BF99DF8D023102A75D8531EDBB20F2BCE
:1027500021D80DF2D1310DF2D9201EF05FF90022FF
:102760000DF297110DF2D92003F02AFE0646002E35
:1027700062D09DF8D033002B5ED09DF84023002A14
:102780005AD09DF89731013B032B00F29D80DFE882
:1027900003F0172634400023089308AA0DF297117E
:1027A000BDF8380304F074F906460028DFD0012391
:1027B000009311230DF2D92208A903F047FDD6E7B3
:1027C000012A40F081809DF9483396F90020934218
:1027D00032D033700121304603F078FE2CE0012A1C
:1027E00072D1BDF94833B6F90020934224D033802A
:1027F0000121304603F06AFE1EE0012A64D1D29B1B
:102800003268934218D033600121304603F05EFEF7
:1028100012E0022A58D1DDEDD27A96ED007AF4EE7C
:10282000477AF1EE10FA07D0C6ED007A0121304662
:1028300003F04CFE00E00026BEB19DF89731013B4D
:10284000032B41D8DFE803F002444D5501238DF8F6
:10285000983196F90030DA17689369925C210DF28D
:10286000D9201EF071FC8DF8D80209AF0026099618
:1028700040F26F1231460AA81EF0DEF8DFF88880B9
:1028800098F91820013A18BF0122394666A819F0B4
:1028900089F980B298F91830012B14BF0023012365
:1028A000079307230693059004970396A37E02934C
:1028B00004F1190301930B23009311A3D3E900231F
:1028C000E17E284617F068FF0DF5866DBDE8F081C2
:1028D00001238DF89831B6F90030DA1768936992C0
:1028E000BCE701238DF898313368DA176893699251
:1028F000B4E702238DF8983133686893AEE700BFE0
:10290000D5A4D139F922B6A7302A00302DE9F041FB
:1029100092B006460C460EA9204619F081F8002810
:1029200037D19DF83830012B36D000250A950B950C
:102930000C950D9501238DF830300895ADF8245095
:102940008DF82650DFF8908098F9182008AFD21A39
:1029500018BF012239460AA819F07AF880B298F90E
:102960001830012B14BF002301230793072306937C
:10297000059004970395A37E029304F11903019334
:102980000A23009312A3D3E90023E17E304617F017
:1029900003FF12B0BDE8F08104F044FD03F016FB24
:1029A00004F052FA04F084FB064D0749284604F06F
:1029B00061FB064905F5BA7004F05CFBB5E700BFA2
:1029C000AFF30080802A003060680608D4730608E0
:1029D000CDD269EBC51A133B302A003000B583B065
:1029E000084601A918F07EFE58B9074B1B68586DC0
:1029F00003681B689DF80410FF2914BF0021012102
:102A0000984703B05DF804FB2C2A003000B5A3B052
:102A1000084601A918F096FD10B123B05DF804FB3B
:102A20009DF805300DF106020021024805F0F6FA86
:102A3000F3E700BF802A003008B5002309F090FEBC
:102A4000024B012283F8602308BD00BF302A00300A
:102A5000F0B52DED028B97B00846384B012283F874
:102A6000C82301A918F02AFE002862D1002706E039
:102A7000324621462846FFF7DFFF0137FFB29DF8B7
:102A80000430BB4255D916AB03EB870313F8525CF5
:102A9000ED00EDB213F8514C6408E400E4B213F811
:102AA000506CF600F6B2264809F07EFEC343C3F32D
:102AB000C01364280CBF002303F00103002BD7D000
:102AC00007EE900AB8EEE78ADFED1E7A28EE278A35
:102AD00007EE905AF8EEE77A67EE887AFDEEE77A2D
:102AE000FF22002117EE903A18B202F049FAC5B25F
:102AF00007EE904AF8EEE77A67EE887AFDEEE77A1D
:102B0000FF22002117EE903A18B202F039FAC4B24F
:102B100007EE906AF8EEE77A27EE888ABDEEC88A5B
:102B2000FF22002118EE103A18B202F029FAC6B2BC
:102B30009EE717B0BDEC028BF0BD00BF302A00301D
:102B4000942D00300AD7233C30B585B00C4602A93D
:102B5000204618F07FFE60B90C4BD3F8E823D3F879
:102B6000EC3352EA030106D1D4E90001074BC3E973
:102B7000FA0105B030BD064DDDE90201CDE90001E5
:102B8000284608F0A3FF45E91201EDE7302A00309E
:102B9000682E003010B5C4B00846694618F07EFAB9
:102BA00068B9BDF80030B3F5007F0AD00E4CDDE9FE
:102BB0004223C4E9EE2310F083FBC4F8C40344B0FD
:102BC00010BDBDF8023007EE903AF8EE677A9FED3F
:102BD000077A67EE877A9FED067A67EE877A024B6F
:102BE000C3EDF07AE2E700BF302A00300AD7233C79
:102BF00035FA8E3C00B583B00849684618F0FCF9F8
:102C0000BDF80400642303FB00F0BDF80030B0FB06
:102C1000F3F080B203B05DF804FB00BF982E0030E3
:102C200010B58EB03A4817F04DFD28B1394B00224F
:102C30001A7001200EB010BD10F04AFB0446354B4F
:102C40001B78002B53D14FF4C870FFF741FC204490
:102C500000F516702E4AC2F8CC0F2F4B1B785B0084
:102C6000DBB28DF8303092F8D02F72B943F0010307
:102C70008DF83030264A92F8D23F0133DBB282F829
:102C8000D23F03F0010382F8D23F08A8FFF72AFCE5
:102C90001F4B93F8D01FC1F11004E4B2062C00D9E9
:102CA0000624224608AB19440DF131001DF0B6FE92
:102CB000174890F8D23F012202FA03F3002106914F
:102CC000DBB20593144404940CAB039318230293D2
:102CD000124B019300920CA3D3E9002317F0F4FCEC
:102CE000011E0BDB00200A4B83F8D00FA2E7FFF791
:102CF00081FF01460A480DF097FAA4E709480DF054
:102D000093FAEFE7AFF30080401DA12026812A0B44
:102D1000982E0030D4250030882E0030843E0030BC
:102D2000F44206082C43060808B5D0E900230248FF
:102D300017F094FD08BD00BF982E003038B504464A
:102D4000174BD3F8C80F50B10268A24218D00546FD
:102D50008068B8B10268A242F9D104301EE00C21AB
:102D600001201CF051F80E4BC3F8C80FB0B104603D
:102D7000D3F8C82F00219160D3F8C80F04300DE0BC
:102D800004300BE00C2101201CF03EF8A86028B1B3
:102D90000460AB6800229A60A868043038BD00BFA8
:102DA000982E0030F0B589B007460E4615461C46F1
:102DB000114817F087FC08B909B0F0BD47EA054093
:102DC000FFF7BCFF0028F7D00C4B93F91830012B0C
:102DD00014BF00230123069307230593BDF83C305D
:102DE00004930E9B03930294019000953A46334658
:102DF000014817F069FCDFE7982E0030302A0030D8
:102E000030B585B010F05CFA154BA3FB003080099B
:102E1000144C2060144B1B68586D03685B6E984718
:102E20002081124B93F9182002AD013A18BF0122FC
:102E30002946204618F01EFD80B201900095182307
:102E400040F2551204A1D1E90001FFF7ABFF05B034
:102E500030BD00BFAFF30080F1C6A7C1D068080F36
:102E6000D34D62108C2E00302C2A0030302A0030D6
:102E700030B5ABB0002118918DF8A4108DF8A510D5
:102E8000402219A81DF0D8FD2B4C00E008342B4B34
:102E90009C4248D06368002BF8D02278284B13441A
:102EA00093F80C33012BF1D101238DF80C30002362
:102EB0008DF80D306068026895689FED1D7B8DED83
:102EC000007B0DF10D0203A9A8479DF80C30002BE3
:102ED000DCD04822002106A81DF0AEFD6068036822
:102EE0005D690DF10E0304AA18A9A8470028CDDDDD
:102EF0009DF8A40001F0F4F802468DF85C009DF8FE
:102F0000A5308DF85F3019A907A81DF087FD189B23
:102F1000069323788DF85D30DDE9042306A909487E
:102F200017F038FEC0E72BB030BD00BFAFF3008014
:102F300000000000000000006C3E00307C3E0030CD
:102F4000302A0030982E00302DE9F04395B02CE067
:102F50000834344B9C421ED060680028F8D095F8A5
:102F600046C022784CFA02FC1CF0010FF0D02E4B28
:102F7000134493F80C33012BEAD10368D3F8109073
:102F80000023009332463B4602A9C8470028DFDCF5
:102F90004FF00008DCE7B8F1000F33D0234C204697
:102FA00017F054FC002384F8D13F204817F04AFC66
:102FB00088B30546002102918DF84C108DF84D1014
:102FC000402203A81DF038FD95F8440001F06CF88C
:102FD0008DF84C0095F84420291D03A81DF01EFD16
:102FE0002B6843F00043029395F847308DF84D303D
:102FF00010F072F90E4E861941F100070D4C4FF09A
:103000000108A6E7094B93F8D13F072B06D80133F7
:10301000064A82F8D13F15B0BDE8F083034817F0A7
:1030200015FCF8E77C3E0030302A0030982E003046
:1030300040420F006C3E00302DE9F041CAB0064618
:103040000C464FF04055E022002128461DF0F4FCCC
:10305000434B2B60A38A013B9BB2C92B02D94AB0D8
:10306000BDE8F0813F4B009300230822194620461B
:1030700017F02EFC00250827A38A013B9D420CDA9D
:10308000394B2B440093002308223946204617F081
:103090001FFC08370135EDB2EEE74FF040531B7DC2
:1030A0001BB9E27E4FF040531A75304617F00AFB09
:1030B0004FF040535875002529957D2229462AA8AE
:1030C0001DF0BAFC8122294608A81DF0B5FCDFF8E6
:1030D000A08098F9182029AF013A18BF012239467B
:1030E00008A818F073FC98F91830012B14BF0023BE
:1030F000012307930723069380B205900497039555
:10310000A37E029304F1190301932823009312A3D1
:10311000D3E90023E17E304617F03EFB32235C1EEC
:10312000E4B253B1FFF710FF104B1B68186D036832
:103130005B68012198472346F1E70D48FEF7BAFF87
:10314000304617F0BFFA03460A4818431CF040F80F
:10315000FFF7DEF8AFF3008026417272DF25D7B7A4
:103160009AAD44C514000030160000302C2A0030FF
:10317000302A0030000008B038B505460C4617F07C
:10318000A1FAE8B1E38A282B26D81AB2DAB1013BBA
:10319000272B18D8DFE803F03B17176845171717D8
:1031A0001759541717171717171717171717171730
:1031B0001717171717171717171717171717174076
:1031C000237E022B00D038BDE38A012BFBD12146A0
:1031D0002846FFF79FF9F6E740F24C42934239D078
:1031E00008D944F627629342EDD121462846FFF7DD
:1031F000D1FCE8E740F22642934230D040F2394217
:103200009342E0D121462846FFF722FCDBE7214626
:103210002846FFF7DBF9D6E721462846FFF70CFFE3
:10322000D1E714480DF000F8134B1B68186D0368C4
:103230005B680A2198471148FEF73CFFFFF768F8E2
:1032400021462846FFF768FABDE721462846FFF7E2
:103250005DFBB8E721462846FFF7C0FBB3E72146F0
:103260002846FFF7D3FBAEE721462846FFF76CFC64
:10327000A9E700BF604306082C2A0030302A00303E
:10328000F0B52DED028B83B006465F4C0023237111
:103290000123637110F01CF85C4BA3FB0030800924
:1032A0002060B6F90230002B03DB7F2B01DC584A8B
:1032B0001370584B93F90E3033B15648002300F881
:1032C0000E3F012103F002F90023194601E001330A
:1032D000DBB2012B0CD8F21892F90C20012AF6D19E
:1032E00006EB830250684C4A9042F0D10121EEE790
:1032F00009B1002333E096F90C30013B07EE903A18
:10330000F8EEE77AF0EEE77A9FED448AF4EEC87AB9
:10331000F1EE10FA4FF0010333734CBF1946002150
:1033200006F10C0003F0D2F872683D4B134407EE2F
:10333000903AF8EEE77AF0EEE77AF4EEC87AF1EE3A
:1033400010FA354B73604CBF01210021301D03F092
:10335000BDF8CEE7334A082191610133DBB2002B7F
:10336000F8D000240DE02A681768A21D06EB82023F
:1033700006EB84010123526849682846B8470134A6
:10338000E4B2012C28D843F2B07000F0F3FD0546FA
:103390000CF002F8244A42F82450244A02EBC401FB
:1033A0004D6002F834403219117B82F80C13204A28
:1033B00002EBC400017142F83450002DDFD096F9C1
:1033C0001820012ACFD02A68576806EB840301220F
:1033D00059682846B847D2E7164800230193164B90
:1033E0000093164B4FF47A6200F1280117F046F96A
:1033F000074B197819B903B0BDEC028BF0BD0D482D
:1034000017F058F9F7E700BF8C2E0030D34D62104B
:10341000882E0030302A003040420F000000003477
:10342000C0BDF0FF000C02587C3E00306C3E003006
:10343000943E0030982E003051230408793104085E
:1034400090F9D931002B7DD070B596B0044690F834
:1034500007330BB300F5E275284608F051FCD4F8A9
:10346000D46394F80813284608F0ECFBC0B2C0EB14
:10347000401005EB8000D0F890309E420CD094F8BC
:103480000813284608F0DEFBC0B2C0EB401005EB85
:10349000800090F831300BB916B070BD94F8081365
:1034A000284608F0CFFBC0B2C0EB401005EB80000F
:1034B000D0F89030C4F8D43394F80813284608F0B4
:1034C000C1FBC0B204F5FA75C0EB4010800050306B
:1034D000054404353422002109A81DF0ADFA00236B
:1034E000022B0FD805EB8302D2ED007A9FED187AFC
:1034F00067EE877A16AA02EB830242ED0D7A01335A
:10350000DBB2EDE700230293039304930593069344
:1035100007938DF820300F4B93F9182002AC013A35
:1035200018BF0122214609A817F0EEFD80B20190D4
:103530000094182340F2E93203A1D1E90001FFF71A
:1035400031FCA9E7704700BFF2C20B46A9D4A7E23D
:103550006F12833A302A003090F9503003B9704727
:10356000F0B5ADF5277D044600F15005284604F07E
:10357000E5FCD4F8D82394F8583104EB0313D3F8BE
:103580009C309A4200F06581C4F8D8334FF4D07271
:1035900000213EA81DF050FA94F8586194F8BA3111
:1035A00033B1A82303FB064393F8A930012B45D878
:1035B000A82303FB064393F8A930012B3ED901232E
:1035C00084F830343146284604F060F9CDE93E01F4
:1035D00094F85811284604F0D9F9CDE94001409AF1
:1035E000419B134337D100238DF80831A82101FBFB
:1035F0000641D1F8C000C217970047EA90778300D0
:103600001B1842EB0702DB18524144934592D1F854
:10361000BC00C217970047EA907783001B1842EB63
:103620000702DB18524146934792D1F8B83003EBBA
:1036300083035B0048934993002223E094F83034DD
:10364000002BBCD10FF040FECDE93E01002200234B
:10365000CDE94023C3E702238DF80831C6E704F122
:103660005003A82106FB01F188310B44043303EB1E
:103670008203196802F10C033EA800EB8303196072
:103680000132D2B2022AEAD994F85811A82303FBD6
:10369000014393F8DA308DF8343194F8BA3133B10C
:1036A000A82303FB014393F8A930012B0FD8A823CB
:1036B00003FB014393F8A930062B0FD8DFE813F082
:1036C00007000700CC00D500DE00E700F100002372
:1036D0008DF835318DF836318DF8373106238DF878
:1036E000383103AA284604F0A1F838B1DDED037A99
:1036F00067EEA77ACDED507ACDED4F7A04AA94F813
:103700005811284604F0A2F828B1DDED047A67EEDE
:10371000A77ACDED517A05AA94F85811284604F0FD
:1037200075F848B1DDED057A67EEA77ACDED547AEC
:10373000CDED537ACDED527A00260696DA22314647
:1037400007A81DF079F96C4F97F91820013A18BFB6
:10375000012206A93EA817F0DFFE80B2019006AB59
:103760000093182340F227425DA1D1E90001FFF741
:1037700019FB202231463EA81DF05EF994F858311D
:10378000A82202FB0343B3F8D62007EE102AB8EEB6
:10379000C77ADFED5A6A27EE267A8DED407AB3F8C4
:1037A000D83007EE903AF8EEE77A67EEA67ACDEDDC
:1037B000417A069607960896099697F91820013AD5
:1037C00018BF012206A93EA817F074FD80B201902F
:1037D00006AB0093182340F2254243A1D1E9000132
:1037E000FFF7E0FA3E963F96409694F85811284627
:1037F00004F0DCFC8DF8FC0094F95E30002B5AD10B
:103800009DF8FC30002B60D105AA94F85811284689
:1038100004F030FD08B1059B3E9306AC00230693EF
:10382000ADF81C308DF81E30334B93F91820013A57
:1038300018BF012221463EA817F014FC80B2019067
:103840000094182344F6236229A1D1E90001FFF76F
:10385000A9FA0DF5277DF0BD02238DF8353100233F
:103860008DF836318DF8373138E703238DF835314F
:1038700000238DF836318DF837312FE703238DF88B
:10388000353101238DF836318DF8373126E70323A2
:103890008DF8353102238DF8363100238DF837311C
:1038A0001CE703238DF8353102238DF836310123CF
:1038B0008DF8373112E7284604F0C2FC00289FD16A
:1038C000409B43F0010340939AE704A9284604F083
:1038D0008DFB002898D1409B43F00203409393E76F
:1038E0005F43370F00E741CAD2BFDBC3C4BDE89BCB
:1038F000697F00BBABB43CBA302A00300AD7233C06
:103900000FB430B5C3B046AC54F8045B7C22002140
:1039100023A81DF091F800210491772205A81DF03D
:103920008BF8039423462A465A210DF1AE000CF081
:103930002BFC592800D95A208DF8AD00104B93F973
:10394000182004AC013A18BF0122214623A817F021
:10395000B9FF80B201900094182343F6FF7206A1CC
:10396000D1E90001FFF71EFA43B0BDE8304004B0D2
:10397000704700BFAFF30080759D040C8EA454D631
:10398000302A003010B584B0CDE900016846FFF759
:10399000CBF9334C00E00834324B9C4208D0FFF79F
:1039A00029F94628F7D921782F480CF03DFCF2E799
:1039B000FFF726FA2D4B93F90E40002C3DD0E4B2D0
:1039C00093F90E3033B12948002300F80E3F01214E
:1039D00002F07CFD2A2C19D02B2C22D04FF4FA6156
:1039E00003A800F04BFC224B1C68206D03685B6849
:1039F0004FF47A719847606D0368DB6A9847B0B1FD
:103A0000012825D01B48FFF77BFF13E01A48FFF77A
:103A100077FF174B1B68186D03685B686421984734
:103A2000F4E71648FFF76CFF154B9847D6E71548A3
:103A3000FFF766FF03A800F02DFC134B00225A711C
:103A40000FF046FC47F23053984205D804B010BD41
:103A50000E48FFF755FFEDE70D481BF0B9FBF5E702
:103A60006C3E00307C3E003070430608302A003047
:103A70002C2A0030F04306089C430608B043060891
:103A800038ED00E0C04306088C2E0030D84306080D
:103A9000263A09B038B504460FF01AFC05462F4BFC
:103AA0001B68C31A322B0FD92D4B1B7863B12D49DC
:103AB0000B7801335A4203F01F0302F01F0258BF74
:103AC00053420B70254B18600FF0FAFB264BD3F8CE
:103AD000CC3F984215D8254B1B68EB1AB3F57A7F7B
:103AE00012D294F92430B3B194F8FC33BBB9204618
:103AF000FFF7A6FC2046FEF7CBFA0FF0D5FB0446F5
:103B000024E0FFF78DF8E6E7184B1D600FF0E4FBAB
:103B1000FFF738FFE5E72046FFF71EFDE7E7002344
:103B200084F8FC3394F8FA2394F8F91394F8F80322
:103B3000FEF782FFDBE70E4B1B68186D03689B687E
:103B400040219847FFF700FAFFF792F90FF0ACFB1E
:103B5000001BB0F57A7FEED338BD00BF8C3E00303D
:103B6000D4250030903E0030982E0030883E003042
:103B70002C2A003008B54FF6FF710120FEF7DAFB62
:103B800008BD00BF30B583B005463A4C40F206226E
:103B90000121204618F0A2FD40F206220221204613
:103BA00018F09CFD344BD3F8E82042F48002C3F8AF
:103BB000E820D3F8102122F48002C3F81021D3F8B2
:103BC0001021D3F8902042F48002C3F89020D3F85B
:103BD000902022F48002C3F89020D3F89030274C34
:103BE000236823F001032360236823F480532360B8
:103BF000236823F470632360214B2361236823F43B
:103C000000332360636823F4006363604023A36090
:103C1000A36843F40043A360AA23E360E36843F48A
:103C20000043E3600321212019F062FC236843F084
:103C300002032360236843F004032360236843F0F6
:103C400008032360236843F020032360236843F0C4
:103C5000010323600B4B1B68186B0368DC6800953D
:103C6000094B019302AB13E90C000849A04703B0CC
:103C700030BD00BF001402580044025800580040F4
:103C8000380F30002C2A0030193E04080C44060876
:103C900090F9243013B9012380F800344FFA82FCE4
:103CA000D309002908BF43F0010323B102F07F02CA
:103CB00080F8FB23704790F8FB33022B11D0032BC5
:103CC00016D0012B06D0013380F8FB33012380F896
:103CD000FC3370470CF00F0C4CEA021280F8FA2308
:103CE000F1E70CF00F0C4CEA021280F8F923EAE736
:103CF0000CF00F0C4CEA021280F8F823E3E700BF47
:103D0000092B00D97047F0B585B005460C46114621
:103D10001F461A4601A81CF081FE242C08BF092F5B
:103D200038D19DF804209DF805301B0243EA024378
:103D30009DF8062013435B421A0C8DF804201A0AE2
:103D40008DF805208DF806309DF807209DF8083085
:103D50001B0243EA02439DF8092013435B421A0CFD
:103D60008DF807201A0A8DF808208DF809309DF883
:103D70000A209DF80B301B0243EA02439DF80C20F9
:103D800013435B421A0C8DF80A201A0A8DF80B2097
:103D90008DF80C30D5F8CC0310B10026354619E06B
:103DA000082000F0E7F8C5F8CC0304719DF8042062
:103DB00042710122827105B0F0BDA8B104AB2B4461
:103DC00013F80C3C4371012383711C44E4B2013F9E
:103DD0001D44EDB2002FEED00028EED00279A242B1
:103DE000EBD006460068F7E7082000F0C3F8306023
:103DF00068B1047104AB2B4413F80C3C43710123EC
:103E000083711C44E4B2013F1D44EDB2E2E7014876
:103E10000FF022FA1444060810B582B09DF8104045
:103E20000094FFF76DFF02B010BD00BFD0F8CC3397
:103E300036291BD023B11A798A4201D01B68F9E7D1
:103E4000B3B134290ED123B11A79242A01D01B68C9
:103E5000F9E77BB19A790AB90020704700229A717C
:103E60008020704700229A7158797047222070474D
:103E7000002070470020704709B980F8C9237047B7
:103E800010B5044610F0080F16D0C0F34642304B70
:103E900083F8FE23C0F3004283F8FF23002183F858
:103EA000FD1322B12B4A936943F001039361294A20
:103EB000D36943F00803D36114F0040F17D0254BE6
:103EC0005A6AD2B2224B93F8FE33232B07D9552BD3
:103ED00007D11F4890F8FD13FFF7DAFE01E0202B11
:103EE00013D21B4A92F8FD33013382F8FD3314F0EC
:103EF000020F18D0164B93F8FE33232B0BD9552BFA
:103F00000BD1144B00229A6207E0114890F8FD1380
:103F1000FFF7B2FFE5E7202B0ED20D4A92F8FD33F2
:103F2000013382F8FD3314F0200F04D0094AD3691D
:103F300043F02003D36110BD054890F8C91390F8F1
:103F4000FD331944C9B2FFF771FF024B9862E4E7F1
:103F5000302A00300058004008B5034B9869FFF73D
:103F60008FFF17F063FF08BD0058004000487047FE
:103F70004844060808B500B9012001211AF044FFA1
:103F800008BD00BF18B108B51AF044FF08BD70475E
:103F900008B500B9012001211AF036FF08BD00BFA5
:103FA00018B108B51AF036FF08BD704710B50268A1
:103FB00054681A46A04710BD002070470120704782
:103FC000002070470020704700207047704700BFF6
:103FD00000207047704700BF704700BF30B583B006
:103FE00084460D46043003C802AA02E9030069B101
:103FF0000C461B8813F0040F08D1DCF80030DB6B93
:10400000604698472A46C1B20098A047012003B0F5
:1040100030BD00BF82B0EC468CE80600031D9CE872
:10402000030083E80500012002B0704770B598B026
:1040300004460E46031D93E8030018AB03E9030092
:1040400069B10D46BDF8703013F0040F0AD1236832
:10405000DB6B204698473246C1B21698A84701202C
:1040600018B070BD00220023CDE900230021ADF877
:10407000081003918DF850108DF85110402204A8BB
:104080001CF0DAFC4622314603A81CF0C7FC0FF0F6
:1040900023F9CDE900010423ADF8083023681B6C37
:1040A000694620469847DAE7082818D90C280BD922
:1040B00010280BD914280BD918280BD920280BD974
:1040C00030280BD90F207047092070470A2070470D
:1040D0000B2070470C2070470D2070470E20704752
:1040E000082818D909280BD00A280BD00B280BD088
:1040F0000C280BD00D280BD00E280BD04020704779
:104100000C2070471020704714207047182070470B
:104110002020704730207047406870470146806813
:1041200038B110B582B00468A4680091A04702B00D
:1041300010BD0020704700BF30B583B004460D4667
:10414000072200F10C0101A800F0B2F863682B43CC
:10415000636001A800F0CEF8012003B030BD00BFBD
:1041600030B583B004460D460E2200F10C0101A8C3
:1041700000F09EF8636823EA0503636001A800F07D
:10418000B9F8012003B030BD30B583B004460D4608
:104190001D2200F10C0101A800F08AF8A56000239F
:1041A000636001A800F0A6F8012003B030BD00BF95
:1041B00008B54368984708BD08B58368984708BDA7
:1041C00010B4044C0460044C0460416082605DF8EB
:1041D000044B7047F44406080445060800B585B052
:1041E0000B4600F1040E0A4A0DF1040C07CAACE8B4
:1041F0000300ACF80020092B08D804AA134413F8D4
:104200000C3C5EF8230005B05DF804FB0020FAE7E3
:10421000943C060808B503689B68984708BD00BF32
:10422000704700BF00207047704700BF007B00F060
:1042300001007047704700BF00207047704700BF03
:1042400082B002AB03E90600002002B0704700BF55
:1042500081608280704700BF836873B110B50446E7
:10426000027B12F0010F07D142F00102027398475E
:10427000237B6FF30003237310BD704710B5044612
:10428000034B1B68186D03681B699847204610BDD7
:104290002C2A003010B50446044B1B68186D0368C7
:1042A0001B6900219847204610BD00BF2C2A003012
:1042B000F8B50446154601600A4B1E68306D036868
:1042C0001B6C9847074610B1736DA3F842502068E5
:1042D00003689B6898471FB1736D0022A3F84220C2
:1042E0002046F8BD2C2A003010B50446FFF7E0FF49
:1042F000204610BD10B5044600680368DB68984787
:10430000204610BD002070470020704700207047F5
:104310000020704700207047704700BF00207047A2
:1043200003207047002070470020704700230B7067
:10433000704700BF00207047704700BF00207047E3
:10434000704700BF704700BF4FF48050704700BFF8
:1043500000207047704700BF704700BF704700BF24
:1043600000207047704700BF002070470020704752
:10437000704700BF00207047002070474368C26844
:10438000934201D28268D1544368013343600120D3
:10439000704700BFF8B505460C46002607E02B68BD
:1043A0009B6814F8011B2846984706443A46571E56
:1043B000002AF4D13046F8BD002070474FF0FF309E
:1043C000704700BF002070470020704738B590F854
:1043D0009C308B4200D138BD04460D4680F89C10BD
:1043E0000EF06EFFC4F8A00023685B682046984773
:1043F0000028F0D184F84D50EDE700BF08B508461D
:104400001AF008FD08BD00BF08B501201AF0FCFC39
:1044100008BD00BF30B585B00C46194615469AB1A7
:10442000531E0D4A00920D4A0092002201920294FE
:104430000393089A684600F04FF80198854205D921
:104440000023235405B030BD1346EAE7002DF9D010
:10445000013D00236355F5E7384606087045060818
:1044600008B410B585B007AC54F8043B039400942D
:10447000FFF7D0FF05B0BDE8104001B0704700BFA6
:10448000F8B505460E46002703E07B1CF0559FB2A9
:104490002246531E9CB242B12B685B69284698475E
:1044A000B0F1FF3FF1D1384600E03846F8BD00BF1B
:1044B0000EB400B582B003AA52F8041B019203683F
:1044C0005B68984702B05DF804EB03B0704700BF2B
:1044D00008B500F001F808BD2DE9F04F8DB0054694
:1044E0000E46059204E02B689B68284698473E4696
:1044F000374617F9011B11F0FF0172D02529F2D1BF
:10450000B71C96F90110C9B22529ECD04FF000086C
:104510004446C1460CE049F0010903E049F00209B4
:1045200049F0040917F9011B11F0FF0100F0BC80EC
:10453000B9F11F0F2ED8A1F12002102A2AD801A309
:1045400053F822F0214504089545040895450408D0
:104550008F450408954504089545040895450408C9
:1045600095450408954504089545040895450408B3
:104570001D45040895450408894504089545040827
:10458000954504081745040849F00809CAE749F0A9
:104590001009C7E7B9F17F0F2CD8A1F13003DBB2C6
:1045A000092B13D819F0400F07D008EB88025200EE
:1045B000D2B213445FFA83F8B4E704EB84025200EA
:1045C000D2B21344DCB249F02009ABE72E2905D062
:1045D0006C290CD06829A5D03E4611E019F0400F97
:1045E00002D00DB0BDE8F08F49F040099AE749F0DC
:1045F000800997E719F0800F58D06C2951D03E46BA
:10460000A1F14503DBB2022B52D9A1F16503DBB264
:10461000022B52D9632900F03682732900F04382BD
:10462000692918BF642900F06D82752900F0A882FD
:1046300029F0060A1FFA8AFA702900F0B18200F206
:10464000A582582900F0AF826F29CAD108231AF435
:10465000807F40F0B3821AF0800F00F0C182059A8B
:10466000111D0591106806AF03F01A02394600F0DB
:104670005BFBC71BFFB22AF0800A1FFA8AFA1AF006
:10468000400F00F0B8822AF001039BB2474580F04A
:10469000C8820AF01402102A00F0A782C1469A4686
:1046A000AAE249F480793DE73E46A9E73E46A7E7FE
:1046B00049F010092031C9B203E029F010091FFAAE
:1046C00089F9059B073323F0070303F108020592DC
:1046D00093ED000BB7EEC00B19F0400F01D14FF076
:1046E000060829F0C0091FFA89F7652909D066294B
:1046F00045D0B8F1000F06D008F1FF385FFA88F80E
:1047000001E047F0400717F0800F0ED0F0EEC07ABE
:104710009FEDA17AF4EEC77AF1EE10FA05DD27F0ED
:10472000C00747F040073FB2BFB217F080030493C1
:1047300028D043463B2B28BF3B2301335FFA83FB42
:104740000721002306930793089309930A93CDF852
:104750002B305A4606A80FF02FFA029082469DF899
:104760001830019303F00903012B17D017F0020F43
:1047700034D117F0040F34D10023039310E047F035
:104780008007C0E7B8F10A0F03D841464FF0000B8D
:10479000D7E74FF0000B0A218846D2E72D23039379
:1047A000019B13F00C091FD1049B002B5AD0029BD4
:1047B0005B445FFA83FB019B13F0100F03D09DF85D
:1047C0001930312B49D04FFA8BF3002B40F3A080E6
:1047D000BBF1080F49D94FF0080B46E02B23039398
:1047E000DEE720230393DBE7039B8BB104239C428A
:1047F00010D9E41AE4B217F0080F0CD12B689B68AB
:10480000202128469847631E13F0FF04F6D102E0EA
:104810000323ECE70024039919B12B689B68284611
:104820009847019B13F0080F02D1DFF8708108E070
:10483000DFF86C8105E02B689B682846984708F1F3
:10484000010898F9001011F0FF0100F0688217F0DC
:10485000100FF0D02039C9B2EDE70BF1FF335FFA4A
:1048600083FBB0E717F0400F2AD017F080030493C2
:1048700053D0029B23EAE3730133039A02B101335D
:10488000B8F1000F02D008F1010213449C4203DD8D
:10489000DBB2E41A5FFA84F917F0090F3FD00399ED
:1048A00019B12B689B682846984717F0080F42D02B
:1048B000049B002B00F08D80029B23EAE37457E0F9
:1048C000029B984506DB13F1040F0FDB47F08007CE
:1048D000434600E043465BB15A1C0CA90A4412F857
:1048E000182C302A04D1013BDBB2F4E74346F2E74F
:1048F000984617F0800FB8D001335FFA83FB029B14
:10490000984508DDDBB2A8EB03085FFA88F8ACE74E
:104910004FF0010BA9E7C846A7E70523ADE74C46D2
:104920003CB12B689B68202128469847013CE4B2A3
:10493000F6E7A146B3E74C463CB12B689B683021B3
:1049400028469847013CE4B2F6E7A146B0E72B6859
:104950009B682E21284698470DE03021013CC8F184
:104960000003A3421EDCE9B12B689B6828469847E8
:10497000B4F1FF3FEBD05445EFDCAAEB0B03A342AD
:1049800007DAAAEB040301330CAA134413F8181C2A
:10499000E4E73021E2E700BF7F96184B6046060847
:1049A0005C460608029BA34206D0002969D02B680A
:1049B0009B682846984764E09DF81930352B06D847
:1049C000F3D1019B13F0100FEFD13121EFE731212B
:1049D000EDE79DF81910312903D0019B03F0EF0397
:1049E00001932B689B6828469847B8F1000F20D1A7
:1049F0002B689B6817F0100F32D045212846984746
:104A0000029B002B04DB6BBB019B13F0100F2BD020
:104A1000029BC3F1000A2D212B689B68284698470A
:104A20003021BAF1090F21DD0131C9B2AAF10A0A18
:104A3000F7E72B689B682E212846984702242B68AD
:104A40009A6823460134E4B20CA90B4413F8181CED
:104A50002846904708F1FF3818F0FF08EFD1C7E764
:104A60006521CBE72B21D7E72B21D5E72B689B6866
:104A7000284698472B689B680AF13001C9B228463E
:104A800098474C464BE1059B1A1D05921B688DF813
:104A900018304FF0010806AF19F0080F13D02B465D
:104AA000454698461EE0059B1A1D05921F6819F0A1
:104AB000400F05D0414638461CF046FB8046EBE7E8
:104AC0004FF0FF31F7E7444507D92B689B68202159
:104AD00028469847013CE4B2F5E72B464546984600
:104AE00000E0013D002D00F01181D8F800309B68F6
:104AF00017F9011BC9B240469847002CF1D0013C80
:104B0000E4B2EEE719F4807F1CD0059B073323F055
:104B1000070303F1080205921868596829F0900903
:104B20001FFA89FA002907DB06AF0A233A4600F08C
:104B300055F9C71BFFB2A2E5404261EB41014AF0C3
:104B4000800AF1E719F0800F11D0059B1A1D05921C
:104B5000186829F090091FFA89FA00280CDB06AFC3
:104B60000A22394600F0E0F8C71BFFB287E5059B33
:104B70001A1D05921868ECE740424AF0800AEEE7F9
:104B800029F010091FFA89FA0A2360E578297FF4D1
:104B900028AD1AF0100F01D04AF0040A102356E590
:104BA0004AF0100AF5E719F0100F04D04AF0060A8F
:104BB0004FF404734BE54FF4047348E5059A07324C
:104BC00022F0070101F10802059206AF03F01A0373
:104BD0003A46D1E9000100F001F9C71BFFB24AE5EE
:104BE000059A111D059110683DE52AF0110A1FFA7A
:104BF0008AFAC14600E0B9461AF0100F19D07B1EA0
:104C00000CAA134413F8183C302B0DD009F1010302
:104C1000DBB21AF0040F3AD009F102095FFA89F900
:104C20000EE0B9469A46E7E72AF0160A1FFA8AFA12
:104C300006E01AF0860F03D009F101095FFA89F93D
:104C40001AF0080F25D04C453DD9A4EB0904E4B275
:104C50001AF0100F3BD02B689B68302128469847EC
:104C60001AF0040F07D02B689B681AF0020F2CD0A3
:104C700058212846984747453BD22B689B683021EE
:104C80002846984708F1FF385FFA88F8F3E7994615
:104C9000D6E71AF0010F08D04C4512D9A4EB090849
:104CA00057FA88F85FFA88F8A1464C45CBD92B68AB
:104CB0009B6820212846984709F101095FFA89F984
:104CC000F3E7B846F1E70024C2E77821D1E71AF00C
:104CD000860FD0D01AF0020F09D120211AF0800FD0
:104CE00000D02D212B689B6828469847C3E72B21CD
:104CF000F4E72B689B68013FFFB20CAA3A4412F814
:104D0000181C28469847002FF3D108E0454606E0D6
:104D10002B689B68202128469847013CE4B2002C70
:104D2000F6D1FFF7E5BB00BF03460846082A3FD08F
:104D3000102A48D010B50022D9B223F00103023363
:104D400042F100024FEA530C4CEAC27C1CEB030315
:104D500042EB52024FEA131C4CEA027C1CEB030CA0
:104D600042EB12124FEA1C2343EA026313EB0C0CD2
:104D700042EB12224FEA1C4343EA024313EB0C03BB
:104D800042EB1242D31842F1000C1B0943EA0C73A8
:104D90004FEA1C128646C3EB4314C3EB840401EBB9
:104DA000440130310170013053EA1C11C4D110BDEF
:104DB00003F0070230320270DB08F9D1704700F8C7
:104DC000012B1B0908D003F00F0101F13002392A31
:104DD000F5D901F13702F2E7704700BF844610466B
:104DE000082B41D0102B58D010B55FFA8CF22CF064
:104DF000010C1CF1020C41F100034FEA5C0141EA95
:104E0000C37111EB0C0143EB53034FEA111C4CEA45
:104E1000037C1CEB010143EB13134FEA112C4CEA0A
:104E2000036C1CEB010143EB13234FEA114C4CEADA
:104E3000034C1CEB010C43EB134313EB0C0C43F141
:104E400000034FEA1C1C4CEA037C19098646CCEB94
:104E50004C14CCEB840402EB44023032027001307B
:104E60005CEA1313C1D110BD0CF00703303303709B
:104E70004FEADC0343EA4173CA089C4611461343D8
:104E8000F2D1704700F8013B4FEA1C1343EA01736B
:104E90000A099C461146134308D00CF00F0202F198
:104EA0003003392BEED902F13703EBE7704700BF2F
:104EB00030EE600AB0EEC00ADFED047AB4EEE70A25
:104EC000F1EE10FA4CBF01200020704700000034C2
:104ED00008B51BF023FBB4EE400AF1EE10FA00D641
:104EE00008BD9FED010AFBE70000000008B5DFEDFB
:104EF000070A1BF0E9FAB5EEC00AF1EE10FA00D489
:104F000008BDDFED027A30EE270AF9E70000B4436E
:104F100010B52DED028BB0EE608AF0EE418AB4EE52
:104F2000400AF1EE10FA0CD6B4EEE00AF1EE10FAF7
:104F300016D4B4EEC10AF1EE10FA14DCBDEC028B0B
:104F400010BD044606F0B2FFA2B24FF4806106F035
:104F500097FF38EE288AB6EE000A28EE000AEDE741
:104F6000B0EE600AEAE7B0EE410AE7E7884202D312
:104F7000904202D87047084670471046704700BFFD
:104F8000884202DB904202DC7047084670471046B8
:104F9000704700BF094A136899B21B0C49F26900B7
:104FA00000FB01331360064B186882B2000C44F218
:104FB000506101FB0200186080B27047DC250030B0
:104FC000D825003091ED011A88B0D0ED077A90ED28
:104FD000010AD0ED040A21EE000A91ED007A61EE9B
:104FE000200A90ED036A21EE271AD0ED066AD0ED73
:104FF000005AE7EE060AD1ED027AA5EE870A90ED97
:10500000056AA7EE261AD0ED026A90ED087AE7EE5F
:10501000860AA6EEA70AA7EE871A08B0704700BF57
:1050200091ED005AD1ED015A91ED026AD0ED006A7E
:1050300090ED017AD0ED027A76EE856A37EE257A28
:1050400077EE867AC0ED006A80ED017AC0ED027AD3
:10505000704700BFD0ED006A90ED017AD0ED027A82
:1050600066EE806A27EE007A27EE800AC0ED006ABD
:1050700080ED017A80ED020A704700BF90ED007A62
:10508000D0ED017A90ED026AC7EE006A87EE807A71
:10509000C6EE007AC0ED006A80ED017AC0ED027ABA
:1050A000704700BFD0ED007AF4EE677AF1EE10FAA7
:1050B00010D6D0ED017AF4EE677AF1EE10FA09D647
:1050C000D0ED027AF4EE677AF1EE10FA6CBF0120AF
:1050D0000020704701207047D0ED007A9FED0F7AD5
:1050E000F0EEE77AF4EE477AF1EE10FA14DCD0ED48
:1050F000017AF0EEE77AF4EE477AF1EE10FA0BDC83
:10510000D0ED027AF0EEE77AF4EE477AF1EE10FA9B
:10511000CCBF01200020704701207047FFFF7F7F38
:1051200008B52B2900F20683DFE811F04400B40231
:10513000AB02960289027402980185017801A101EF
:1051400058002C00AE01BB014500FF002F011A01E1
:1051500071015A0151013801CA0159025002470236
:1051600045005800380225021602E401D901F0007A
:10517000E500DE00CF00C0008F007C006300ED0280
:10518000DA02C702D0ED017AD0ED005A9FEDE36A52
:1051900037EEA57AD0ED026A77EEE57AF1EE666A2F
:1051A00027EE067A67EE867AC0ED026A80ED017A14
:1051B000C0ED007A08BD90ED007AD0ED016AD0ED27
:1051C000027AB1EE477AF1EE666AF1EE677A80ED27
:1051D000017AC0ED006AC0ED027A08BDD0ED027A16
:1051E0000268F1EE677A436842600360C0ED027ABC
:1051F00008BDD0ED015AD0ED007AD0ED026A35EE4F
:10520000A77A9FEDC66A77EEE57AF1EE666A27EE39
:10521000067A67EE867AC0ED016A80ED027AC0ED0B
:10522000007A08BDD0ED007A90ED026ADFEDBB6A2E
:1052300037EE867A77EEC67A27EE267A67EEA67A7A
:1052400080ED027AC0ED007A08BDD0ED017A9FEDC5
:10525000B46ADFEDB46A9FEDB47A67EEA66AD0ED6A
:10526000005A27EE877ADFEDB14A67EE867A9FED26
:10527000B05A9FEDB04AA5EEA47A90ED026AE5EE31
:10528000857ADFEDAD4AE5EE846A9FEDAC5ADFED3D
:10529000AC5AA6EE057AE6EE257AE6EE246A80EDB3
:1052A000017AC0ED027AC0ED006A08BD90ED027A85
:1052B000D0ED007AB1EE477A4368F1EE677A836009
:1052C00080ED007AC0ED017A08BDD0ED007A90ED56
:1052D000017AF1EE677A8368B1EE477A0360C0ED38
:1052E000017A80ED027A08BD4268816803684160F6
:1052F0000260836008BDD0ED017A8268F1EE677AC2
:10530000036802608360C0ED017A08BDD0ED017AC8
:1053100090ED027AF1EE677A0368B1EE477A836026
:10532000C0ED007A80ED017A08BD90ED016AD0ED04
:10533000007AD0ED026A37EE867ADFED825A77EE98
:10534000C67A9FED766AF1EE666A27EE257A67EEF9
:10535000867AC0ED026A80ED017AC0ED007A08BD60
:1053600090ED026AD0ED007ADFED6C6A37EE867A56
:10537000436877EEC67A836027EE267A67EEA67AD0
:1053800080ED007AC0ED017A08BDD0ED027A436865
:10539000F1EE677A8360C0ED017A08BDD0ED025A64
:1053A000D0ED007AD0ED016A37EEE57A9FED5B6AC9
:1053B00077EEA57AF1EE666A27EE067A67EE867AD0
:1053C000C0ED026A80ED007AC0ED017A08BDD0ED33
:1053D000017A8368F1EE677A4360C0ED027A08BD16
:1053E000D0ED026AD0ED007ADFED4C5A37EEE67A66
:1053F0009FED546A77EEA67A436827EE067A8360BB
:1054000067EEA57A80ED007AC0ED017A08BD82686A
:105410004168036881600260436008BD90ED017AD5
:10542000D0ED027AB1EE477AF1EE677A80ED017A3B
:10543000C0ED027A08BDD0ED007A90ED016ADFED93
:10544000376A36EE677A77EE867A27EE267A67EE47
:10545000A67A80ED017AC0ED007A08BDD0ED007A21
:105460004368F1EE677A0360C0ED017A08BDD0EDC4
:10547000007AD0ED015A9FED296A37EEE57AD0ED3A
:10548000026A77EEA57A89E690ED007AD0ED027A8D
:10549000B1EE477AF1EE677A80ED007AC0ED027ADC
:1054A00008BD90ED016AD0ED007AD0ED026A36EECB
:1054B000677ADFED1A5A77EE867A9FED226A42E725
:1054C000D0ED027A90ED017AF1EE677A0368B1EEE1
:1054D000477A4360C0ED007A80ED027A08BDD0EDD6
:1054E000007A4268F1EE677A836882604360C0EDBB
:1054F000007A08BD90ED017AD0ED026AD0ED007A15
:10550000B1EE477AF1EE666AF1EE677A80ED027AE3
:10551000C0ED016AC0ED007A08BD00BFF304353F5D
:10552000DB26B93E46D0BC3EC9355BBF4F0DAABE97
:10553000C6AC6EBFCF78123E4D1F6BBFF184CABEA2
:10554000F63BCC23F30435BFF304353F81177E3F90
:10555000A296F93DA296F9BDD0ED017A90ED007AC0
:10556000F1EE677A8368B1EE477A4360C0ED007A66
:1055700080ED027A08BDD0ED016A90ED027AD0ED9F
:10558000007AF1EE666AB1EE477AF1EE677AC0ED25
:10559000016A80ED007AC0ED027A08BD90ED027AD2
:1055A000D0ED007AB1EE477A4368F1EE677A036096
:1055B00080ED017AC0ED027A08BDD0ED027A036871
:1055C000F1EE677A8360C0ED007A08BDD0ED007A15
:1055D0008368F1EE677A0360C0ED027A08BD90ED52
:1055E000026AD0ED007AD0ED016A37EE867A5FED7F
:1055F0002A5A77EEC67A1FED2D6AF1EE666A27EE1B
:10560000067A67EEA57AC0ED026A80ED007AC0EDF9
:10561000017A08BDD0ED017AD0ED006A5FED375A0E
:1056200037EEA67A1FED386A77EEE67A27EE257A0E
:1056300067EE867A80ED017AC0ED007A08BD90EDC4
:10564000007AD0ED017AB1EE477AF1EE677A80ED1B
:10565000007AC0ED017A08BDD0ED007AD0ED016A84
:105660005FED475A37EEE67A1FED4A6A77EEA67A83
:1056700027EE257A67EE867A80ED017AC0ED007A12
:1056800008BDD0ED017A0368F1EE677A4360C0EDA2
:10569000007A08BDD0ED007A90ED016A5FED566AA0
:1056A00037EE867A77EEC67A27EE267A67EEA67A06
:1056B00080ED017AC0ED007A08BDD0ED017A90ED61
:1056C000026A5FED5F6A36EE677A77EE867A27EEDA
:1056D000267A67EEA67A80ED027AC0ED017A08BDDF
:1056E000D0ED017A90ED026A5FED696A37EE867A55
:1056F00077EEC67A27EE267A67EEA67A80ED027AF2
:10570000C0ED017A08BDD0ED027A5FED706A1FED41
:10571000705A27EEA67A90ED006A67EE857A5FED03
:10572000735AA6EE257AE6EE267A80ED027AC0ED6F
:10573000007A08BD06F0BAFB40F211124FF4800166
:10574000BDE8084006F09CBB90ED020AD0ED017A5E
:1057500020EE000A90ED007A27EE077AA7EEA70A5E
:10576000B7EEC77AB7EEC00A37EE007BB5EE407BE6
:10577000F1EE10FA04D4B1EEC70BB7EEC00B7047D0
:10578000B0EE470B08B51AF073FEB7EEC00B08BDBC
:10579000024A0260024A0260704700BF788306082E
:1057A000D43E060838B5044605682DB128460EF0EB
:1057B0005BF82846FEF7E6FB024B6360024B636032
:1057C000204638BD78830608D43E0608012800D05C
:1057D0007047F8B54FF6FF73994200D0F8BD134CEF
:1057E00020460AF09FFC124F3A46124920461AF012
:1057F00059FB114C0026204640F8046B0AF092FC3D
:105800001420FEF7B7FB05469B210EF01BF8256020
:105810003A460A4920461AF045FB3146084801F04D
:1058200013FE0721074801F00FFED7E7A83E00301E
:105830003CCD003091570408C43E0030A557040801
:10584000F83E0030E03E003070B504460E46154686
:1058500013460246044801F063FE2B4622463146B9
:10586000024801F05DFE70BDF83E0030E03E0030C1
:1058700002EB820200EB8202507820B91BB1128A3F
:1058800012F0080F02D09840084470473F2098401B
:105890000844704710F0400F08D1C00908D0054BEC
:1058A0001B88184214BF0120002070470020704759
:1058B00001207047F03E0030013080B201E001303D
:1058C00080B2084B1B8883420AD900EB4003064A8A
:1058D000126802EBC3031B898B42F0D10120704791
:1058E00000207047FC3E0030003F0030038A13F078
:1058F000100F01D1C0687047C3681868704700BFB7
:10590000838A13F0100F01D100697047036918688A
:10591000704700BF838A13F0020F03D1C3680B6086
:1059200001207047C36818680860003818BF01205C
:10593000704700BF30B583B00C4615460B8A13F094
:10594000010F05D113F0020F08D1012003B030BDC3
:105950008A682B6813442B600120F7E700EB4000B6
:10596000094B1B6801A903EBC000FFF7D3FF40B14F
:105970002A6801990A44A368D35813B15B1A2B60B3
:10598000E4E70020E2E700BF003F00302DE9F04FE0
:1059900089B08046059192461D46DDF848B09DF8D5
:1059A0004C9000242AE0B9F10B0F23D83846FFF7BA
:1059B0009DFF064600B3149B079307AA394650463D
:1059C000FFF7B8FFC0B14B46224659462846FFF7BD
:1059D0004FFF079B029309F10603DBB2019300908E
:1059E0003346524605994046FFF7D0FF20B109B033
:1059F000BDE8F08F0020FAE70134E4B204EB840341
:105A000005EB830715F8236036B3062ECBD04B4643
:105A1000224659462846FFF72BFFC8F39133984298
:105A2000EAD1C8F30423B342E6D10AEB4A03DE000D
:105A30000A4A106807A900EBC300FFF76BFF0028B4
:105A4000DAD0BB68079A1344149A1344059A13607A
:105A5000024B18683044CAE70020C8E7003F003016
:105A60002DE9F04F8DB007460E46934608939DF8FA
:105A700058A0DDF85C80DDF8689002EB4203DA00A4
:105A800009924C4A10680BA900EBC300FFF742FFD4
:105A9000002800F087800024CDF85C80B846179F6E
:105AA0003DE02846FFF722FF0790002835D0BAF1E5
:105AB0000B0F61D80A970AAA29465846FFF73AFF02
:105AC00058B399F80030012B58D85A1C89F8002097
:105AD00009EB83035D605346224608993046FFF781
:105AE000C7FE03461B9A0592CDF81090199A0392AF
:105AF000189A02920A9A01920AF10602D2B2009210
:105B00005A4607994046FFF7ABFF034600284CD1A1
:105B100099F80030013B89F800300134E4B204EB1D
:105B2000840306EB830516F82320002A3CD0AB68DB
:105B30003B44062AB5D00B990B44434520D0052A97
:105B4000EBD11A1D904503D003F108029045E4D132
:105B50004746FB1A9B081B9A137053462246089926
:105B60003046FFF785FE189B1860199B1D60114B8E
:105B70001B68099A134418E0002316E0002314E080
:105B80005346224608993046FFF772FE189B18606C
:105B9000199B1D6000231B9A1370064B1B68099A02
:105BA000134402E0002300E0002318460DB0BDE8D6
:105BB000F08F00BF003F00302DE9F04F89B005465F
:105BC0000F4616469846DDF848900024146015E00C
:105BD0005046FFF795FE014670B1CDF81490CDF810
:105BE00010800396029700230193009322462846D3
:105BF000FFF736FF824688BB0134A4B2194B1B88DD
:105C0000A34229D904EB440C174B1B6803EBCC0AC5
:105C100013F83CB007A95046FFF77CFE0028EBD0F4
:105C2000BBF1060FD4D0079BAB4210D0BBF1050FE0
:105C3000E2D11A1D954203D003F108029542DBD14F
:105C4000EB1A9B0889F8003000233B6006E0002334
:105C50003B6089F8003001E04FF0000A504609B07F
:105C6000BDE8F08FFC3E0030003F00302DE9F043EE
:105C700089B00646174698460C88C4F3080404EB1E
:105C80004400254B196801EBC00511F8309007A9B5
:105C90002846FFF73FFE002839D00023C8F800301F
:105CA000B9F1060F0ED00798B04224D0B9F1050F14
:105CB0002FD1031D9E4223D000F108039E421FD026
:105CC000002514E02846FFF71BFE054678B1119B1E
:105CD0000593109B0493CDF80C8002970023019349
:105CE0000093224601463046FFF7BAFE0546284695
:105CF00009B0BDE8F08300233B60119A1370F6E70A
:105D0000361AB608119B1E7000233B60EFE7002592
:105D1000EDE70025EBE700BF003F0030431E042BFA
:105D200004D8DFE803F008080508070000207047E2
:105D3000042070470C2070472DE9F04F83B0804657
:105D40008A4691469B4600242746254635E0C3F106
:105D5000200CA3F1200127FA03F205FA0CFC42EA19
:105D60000C0225FA01F10A4312F0010F59D1012169
:105D7000A3F12002C3F1200C01FA02F221FA0CFC7B
:105D800042EA0C0201FA03F31F431543062829D007
:105D9000FFF7C4FF0190002847D07068FBF7F8F9BF
:105DA0005844102843D8BAF80030019A1A441346D0
:105DB0000433AAF800300134E4B204EB840308EBA6
:105DC000830618F8230040B373783F2B27D8B9F126
:105DD000000218BF0122002B18BF0022002AB6D0F3
:105DE0003F23B4E7B9F10B0F1DD83046FFF77EFD16
:105DF00001900028DFD07068FBF7CAF90BEB0003B5
:105E000009F10602DBB2D2B251460198FFF794FFC6
:105E10000028D0D103B0BDE8F08F0120FAE70020C0
:105E2000F8E70020F6E70020F4E70020F2E7002082
:105E3000F0E700BF2DE9F04182B00423ADF8063051
:105E4000002419E024B90023184602B0BDE8F0810F
:105E50003046FFF755FD804660B17068FBF798F952
:105E6000C3B200220DF106014046FFF765FF03466D
:105E7000E0B9E9E70134A4B2164B1B88A34222D94A
:105E800004EB4403144A126802EBC30612F83350C1
:105E90003789062DD6D02846FFF740FF0346A0B12C
:105EA000BDF8062013440433ADF8063039462046C9
:105EB000FFF702FD034650B9062DDBD0B28A12F07F
:105EC000020FD7D0C0E70123BEE70023BCE70023C1
:105ED000BAE700BFFC3E0030003F00304378C3F318
:105EE0004013007840EA0320704700BF2DE9F041DD
:105EF00088B005900E46002416E02846FFF700FD06
:105F0000034678B100220292019200922246314665
:105F10000598FFF73BFD0546284608B0BDE8F0812F
:105F20000025F9E70134A4B2124B1B88A3421FD904
:105F300004EB4403104A126802EBC30512F83380E5
:105F40002F8905A8FFF7CAFFB842EBD1B8F1060FB9
:105F5000D3D09DF8153003F01F034345E2D107A9C4
:105F60002846FFF7D7FC0028DAD0079B3360D3E739
:105F70000025D1E7FC3E0030003F00300170C1F346
:105F80000021437861F345134370704710B582B028
:105F900004469DF8053043F01F038DF8053040F2AC
:105FA000FF1101A8FFF7EAFF019BFF2262F39F3375
:105FB0000193042221460DEB0200FFF745FC024B42
:105FC0001C8002B010BD00BFEC3E003000B583B0B5
:105FD00050238DF8043041238DF8053006238DF8C9
:105FE000063000218DF8071004220DEB0200FFF7A8
:105FF0002BFC0420FFF7CAFF03B05DF804FB00BFD1
:1060000010B582B0002401940094042322460DEBC5
:1060100003011D4801F03AFA0423224669461B4851
:1060200001F034FA9DF80430502B10D09DF8003068
:10603000502B03D19DF80130412B11D0FFF7C6FF43
:106040001149124801F0B6FA012002B010BD9DF8C6
:106050000530412BEAD19DF80630062BE6D1EFE75B
:106060009DF80230062BE9D10849074801F0A2FA51
:106070000028E3D005F01AFF4FF4B3724FF08051BF
:1060800005F0FEFEE0E700BFF83E0030E03E0030E5
:10609000437803F01F031F2B0ED010B50446FFF703
:1060A0001DFF40F2FF13984208D02368013B13F113
:1060B000030F05D8002010BD012070470120FAE72A
:1060C0000120F8E7F0B583B005460E4604240CE045
:1060D00001A8FFF7DDFF68BB9DF8050000F01F0079
:1060E000FFF71CFE021D224494B2184B5B889C42B1
:1060F00025D2042322460DEB0301144801F0C6F912
:106100009DF805306A78534013F01F0FE0D101A8C5
:10611000FFF7E4FE07462846FFF7E0FE8742D7D1A7
:106120002A68019B5A400A4B1340002BD0D134807F
:10613000012008E03480074B1C80002003E04FF66C
:10614000FF733380002003B0F0BD00BFF83E003085
:1061500000C0FFFFEC3E003070B50D4614461E46F1
:10616000114628461AF0F0FF821CA2420AD85F238B
:106170002B54411C06F158036B540330A04201D844
:106180000023AB5470BD00BF2DE9F04F83B00190E8
:10619000894690461E469DF830B00D9F0E9D9DF895
:1061A0003CA02A46496838461AF0BAFF002401E0AC
:1061B0000134E4B23378A3420FD9294638461AF0A5
:1061C000C3FFC0B28542F3D906EB84035B682A1A89
:1061D000596838441AF0A4FFEAE7B8F1000F22D05A
:1061E000294638461AF0B0FFC0B285420DD8BBF13F
:1061F000000F0CBF53464AF001031BB198F8003062
:10620000052B09D003B0BDE8F08F2A1AD8F8041086
:1062100038441AF085FFEAE75B462A46394601987A
:10622000FFF79AFFEEE7BBF1000F0CBF53464AF0B1
:106230000103002BE6D099F80030052BE2D15B4634
:106240002A4639460198FFF787FFDBE72DE9F04141
:106250008AB0074690461E4605AC00250595069572
:1062600007950DF113050195009408AB09AAFFF7F6
:10627000FDFC88B101469DF8403003930296CDF8AD
:1062800004809DF81330009305AB089A3846FFF759
:106290007BFF0AB0BDE8F081002388F80030F8E702
:1062A0002DE9F04F85B080468A4693461F4600246C
:1062B00025E075682846FAF76BFF024629464046F6
:1062C0001AF0F8FEC8B93046FFF710FB0546A0B13A
:1062D000CDF80CB003AA31465046FFF72BFB60B156
:1062E0007068FAF755FF0E9B00932B46039A5146B0
:1062F0004044FFF7D5FF002857D10134E4B204EB46
:10630000840307EB830617F82350002D54D0062D85
:10631000CFD0D6F80490494640461AF0B1FE98B363
:10632000052DEAD1102148461AF00EFFC5B22A46C3
:10633000494640461AF0E0FE0028DED118F9053043
:106340005F2BDAD1013518F90530583BDBB2022B4F
:10635000D3D80AEB4A03194A106803A900EBC3001B
:10636000FFF7D8FA0028C8D0B068039B18445844F7
:1063700004230E9A137018F90530592B18D05A2B94
:1063800018D0582BB9D110E00AEB4A030B4A106819
:1063900003A900EBC300FFF7BDFA0028ADD00E9BA8
:1063A0001D70B068039B1844584405B0BDE8F08FD9
:1063B0000430FAE70830F8E70020F6E7003F003045
:1063C0002DE9F04788B007468846914600241CE036
:1063D000D6F804A0102150461AF0B6FEC5B22A46DF
:1063E000514638461AF088FE68B93046FFF788FAF9
:1063F000034640B1CDF80080002221467819FFF70E
:106400004FFF0546F0B90134A4B21D4B1B88A342CF
:1064100030D904EB44031B4A156805EBC30615F895
:106420003350062DD4D0716838461AF029FE002862
:10643000E9D188F8005005A93046FFF76BFAB8B1EA
:10644000059D18E0B9F1000F15D0002303930593C3
:10645000069307930DF10B03009305AB04AA03A960
:10646000FFF7AAFB049B33B11B8AA9F8003002E0B6
:10647000002500E00025284608B0BDE8F08700BFF1
:10648000FC3E0030003F003010B58EB004460023C3
:106490000D9309930A930B930DF12303009309AB1A
:1064A0000CAA0DA9FFF788FB70B1014601230393E5
:1064B0001123029304AB01939DF82330009309ABA1
:1064C0000C9A2046FFF760FE0EB010BD70B586B086
:1064D00004460D4604908DF814102B4E4FF4CE72E6
:1064E000311D01A8FDF7E4FE052202A930680DF078
:1064F0000BFB052814BF0026012601A8FDF7FAFEB4
:106500000EB3029BA3421ED19DF80C30AB421AD1B0
:1065100037E0052204A920680DF07CFA052814BF95
:10652000002401241CE0206D03681B6901219847A9
:10653000206D03689B684FF4FA719847206D0368DB
:106540001B6900219847104C40F25712211D01A8E9
:10655000FDF7AEFE20680DF0E1F90428D9D800243B
:1065600001A8FDF7C7FE64B9084B1C68636D93F87A
:106570009C30002BD7D0206D03681B6C98470028F7
:10658000D1D006B070BD00BFC43E00302C2A003010
:1065900030B583B0C8235D1EADB223B3134C4FF4A6
:1065A000A172211D01A8FDF783FE20680DF08EF970
:1065B0000F4CA4FB0034A40801A8FDF79BFE94B186
:1065C0000C4B1C68206D03681B690A219847206DDD
:1065D00003685B680A219847206D03681B690021E6
:1065E00098472B46D7E703B030BD00BFC43E00300C
:1065F000CDCCCCCC2C2A003000B58BB00023099335
:106600000593069307930DF11303009305AB08AAB6
:1066100009A9FFF7D1FA58B30246089B03B31978CA
:106620009DF80D3061F304038DF80D30118903A836
:10663000FFF7A4FC039B099A62F39F3303930DF1C8
:106640000A0103A8FFF73EFDA0B19DF80D3003F04D
:106650001F03052B0FD09DF8133063B100200AE013
:1066600001789DF80D3061F304038DF80D30DDE7FE
:10667000002000E000200BB05DF804FB184B1B88E5
:106680000BB90020704770B588B005460E46002350
:1066900007930393049305930DF10B03009303AB4E
:1066A00006AA07A9FFF788FAA8B100230C4A1288A6
:1066B0009A4212D903EB43020A490C6804EB8201A7
:1066C00054F82220AA4202D001339BB2EEE70B7AA3
:1066D0003370012002E0002000E0002008B070BD0F
:1066E000F43E0030E83E003010B582B004460DF1B3
:1066F0000701FFF7C3FF08B102B010BD2046FFF746
:106700007BFFF9E70138032816D8DFE800F002081C
:106710000E13FDEEC07A17EE903A0B707047BDEE87
:10672000C00A10EE103A0B807047BDEEC00A81ED32
:10673000000A704781ED000A704700BF03886FF3BD
:106740000803038003686FF35E33036043786FF3DD
:10675000440343700B4B1B8883B100B583B019B160
:10676000094B1B681B780B7001A9074B1868FFF7D2
:10677000D1F828B1019803B05DF804FB0020704700
:106780000020F8E7FC3E0030003F00302DE9F04FDC
:106790008BB081460D46924606939DF850B0DDF8C9
:1067A00058809DF860300793002434E03846FFF7A6
:1067B0009DF8064668B3159B099309AA39464846D1
:1067C000FFF7B8F828B35B46224606992846FFF73C
:1067D0004FF80346079A0492179A0392CDF808805F
:1067E000099A01920BF10602D2B20092524631464A
:1067F0004846FFF7CBFF60B1A2E05B462246069910
:106800002846FFF735F8D8F80030C3F351339842E3
:1068100059D00134E4B204EB840305EB830715F887
:106820002360002E00F08B80388AFFF733F80028B1
:10683000EFD0062EBAD09AF80030002BDDD0B8F891
:10684000003069F30803A8F800305B462246069939
:106850002846FFF70DF8D8F8003060F35E33C8F82B
:10686000003098F801306FF3440388F80130179B2B
:1068700003B11E7009EB4903334A106809A900EB04
:10688000C300FFF747F80028C3D0BB68099A134438
:10689000159A9818079A002A52D02C4A1278002A82
:1068A0004ED03A78012A4BD13A8A12F0040F47D0E1
:1068B000159A9B56002B43D198F8033043F0800380
:1068C00088F803303CE001238AF8003098F903305F
:1068D000002B2CDB052E9CD198F80130C3F3430329
:1068E000022B96D8013398F8012063F3440288F80C
:1068F0000120179B13B10423179A137009EB490366
:10690000114A106809A900EBC300FFF703F800283B
:106910003FF47FAFB868099B1844159B184498F85A
:106920000130C3F34303013B00EB830008E098F818
:1069300003306FF3C71388F80330002000E0002015
:106940000BB0BDE8F08F00BF003F0030E025003005
:106950002DE9F04788B091460388C3F3080300226D
:106960008DF81F203C4A12889A426ED90746884605
:106970001C4603EB4302D0003849096811F8322065
:10698000052A06D0062A34D05C1C01238DF81F305E
:106990002FE07978C1F343010229F3D801317B78E4
:1069A00061F344037B70B8F1000F02D0042388F830
:1069B00000307B78C3F343035A1E284B1B681844EE
:1069C000C36803EB820343E03A8864F308023A8029
:1069D0003A686FF35E323A607A786FF344027A7005
:1069E000B8F1000F01D088F80030EB6830E00134D6
:1069F000A4B2194B1B88A34229D904EB44034FEAE4
:106A0000C30A164A166806EBC305A88AFEF742FFBA
:106A10000028ECD016F80A30062BD5D12846FEF710
:106A20006FFF01460028E2D0CDF81090CDF80C8021
:106A300002970023019300930DF11F022046FFF7F8
:106A4000A5FE03460028D2D002E0002300E0002388
:106A5000184608B0BDE8F087FC3E0030003F00302B
:106A600030B583B004460D4601220DF107012046E2
:106A7000FFF76EFF024618B19DF80730042BF3D8DC
:106A80001AB115B19DF807302B70104603B030BD18
:106A9000F8B506460F4615461046FFF74FFE002490
:106AA00005E00134A4B239462846FFF7D9FFB442C5
:106AB00034BF0023012308B1002BF2D0F8BD00BF82
:106AC0000139032919D8DFE801F00209101590F9FE
:106AD000003000EE103AB8EEC00A7047B0F900304E
:106AE00000EE103AB8EEC00A704790ED000AB8EE1A
:106AF000C00A704790ED000A70479FED010A704789
:106B00000000C07FB4EE400AF1EE10FA62D610B574
:106B10000446F0EEC07A9FED307AF4EE477AF1EE5B
:106B200010FA20DC04291CD003291DD0022934D0FE
:106B3000012918D1B5EEC00AF1EE10FA47D4DFED05
:106B4000277A40F60A009FED261ADFED260A37EE77
:106B5000800AFEF7DDF9FDEEC07A17EE903A237059
:106B600001E080ED000A10BDB5EEC00AF1EE10FAAA
:106B700010D4DFED1A7A4FF400609FED1B1ADFEDA1
:106B80001B0A37EE800AFEF7C3F9BDEEC00A84ED9A
:106B9000000AE8E7DFED167AEDE7B5EEC00AF1EEA0
:106BA00010FA11D4DFED0D7A40F605009FED111AB1
:106BB000DFED110A37EE800AFEF7AAF9BDEEC00A32
:106BC00010EE103A2380CEE7DFED097AECE7DFED37
:106BD000087AB6E7704700BFFFFF7F7F0AD7233CE4
:106BE0000000FE42000000C30000004F000000CF84
:106BF0000AD723BC00FEFF46000000C790F900C082
:106C0000BCF1230F30D0F0B583B00E4615461C46BC
:106C10000023019301AA17491BF0DEF8074628B3A9
:106C2000FAF7B6FA102802D9002003B0F0BD01AA85
:106C3000104900201BF0D0F8D0B100211BF060F803
:106C400085ED000A376001AA0A4900201BF0C4F84C
:106C500030B10949FAF792FA10B901202070E4E73F
:106C6000002323700120E0E7002070470020DCE7CC
:106C70000020DAE7644606086C460608F0B59DB0C9
:106C80000746214D6E8AB6B200230380143528E0F2
:106C9000944235D02246294603A819F0BFFE1CAB0A
:106CA0002344002203F8642C361B013EB6B20134A3
:106CB00025449DF90C30934218BF232B11D00DF1C0
:106CC000020302AA01A903A8FFF798FF48B1002216
:106CD0000DF103010198FFF773FB10B13B880133FD
:106CE0003B806EB13246632E28BF6322002494425B
:106CF000CED22B5D5BB20A2BCAD00134A4B2F6E728
:106D000001201DB0F0BD00BFB0460608F0B59FB031
:106D1000424B186808B1FDF743F900233F4A13605E
:106D20003F4A13803F4A1380ADF876300DF176006C
:106D3000FFF7A4FF08B91FB0F0BDBDF8760000EB67
:106D400040008000FDF724F9344B186028B1364D1F
:106D50006E8AB6B20027143541E034480CF07CFA54
:106D6000944257D02246294604A819F057FE1EAB7C
:106D70002344002203F8682C361B013EB6B20134CE
:106D800025449DF91030934218BF232B27D00DF1D5
:106D9000060303AA02A904A8FFF730FFF8B10022F6
:106DA0000DF107010298FFF70BFB0446B8B107EBA2
:106DB00047039A00194B196888501B681344039ABB
:106DC0005A609DF806201A721AB1164A13880133C8
:106DD00013800137BFB22046FFF70EFC90B1BDF81B
:106DE0007610B94216D9AEB13246632E28BF63225F
:106DF00000249442B4D22B5D5BB20A2BB0D0013494
:106E0000A4B2F6E79DF807109DED030A2046FFF7B0
:106E100079FEE4E7024B19808DE700BFE83E0030C1
:106E2000F43E0030E63E0030B046060878460608DC
:106E300008B5044B5B8A9BB203B908BDFFF766FF38
:106E4000FBE700BFB046060830B585B00020FFF76D
:106E5000EFFF264B1B788BB9244B01221A70244B71
:106E60001B681C6D23689D6A224A02AB92E80300EE
:106E700083E8030093E806002046A84704240BE0BB
:106E80001D4A14802EE09DF8050000F01F00FEF75B
:106E900045FF021D224494B2184B5B889C4220D2CD
:106EA000042322460DEB0301144800F0EFFA01A879
:106EB000FFF7EEF803460028E2D169460198FFF794
:106EC00015F80028DFD09DF8050000F01F00FEF740
:106ED00025FF0346221D92B20099084800F0D6FA19
:106EE000D1E70023184605B030BD00BFF63E0030A4
:106EF0002C2A0030A03C0608EC3E0030F83E003062
:106F00000023104A12889A4218D910B403EB4302A6
:106F10000D4C246804EB820C54F82220824208D0E5
:106F200001339BB2074A12889A42EFD891ED000ACA
:106F300001E09CED010A5DF8044B704791ED000AF9
:106F4000704700BFF43E0030E83E0030F0B58DB031
:106F5000044600230B930793089309930DF11B0339
:106F6000009307AB0AAA0BA9FEF726FE00287AD0E9
:106F700005460A9B002B37D01A789DF8153062F32E
:106F800004038DF81530298905A8FEF7F7FF059B46
:106F90000B9A62F39F3305930DF1120105A8FFF7D9
:106FA00091F8064640B39DF8153003F01F03052BFA
:106FB00003D09DF81B30002B57D19DF81B300BB12F
:106FC000A4EB83049DF8150000F01F00FEF7A6FE59
:106FD0000346BDF81220043292B22146244800F044
:106FE00055FA30460DB0F0BD02789DF8153062F3C9
:106FF00004038DF81530C6E703A92846FEF78AFC7E
:107000000028EED00A9901B300231A4608E00CA824
:1070100000EB830050F8100C806802440133DBB2AF
:107020009DF81C009842F2D89DF8157007F01F07D4
:107030008D68039B1D4415440C312046FFF760FF0B
:1070400029463846FFF75EFBCBE79DF8157007F041
:107050001F0705F110012046FFF752FF039938463C
:10706000FFF750FBBDE70026BBE70026B9E700BFEE
:10707000F83E00302DE9F04180460E46002401E044
:107080000134E4B204EB840306EB830116F82350C9
:1070900065B1042DF4D88F6847440C313846FFF7AA
:1070A0002FFF39462846FFF72DFBE9E7BDE8F081C1
:1070B000F0B583B0FEF7A4FF002401E00134A4B2D0
:1070C000104B1B88A3421AD904EB44030E4A1268E2
:1070D00002EBC30612F83350042DEFD801A9304655
:1070E000FEF718FC0028E9D0019F06F11001384690
:1070F000FFF706FF39462846FFF704FBDEE703B03B
:10710000F0BD00BFFC3E0030003F003070B582B0E3
:107110004FF419621C4901A8FDF7CAF81B4B1C88E3
:107120003CB11B4B1A881B4B1B889A4225D0042369
:1071300006E0042304E0154B1C80164B1E802B46F2
:10714000124A14882CB1124A1188124A12889142AC
:1071500013D05D1EEDB283B1002400940C4B1E8849
:1071600021466846FFF7EAFA0028E4D00134A4B2C9
:1071700000216846FFF774FCF6E701A8FDF7BAF8AE
:10718000204602B070BD00BFA83E0030EE3E003089
:10719000E43E0030F23E0030024A1388013313808F
:1071A000704700BFE43E0030F0B52DED028B93B088
:1071B00004460D46002311930D930E930F930DF18A
:1071C000330300930DAB10AA11A9FEF7F5FC0028BC
:1071D00000F091800646109BFBB11A789DF82D3087
:1071E00062F304038DF82D3031890BA8FEF7C6FE3B
:1071F0000B9B119A62F39F330B939DF82D3003F094
:107200001F03052B03D09DF83320002A73D19DF86E
:10721000337057B1A4EB870708E002789DF82D3052
:1072200062F304038DF82D30DEE72746012B66D08C
:10723000012303931123029306AB01939DF833308E
:1072400000930DAB109A31462046FEF79DFF0DF1DD
:1072500016010BA8FEF736FF00285AD1BDF81620FC
:107260004FF6FF739A4246D09DF82D1001F01F0192
:1072700004292BD82046FFF723FCB0EE408A109952
:10728000002955D00C312046FFF73AFEF0EE408A37
:10729000F0EE680AB0EE480AFDF70AFE00B155B3F9
:1072A000A5B99DF82D3003F01F03032B0ED078EE07
:1072B000688AF0EEE88AB0EEC88ADFED2F7A28EE11
:1072C000278AF4EEC88AF1EE10FA14D4BDF81640FD
:1072D0009DF82D0000F01F00FEF720FD2318083355
:1072E000264A528893422BD3254B1B68186C03689F
:1072F0001B682449984713B0BDEC028BF0BD109B6E
:10730000002B95D01B8A13F0040F91D0FFF744FF98
:107310008EE79DF82D0000F01F00FEF7FFFC0246EF
:10732000BDF81610043189B23846FEF78DFAE2E74F
:1073300006F110012046FFF7E3FDF0EE408AA7E7D3
:1073400014FA80F080B2043080B2FEF71FFE9DF880
:107350002D0000F01F00FEF7E1FC0246BDF81610FC
:10736000043189B23846FEF76FFA0422BDF81610D0
:107370000BA8FEF769FABEE717B7D138F83E003020
:107380002C2A0030A046060810B584B012E0052271
:1073900002A920680CF0D8FB052814BF00240124A2
:1073A00001A8FCF7A7FF9CB101229DF80C100298E0
:1073B000FFF7FAFE0C4C4FF4BB72211D01A8FCF73D
:1073C00077FF20680CF082FA0428E0D80024E7E771
:1073D000064B1B68186D03685B6B984708B904B0CF
:1073E00010BDFFF793FEFAE7C43E00302C2A0030B0
:1073F00008B5FFF7C9FF08BD10B50446034B03608D
:10740000034B0360FCF7BEFD204610BD78830608E1
:10741000D43E060808B54FF6FF710120FEF7D6F9F5
:1074200008BD00BF08B5064B1B68D86B03685B68D6
:10743000984700B108BD034808F0F6FEFAE700BF20
:107440002C2A0030C4660608017000234380112BEB
:1074500018D810B403E00133DBB2112B0FD803EBC3
:107460004302094C14F812208A42F4D103EB430280
:1074700004EB42029288448822444280EBE75DF8A4
:10748000044B7047704700BFE46606082DE9F843D7
:1074900006460F461D46002416E0A2EB0E0E1FFA0C
:1074A0008EF20FE01C4B1B68D86B0368D3F8089072
:1074B0000A44434692B23946C847B5EB080525D081
:1074C000474400220134E4B2112C1FD8134B04EBC3
:1074D000440C03EB4C0CBCF804E0BCF8021004EBC9
:1074E000440013F8100033789842EBD17245D4D29F
:1074F0005FFA85F808EB02037345D3DD5FFA8EFE71
:10750000D3B2AEEB030E5FFA8EF8CBE7B5FA85F097
:107510004009BDE8F88300BF2C2A0030E466060865
:107520002DE9F843064617461D46002416E0A1EB58
:107530000E0E1FFA8EF10FE01C4B1B68D86B036810
:10754000D3F80C90114443463A4689B2C847B5EB8C
:10755000080525D0474400210134E4B2112C1FD87E
:10756000134B04EB440C03EB4C0CBCF804E0BCF8EC
:10757000022004EB440013F8100033789842EBD15A
:107580007145D4D25FFA85F808EB01037345D3DD6A
:107590005FFA8EFECBB2AEEB030E5FFA8EF8CBE74E
:1075A000B5FA85F04009BDE8F88300BF2C2A003009
:1075B000E46606082DE9F0418AB080460F464B8804
:1075C000ADF824304288ADF826209A4203D909ABA1
:1075D0001C88002506E00DF12603F9E7A41BA4B2E0
:1075E0003544ADB2B4B12646202C28BF2026334600
:1075F0002A4601A93846FFF749FF38B1334601AAA8
:1076000029464046FFF78CFF0028E7D100200AB04A
:10761000BDE8F0810120FAE770B504460023002B95
:1076200001DB013BFBE7002300E0013B002BFCDA20
:10763000002300E0013B002BFCDA04F114030022DC
:10764000002A06DB00211960596099600C33013A69
:10765000F6E7002300E0013B002BFCDA002300E00A
:10766000013B002BFCDA4FF0FF33E36204F1300002
:1076700008F058FD04F158050026002E0ADB05F13C
:107680000C000BF0A7FE00236B63AB63EB63A83524
:10769000013EF2E70023C4F85031C4F85431C4F875
:1076A000583107492046FFF7E5FC064B1B681BB91C
:1076B000044B1C60204670BD03480BF0CDFD00BF9D
:1076C00060680608043F00305067060817290FD885
:1076D000DFE801F00C0E0E0E0E0E0E0C0E0C0E0E50
:1076E0000E0E0C0E0E0E0E0C0E0C0C0C0020704725
:1076F00001207047F8B52DED028B05460F4690F935
:107700000230032B02D00024264637E000F12A0481
:107710002046FEF7E9FF0028F5D195F92A30013B14
:1077200007EE903AF8EEE77AF0EEE77A9FED368AC8
:10773000F4EEC87AF1EE10FA4FF0010385F82A3022
:107740004CBF194600212046FEF7C0FE95F90230D5
:1077500007EE903AF8EEE77AF0EEE77AF4EEC87AC0
:10776000F1EE10FA4FF00003AB704CBF0121194647
:10777000A81CFEF7ABFEC6E70134E4B29CB929575A
:10778000C9B22846FFF7A2FF0028F5D032460521EE
:10779000384603F0CDFF04F1400305EB8303586046
:1077A0000136F6B2E8E70024AC604FF4E170B3EEC6
:1077B0000E1AF1EE040A95ED090AFDF7A9FBB7EEE2
:1077C000007AC7EE007AC5ED597A3CB9A82202FBCF
:1077D000045282F85840631CDCB2F6E700237BB900
:1077E0001A4603F1080135F91110002901DDC829F5
:1077F00003DD0832C82125F812100133DBB2EEE7B1
:10780000BDEC028BF8BD00BF000000348446A82305
:1078100001FB03330344587800B97047A82303FBE6
:1078200001CCDCF898301360F7E700BF8446A8234A
:1078300001FB03330344987800B97047A82303FB86
:1078400001CCDCF89C301360F7E700BF8446A82326
:1078500001FB03330344D87800B97047A82303FB26
:1078600001CCDCF8A0301360F7E700BF054BA0FBAC
:107870000303401843F10001034BC01841F14901D3
:10788000704700BF00840C24B0F5F790F8B50446AB
:107890000D46A82303FB0103D3F8B0304BB9A8234E
:1078A00003FB0103D3F8B800D3F8BC1050EA01037E
:1078B0003AD0A82303FB0543B3F86060002E61D0E3
:1078C000A82303FB0543D3F8B820D3F8BC301343F7
:1078D00034D005F1400354F823108F6C2FBB896B13
:1078E0003046FFF7C3FF4A0142EAD06243011B1A48
:1078F00062EB0102920042EA93729B001B1841EB7B
:107900000201CF0047EA5377DE000BF0DDFCA8232D
:1079100003FB0545D5F8B830D5F8BC20C01A61EB9B
:107920000201301841EB0701F8BD4FF47A720023D1
:10793000D1E91001F8F75AFE3918D1E7A82101FB67
:107940000545E96D3046FFF791FF06460C460BF002
:10795000B7FCD5F8B020821A911944F10003580100
:1079600040EAD1604A01521A60EB0300800040EA0D
:1079700092709200521843EB0001C900D00041EA16
:107980005271D1E700200146CEE700BF38B5A823E9
:1079900003FB0103B3F8605025B3403150F82110C8
:1079A0008C6CB4B9896B2846FFF760FF4A0142EA44
:1079B000D06243011B1A62EB0102920042EA937209
:1079C0009B001B1841EB0201C900D80041EA53712A
:1079D00038BD4FF47A720023D1E91001F8F706FEA2
:1079E0002118E0E700200146F2E700BF283100EB54
:1079F000C10042600381704708B54356022B03D192
:107A0000038D13F0040F04D12E23044AFFF7EEFF79
:107A100008BD2E23024AFFF7E9FFF9E730680608A0
:107A20008C69060870B5044601F1400300EB83033E
:107A3000586800B30D4601F1280304EBC3031B890A
:107A4000CBB103681B6A984705F1280604EBC6060C
:107A50003289824228BF0246403504EB85046068C3
:107A60000368DB6892B27168984773680344736077
:107A70003389181A308170BD2DE9F04383B0054673
:107A80000C460BF01DFCA82303FB0453002283F8D3
:107A900059204FF6FF72A3F88620A3F888202B57B1
:107AA000092B00F06581074605DBA3F11602D2B26F
:107AB000012A40F25D8104F1400205EB8202526826
:107AC000002A00F05581C4EBC40205EBC20201217B
:107AD00082F811110B2B5AD00F2B6BD00A2B43D0ED
:107AE0000026C4EBC40305EBC303D3F80C31FB1A27
:107AF000B3F5966F2BD9C4EBC40205EBC20292F822
:107B000010310133DBB282F81031082B65D0C4EBA1
:107B1000C40805EBC80898F8101104F1400905EBFA
:107B20008909D9F8040003685B6A934A52F8211066
:107B30009847D9F804000368DB6D00219847C8F81E
:107B40000C7195F91330002B01DD002E4AD095F908
:107B50001330002B40F39E80002E40F09B80214686
:107B60002846FFF75FFF95E04FF4CC70FCF702FA70
:107B70000646A82204FB02F2583204F1400305EB4A
:107B800083035B682A44294601F0D6F9A9E74FF43C
:107B9000BC70FCF7EFF90646A82204FB02F258324B
:107BA00004F1400305EB83035B682A44294600F097
:107BB000F1FB96E74FF4C870FCF7DCF90646A82203
:107BC00004FB02F2583204F1400305EB83035B68C7
:107BD0002A44294600F0A6FE83E71346002283F8D4
:107BE000102194E721462846FFF706FFAFE795F9F5
:107BF00013305BB9C4EBC40305EBC30393F8102146
:107C00005D4B53F82230B3F5164F12D2C4EBC403C8
:107C100005EBC30393F81021574B53F82230B3F50B
:107C2000E13F03D32A8D12F0040F02D1B3F5613F77
:107C300052D1C4EBC400C00000F584702844414612
:107C40000A3002F0B1F8002846D04FF49B60FCF7F0
:107C500091F90646A82204FB02F2583204F14003CF
:107C600005EB8303002100915B682A44294603F059
:107C70008DF931E04FF4E12235E0C4EBC40305EBAC
:107C8000C30393F810113C4B53F82130934230D08A
:107C9000002E57D104F1280305EBC3031B89002BE9
:107CA00050D104F1400305EB8303586803681B6956
:107CB0009847002846D0002E44D104F1400305EB3C
:107CC0008303586803685B6998475FFA80F82B570D
:107CD000012B8CD0022B8AD0B5F9283013F0010F7C
:107CE000C8D04FF461322B57112BC6D0122BCFD1F5
:107CF000C3E7C4EBC400C00000F5847028444146CB
:107D00000A3002F051F80028C2D02B57112B16D0A0
:107D10004FF002084FF49B60FCF72CF90646A822AE
:107D200004FB02F2583204F1400305EB8303CDF863
:107D300000805B682A44294603F028F9A8E74FF041
:107D40000108E7E7A6B1A82303FB0453012283F847
:107D5000592004F1400345F8236005EB0413DF6468
:107D6000053424014FF47A632B53304603F01EFB95
:107D700003B0BDE8F08300BF10680608F8B54356AD
:107D8000072B68D004460D46002B59D090F80A31D5
:107D9000CB4013F0010F5ED101F1400350F82330C6
:107DA000002B59D090F91330002B58DC05F140031B
:107DB00054F8230003689B68984707460BF080FA45
:107DC0000646002F55D104EB0513DB6CC31AB3F53F
:107DD0007A6F40D9A82202FB05F707F1580000216D
:107DE000204418F029FEE31983F858504FF6FF722B
:107DF000A3F88620A3F8882004EB0513DE646B1D2E
:107E00001B014FF47A62E25263570E2B2AD0092BE2
:107E100028D0162B26D0172B24D005F1400354F878
:107E2000230010B103685B68984705F14003002206
:107E300044F82320A82303FB054383F859203FE09F
:107E4000A82101FB050484F859304FF6FF73A4F80C
:107E50008630A4F88830F8BDFFF70EFEFBE7FFF789
:107E6000E1FDA3E7A82303FB0543012283F8592082
:107E700026E0A82303FB054393F8C0306BB1A82785
:107E800007FB05474FF47A720023D7E92E01F8F774
:107E9000ADFB0646002387F8C03004EB0511CB6C20
:107EA000F21A6B1D1B01E252CE64A82303FB0543AB
:107EB00093F85930012B03D994F86A3103B98E64D1
:107EC0006B1D1B01E35AF52B26D96A1D04EB021228
:107ED000917801319170B3F5FA6FBCD26A1D04EB51
:107EE0000212D2ED017AF5EEC07AF1EE10FA19D94C
:107EF0009FED107A27EE877A07EE903AF8EEE77A50
:107F0000DFED0D6A67EEA67A77EE277A053504EB8A
:107F10000514C4ED017A9EE76A1D04EB02120021EC
:107F20009170D8E707EE903AF8EE677AC2ED017AE1
:107F300091E700BF48E17A3F0AD7A33C30B583B050
:107F4000054640F2064200F1300101A8FCF7B0F905
:107F5000002434B921462846FFF710FF0134E4B26B
:107F6000F7E7002301E00133DBB24BB903F1400234
:107F700055F82220002AF6D05A1C85F80921F2E78C
:107F800001A8FCF7B7F903B030BD00BF61B9944652
:107F90000A46403250F8220030B110B502685469E8
:107FA0001A466146A04710BD704700BFF8B50446A9
:107FB0000E46174690F906107F2910D1002501E0E2
:107FC0000135EDB285B96357122BF9D0172BF7D0D5
:107FD0003B46324629462046FFF7D8FFF0E71346D6
:107FE0003246C9B2FFF7D2FFF8BD00BF70B50546F3
:107FF0000E460024002C0FDC2B5743B104F1400344
:1080000055F8230028B103681B69984708B101346B
:10801000F0E73470012000E0002070BD2DE9F04150
:10802000044690461E4611F0010F43D00D46D0F88D
:108030004C31002B43D0C5F34107ED08D4F84C3147
:108040001A783AB15978A94243D000229A70D4F8EC
:108050004C311A70D4F84C315D70D4F84C110123B6
:1080600003FA07F20B7813430B70D4F84C01B423D6
:1080700003FB070032464146063018F0CFFCB32E12
:108080002CD8D4F84C317A1C9A70D4F84C3107EBC8
:108090004701C1EB011106EB81019980D4F84C1125
:1080A0008A782AB1087801239340013B984222D074
:1080B000BDE8F0811A464146FFF778FFF8E740F245
:1080C000D621012016F0A0FEC4F84C010028B2D140
:1080D000EEE7FA4012F0010FBCD0B6E7D4F84C310D
:1080E0001A780F2ADAD104229A70D4F84C314FF45E
:1080F00034729A80D2E78A8806312046FFF756FF0D
:10810000D4F84C2100239370D4F84C211370CFE79E
:108110001A4B136081BB8C4601F1100330F9133008
:10812000002B13DC10B501F1400350F823402CB1B3
:10813000A82303FB010393F85930BBB910F90C00D5
:1081400080B1012814BF0020012010BD07EE903A35
:10815000F8EEE77A9FED0A7A67EE877AC2ED007A49
:1081600001207047002313600120EEE723689B6A1B
:10817000114620469847E8E700207047CDCCCC3D1B
:108180006F12833A90F809318B420AD9083130F9DD
:108190001130002B07DD1846C72B00DDC82080B248
:1081A0007047C8207047C820704700BFC1BB08B5E2
:1081B0000A4690F92A3013F0FF0333D1C35613F067
:1081C000FF0F31D04356122B0BD0172B0CD0DFED05
:1081D0001A7A531D00EB03139B78012B07D900205B
:1081E00021E0DFED167AF4E7DFED147AF1E7531DB5
:1081F00000EB031393ED017AB4EEE77AF1EE10FA97
:1082000014D5A82303FB0203D3F8C430042B0FD8E2
:10821000403250F8220068B10368DB6A984702E0F8
:1082200000207047002008BD0020FCE70020FAE78E
:108230000020F8E70020F6E70000574300007543F0
:1082400038B590F90E3073B1054600246CB904F1CD
:10825000400355F8230018B103681B6B984730B1F1
:108260000134E4B2F2E7002000E0002038BD012034
:10827000FCE700BF51B908B50B46403350F8230066
:1082800030B103689B6C1146984708BD00207047C9
:108290000020FAE70120704700207047704700BFB8
:1082A000704700BF014B0B6001207047CDCC4C3EA6
:1082B000012070470120704701207047002070475F
:1082C000704700BF00207047704700BF062070470E
:1082D00000487047BC690608024A0260024A026010
:1082E000704700BFCC6906082C71060810B504461B
:1082F000034B0360034B0360FBF744FE204610BDB5
:10830000CC6906082C71060800B587B000220192DE
:10831000029203920492CDF813204FF0020E8DF8D2
:1083200004E064238DF806300D238DF807304FF0FC
:10833000030C8DF80BC001238DF80D308DF80FE084
:108340004FF0040E8DF810E04FF0070E8DF812E09C
:108350008DF816C08DF8111090F8661101EB030C22
:1083600080F866C18DF8081007E006A9194411F8D5
:10837000141C0A44D2B20133DBB2112BF5D98DF8AB
:10838000152040680368DB68132201A9984707B0ED
:108390005DF804FB10B5044602F068FF0F4B236044
:1083A000002184F86611C4F8681184F86C110C4B34
:1083B0001868C4F86D011B7984F8713184F85A107B
:1083C0002046FFF7A1FF03212046FFF79DFF0AF09B
:1083D00077FF6E30C4F86801204610BDCC690608EE
:1083E000A83C060810B586B00024009401940294BD
:1083F000039404948DF8144002238DF80030642314
:108400008DF802300F238DF803304FF0030C8DF8F8
:1084100007C001238DF809304FF0070E8DF80BE0EF
:108420004FF0060E8DF80CE04FF00A0E8DF80DE0BF
:108430008DF80F308DF811308DF814C08DF80E20A6
:1084400090F8662102EB030C80F866C18DF80420D9
:108450008DF81110224607E006A9194411F8181CDE
:108460000A44D2B20133DBB2132BF5D98DF81320B5
:1084700040680368DB6815226946984706B010BD5E
:1084800000B58C468B1893F907E0002000216EF3AD
:10849000070093F906E06EF30F2093F905E06EF301
:1084A000174093F904E06EF31F6093F903E06EF355
:1084B000070193F902E06EF30F2193F9013063F3A2
:1084C00017411CF9023063F31F6141EC100B5DF89A
:1084D00004FB00BF881890F903C000236CF3070366
:1084E00090F902C06CF30F2390F9010060F3174379
:1084F0008A5662F31F6300EE103A70478B1893F9A7
:1085000003C000206CF3070093F902C06CF30F2046
:1085100093F9013063F317408B5663F31F60704784
:108520008B1893F901304FF0000063F307008B566E
:1085300063F30F2080B2704790F85D30402B01D07C
:10854000002070472DE9F0472DED048B04460325EC
:10855000002744E004F15F09D4F80CA032464946F4
:108560002046FFF7CBFFCAF80400D4F80CA0AA1DE0
:1085700049462046FFF7D4FFAAF8080005F1080392
:10858000E268234493F85F3082F8323005F1090342
:10859000234493F85F300A35254495F85F2013F0A3
:1085A000010F16D0E3680321597012F0010F13D0A8
:1085B000E3680421597012F0020F0DD012F0040F7D
:1085C00003D0E36806225A7006E0E36805225A7079
:1085D00002E0E36801225A70013708EB060594F8BF
:1085E0005E30AB4240F2BA80631993F85F206B1C97
:1085F000234493F85F80AE1C012AABD0022A31D00D
:10860000082A67D0092A00F097800C2AE5D104F1E6
:108610005F09AA1D49462046FFF75CFFB0EE408A7D
:1086200005F10A0249462046FFF754FF38EE008A5A
:10863000E368B6EE000A28EE008A83ED118AD4F8CA
:108640000CA005F1120249462046FFF743FF8AEDD0
:10865000120AE268012382F85230E26882F853304D
:108660001F44BAE704F15F09324649462046FFF746
:1086700007FF9FED419B20EE090B9FED418B20EE04
:10868000080BE368BDEEC00B83ED050A05F10A0295
:1086900049462046FFF7F4FE20EE090B20EE080BBA
:1086A000E368BDEEC00B83ED060A05F112024946F0
:1086B0002046FFF7E5FE9FED347B20EE070BE368D5
:1086C000BDEEC00B83ED040AE5680AF0F9FDA8656C
:1086D000013782E7A31993F85F3013F0010F01D13E
:1086E00001377AE704F15F09D4F80CA0EA1C494687
:1086F0002046FFF7EFFE8AED070AEA1D49462046AD
:10870000FFF7E8FEE368DFED227A20EE270A83ED2B
:10871000080A204602F0C6FD05F10B024946204634
:10872000FFF7D8FEE368B1EE400A83ED0F0AE36875
:10873000012283F85020D3E7AA1D04F15F012046EF
:10874000FFF7C8FEDFED137A20EE270AE368BCEEE0
:10875000C00A10EE102ADA8501373EE7052F07D050
:10876000E36801225A700020BDEC048BBDE8F0875D
:108770000120F9E7AFF30080F8C1631ADCA54C4093
:1087800000000000D01263410000000000005940CA
:10879000E02E65420000C84208B590F85A30013B0F
:1087A000052B04D8DFE803F0111D29354C5A0229A6
:1087B0005BD180F85B10012380F85A300023A0F8C9
:1087C000623180F8643118460AE080F85C100223B8
:1087D00080F85A3090F86431194480F86411002010
:1087E00008BD80F85D10032380F85A3090F864319A
:1087F000194480F864110020F2E780F85E10042329
:1088000080F85A3090F86431194480F864110020DF
:10881000E6E7B0F86231C21882F85F1001339BB20C
:10882000A0F8623190F86421114480F8641190F846
:108830005E2093421BD3052380F85A300020CFE7F7
:1088400080F85F11062380F85A3090F864318B422B
:1088500001D00020C4E7FFF76FFEC1E780F8601188
:10886000002380F85A301846BAE70020B8E7002005
:10887000B6E700BF38B504460AF022FD94F86C3123
:10888000042B04D80546D4F86821824201D3002580
:1088900022E02344002293F86D112046FFF7A2FD49
:1088A00094F86C312344032293F86D112046FFF7AE
:1088B00099FD6E35C4F8685194F86C31013384F831
:1088C0006C31E4E7606803685B699847C1B2204691
:1088D000FFF762FF2843C5B2606803681B699847C9
:1088E0000028EFD1284638BD062070470048704761
:1088F0001C6A0608024A0260024A0260704700BF12
:10890000E06A06082C71060810B50446034B0360A4
:10891000034B0360FBF736FB204610BDE06A0608F8
:108920002C71060810B5044602F0A0FC114B236020
:10893000002384F860306366A36684F86C30AA2351
:1089400084F87131442384F87231122384F873312E
:10895000A36893F913305BB160680368DB680E228B
:108960000549984760680368DB68222203499847F5
:10897000204610BDE06A0608246A0608346A060824
:1089800070B50446B0F87551B0F8792190F874319B
:108990001A44D0F8811102F019FD2A2D1BD0632D45
:1089A00000F0C780AE2D00F0F88094F85A0010F067
:1089B000010000F00D8194F85A30C3F3400013F029
:1089C000020F00F00581E26DE3685B689A4200F0F7
:1089D00000810020FCE0E368B4F87F211A81E3689D
:1089E000D4F881215A60E6680AF06AFCB065D4F8D0
:1089F0007520D4F879309FED7E7B43EC162B26EE64
:108A0000076BE368BDEEC66B83ED056AD4F87D2085
:108A1000D4F8813043EC162B26EE077BE368BDEEDD
:108A2000C77B83ED067AD4F88520D4F889309FED92
:108A3000727B43EC162B26EE077BE368BDEEC77B0B
:108A400083ED047AE36894F8AE2083F83220D4F8FA
:108A5000953007EE903AD4F8993007EE103A77EE59
:108A6000877AE368B6EE007A67EE877AC3ED117A0B
:108A7000E368D4F89D209A64E268012382F85230BA
:108A8000E26882F85330D4F8A53007EE903A9FEDB3
:108A90005C7A67EE877AE368FCEEE77AC3ED1E7ACC
:108AA000E36894F8AE2083F87C20D4F86D30002B76
:108AB00035D1D4F87130103B352B2CD8DFE803F0DA
:108AC0001B1F1F2B1F2B2B2B2B2B2B2B2B2B2B2B2A
:108AD0002323232B2B2B2B2B2B2B2B2B2B2B2B2BFE
:108AE000272B272B2B2B2B2B2B2B2B2B2B2B2B2BDE
:108AF0002B2B2B2B1F1FE36803225A7012E0E36815
:108B000004225A700EE0E36805225A700AE0E36816
:108B100006225A7006E0E36801225A7002E0E36818
:108B200001225A7094F85A3043F0010384F85A3005
:108B300035E7D4F87D20D4F88130E16843EC172B79
:108B4000F7EEC77BC1ED077AD4F88520D4F88930D9
:108B5000E16843EC172BF7EEC77BC1ED087A20469E
:108B600002F0A0FBD4F88D20D4F8913043EC172B01
:108B7000F7EEC77BE368F1EE677AC3ED0F7AE3683F
:108B8000012283F85020D4F88131E36594F85A30FB
:108B900043F0020384F85A3004E7D4F8753007EE46
:108BA000103ADFED186A27EE267AE368BCEEC77A42
:108BB00017EE102ADA85D4F8793007EE903A67EE8E
:108BC000A67AE368FCEEE77A17EE902A1A86002070
:108BD00070BD94F85A306FF3000384F85A30DBB25A
:108BE0006FF3410384F85A30F2E700BFAFF300801F
:108BF00000000000D0126341000000000000594056
:108C000000007A440000C8420846082301E04008FA
:108C1000013B002B06DD10F0010FF8D0024A82EA7A
:108C20005000F5E7704700BF2083B8EDF8B5054662
:108C30001446184609E0070A14F8011B4140C9B25E
:108C40002846FFF7E1FF784031464E1E0029F2D159
:108C5000F8BD00BF38B5044690F86C30013B082BD6
:108C600006D8DFE803F0101B263149656C778200D7
:108C7000AA2902D1012380F86C30002084F88D01EC
:108C800084F88E011FE0442903D0002084F86C0092
:108C900019E0022380F86C30002014E0122903D080
:108CA000002084F86C000EE0032380F86C30002074
:108CB00009E080F87411042380F86C30002084F8F7
:108CC0008D3184F88E0138BDB0F88D311B2B03D95E
:108CD000002084F86C00F6E7C21882F871110133A5
:108CE0009AB2A0F88D3190F874319A425FD305237F
:108CF00080F86C300020E6E7B0F88D31FF2B03D907
:108D0000002084F86C00DEE790F87421981A204463
:108D100080F86D10013399B2A4F88D31B4F879312F
:108D20001A44914245DB062384F86C300020CAE7E0
:108D3000C0F86D11072380F86C300020C3E7D0F82D
:108D40006D3103EB0121C0F86D11082380F86C3000
:108D50000020B8E7D0F86D3103EB0141C0F86D1188
:108D6000092380F86C300020ADE7D0F86D5105EB99
:108D70000165C0F86D51002380F86C3000F271126B
:108D800090F87411FFF752FF034604F16D02B4F836
:108D900079112046FFF74AFF854204D0A36E0133C4
:108DA000A36600208FE72046FFF7EAFD8BE700204F
:108DB00089E7002087E700BF2DE9F041044683687A
:108DC00093F913300BB9002529E00AF079FA05462A
:108DD00094F86030052BF6D8154A52F82360636E7C
:108DE0008342F0D267683B68D3F80C803046F8F7CE
:108DF000CFF9024631463846C047C835656694F813
:108E00006030013384F86030DDE7606803685B69D7
:108E10009847C1B22046FFF71DFF2843C5B26068DE
:108E200003681B6998470028EFD12846BDE8F08108
:108E3000C06A06080620704700487047306B060875
:108E400001207047014B0B60012070470AD7A33DFA
:108E5000836F0B6001207047836893F90E30022BFB
:108E600008D0406F00F42070B0F5207F14BF0020C0
:108E700001207047436F03F42073B3F5207F08D0BF
:108E8000064B1B685B6D93F89C3023B990F87C000F
:108E90007047012070470020704700BF2C2A003027
:108EA000836893F9133033B1036E042B01D0002093
:108EB0007047012070470120704700BF836F13F493
:108EC000746F0CBF01200020704700BF10B504462E
:108ED000044B0360406E15F09DFF034B236020465A
:108EE00010BD00BF186E06082C71060810B50446A8
:108EF000FFF7ECFF2046FBF745F8204610BD00BF0A
:108F0000836893F9133013B1026E042A00D17047BD
:108F100000B583B0C3681978032301930423009339
:108F200090F85A3001310348FAF7EAFC03B05DF8D3
:108F300004FB00BF346B060810B5044602F096F936
:108F40000C4B23600C4BE3660023236784F87E30D0
:108F50000AF0B6F9A066E368012283F87D20A368D1
:108F6000B3F9283013F0020F02D0E36883F82C2005
:108F7000204610BD186E0608686B060870B584B0F0
:108F80000446B0F88430C3F30C0340F6BC7293423D
:108F900026D8B3F57A6F40F24982A3F6A1731B2B52
:108FA00000F24682DFE813F060014402440244020A
:108FB0004402440255004402440244024402440272
:108FC0004402700144024402440244024402440246
:108FD00044024402440244024402440244029E0108
:108FE00041F21472934232D1B0F88620D0F8881042
:108FF00002F0ECF9D4F890200192D4F89410029188
:10900000D4F89830039307EE901A07EE103AF4EE76
:10901000C77AF1EE10FA40F3588102ABD3ED007A33
:1090200007EE102AB4EEE77AF1EE10FA00DD01AB9C
:1090300093ED000ADFEDBF7AB4EEE70AF1EE10FA25
:1090400080F24581E368002083F85100F1E10020BF
:10905000EFE1B0F88C3099B24FF6FF72914205D033
:10906000C2681381C368D0F888205A60B4F886209B
:10907000D4F88810204602F0A9F9E5680AF020F932
:10908000A865D4F8AC30DFEDAC7A07EE103AB4EE58
:10909000E77AF1EE10FA55DCD4F89020D4F8943049
:1090A0009FED9E7B43EC162BB4EEC76BF1EE10FAEE
:1090B00034DD9FED9C5B43EC172B27EE057B9FED8A
:1090C0009B6B27EE067BE368BDEEC77B83ED057ADD
:1090D000D4F89820D4F89C3043EC172B27EE057B6E
:1090E00027EE067BE368BDEEC77B83ED067AD4F8F6
:1090F000A020D4F8A43043EC172BB7EEC77BD4F8EC
:10910000A83007EE903A77EE677A9FED8C7A67EE9B
:10911000877AE368FDEEE77AC3ED047A94F8CA3003
:10912000FF2B02D0E26882F8323094F88E3003F0E0
:109130000F03082B65D8DFE803F0616D7175797D49
:1091400081858900E2685363E368D4F8B0209A63AC
:10915000D4F8B430E26807EE903AF1EE677AC2EDE7
:109160000F7AE368012583F85050E66896ED0D0A02
:1091700020EE000AD6ED0E7A67EEA77A30EE270AC7
:10918000FBF7A6FE86ED070AE368D3ED0D0A93ED23
:109190000E0A17F097F9B7EEC00A9FED627B20EE3A
:1091A000070BE668B7EEC00BFBF7A0FE86ED080ADA
:1091B000B4F8CE30E26803EB8303AB409367B4F8B6
:1091C000DA3007EE103AB8EE477AE368DFED5C6A12
:1091D00027EE267A83ED117AB4F8DC3007EE903A68
:1091E000F8EE677AE36867EEA67AC3ED127AE36871
:1091F00083F85250E36883F853504DE7E368012247
:109200005A7094F88E3013F0400F23D0E368012099
:1092100058700EE1E36803225A70F2E7E368042213
:109220005A70EEE7E36803225A70EAE7E368062221
:109230005A70E6E7E36805225A70E2E7E368042221
:109240005A70DEE7E36806225A70DAE7E36805221F
:109250005A70D6E713F0800F01D10120E9E0E368EE
:1092600002225A700120E4E0B0F88620D0F888107D
:1092700002F0ACF8E368B4F89420DA85E368B4F857
:1092800096201A860020D4E0B0F88620D0F8881006
:1092900002F09CF8D4F894306367A26FD4F8983049
:1092A00082EA030111F4746F04D1D4F89830A367F3
:1092B0000020BEE0E168097803F4746302F474628C
:1092C00001312048FAF71CFBEFE703ABA6E6E368A1
:1092D000012283F85120E46817F020F984ED100A88
:1092E0000020A6E0B0F88620D0F8881002F06EF8D2
:1092F00094F88E3043BBE368002083F87C00E36879
:109300009867E368C3F88400E368C3F88000E36803
:10931000C3F888008DE000BFAFF3008000000000BC
:10932000006A08C1F8C1631ADCA54C4000000000C7
:10933000D012634100000034005043C80000C8420E
:109340000AD7A33B786B0608E36894F8902083F86B
:109350007C20B4F8BD304FF6FF72934256D003EB39
:1093600083035B00E2689367D4F89420D4F89830C4
:109370009FED327B43EC162BB4EE476BF1EE10FA07
:1093800046D0D4F89C00D4F8A01041EC160BB4EEF3
:10939000476BF1EE10FA3BD0D4F8A400D4F8A81033
:1093A00041EC160BB4EE476BF1EE10FA30D0B4F886
:1093B000B8004FF6FF7188422AD09FED226B43EC34
:1093C000172B27EE067BE368BDEEC77B83ED217A82
:1093D000D4F89C20D4F8A03043EC172B27EE067B62
:1093E000E368BDEEC77B83ED207AD4F8A420D4F8DF
:1093F000A8309FED167B43EC162B26EE077BE36827
:10940000BDEEC77B83ED227A002012E00023A9E79E
:10941000E3680020C3F88400E368C3F88000E368D1
:10942000C3F88800E36883F8540002E0002000E0FD
:10943000002004B070BD00BFAFF30080BBBDD7D922
:10944000DF7CEBBD0000000000408F40000000000A
:1094500000408FC02DE9F04104460D4690F87E3063
:10946000013B082B06D8DFE803F03D4F57626974D3
:109470007B95D100242906D1012380F87E3000207D
:10948000A4F8880146E090F88F315E1CF6B280F8AF
:109490008F614FFA81F8034483F88A81924F934B8E
:1094A0009F4210D03246032EA8BF032204F5C57197
:1094B000386817F021FE98B9042E08D1A8F13003BE
:1094C000092B40F20981002084F88F0122E0042E4C
:1094D00040F204813E2DF6D1012384F89031F2E769
:1094E0000437DCE7402905D0522908D0002084F851
:1094F0007E000FE0022380F87E3000200AE009237E
:1095000080F87E30002005E0A4F88210032380F864
:109510007E300020BDE8F081B0F8821001EB05211B
:10952000A0F88210042380F87E300020F2E7A4F82F
:109530008410052380F87E300020EBE7B0F884101B
:1095400001EB0521A0F88410062380F87E3000206E
:10955000E0E7A4F88610072380F87E300020D9E7E2
:10956000B0F8861001EB052189B2A0F88610082317
:1095700080F87E3011F0030F02D0002380F87E3097
:10958000072900F2AD80002084F87E00236F0133AC
:109590002367BFE7B0F88831FF2B02D8C21882F8E2
:1095A000881001339BB2A4F88831B4F88620083AB9
:1095B0009342C0F29780B3F5807F03D9002084F8EE
:1095C0007E00A7E70022022104F184000AF0C2FC19
:1095D0000246022104F186000AF0BCFC0246B4F8FF
:1095E0008610083904F188000AF0B4FC002384F8DE
:1095F0007E30B4F88230834204D0236F0133236776
:10960000002087E72046FFF7B9FC83E7B0F88831F0
:10961000FE2B0AD8C21882F8881001339BB2A0F83A
:1096200088310A2905D0002074E7002084F87E00E4
:1096300070E7C218002182F8881090F888203A2A32
:1096400003D0002084F87E0064E7456E002DF8D03A
:109650005A1F00F18A01284617F04EFD0028F0D16C
:10966000284615F0D7FB00236366236E042B06D82B
:10967000DFE803F003090C1A29000123236609F02F
:109680001FFEA066DDE702232366F8E794F85A3050
:109690000133DBB284F85A30032BF0D9032323665D
:1096A000002384F85A30EAE794F85A300133DBB2E9
:1096B00084F85A30A26892F90C200AB1022BDED944
:1096C00004232366DBE702F0F1FB4FF4AF724FF4A3
:1096D000801102F0D5FBD2E700201BE7002019E73C
:1096E000002017E7002015E7E86D0608006E060861
:1096F00008B540680368DB6811220149984708BD36
:10970000A46B0608836893F90E3083B310B5044642
:10971000436F13F4007F07D013F4807F17D113F049
:10972000800F1CD0012011E0C36819780131114865
:10973000FAF7E6F8E368197801310F48FAF7E0F82C
:109740002046FFF7D5FF002084F87C0010BDC368D9
:10975000197801310948FAF7D3F80020F6E7C36811
:10976000197801310648FAF7CBF80020EEE701201E
:10977000704700BFB86B0608D86B0608FC6B06087C
:10978000186C060810B504460448FAF7B9F8606882
:109790000368DB6813220249984710BD406C060835
:1097A000546C0608F0B583B00546406803681B6931
:1097B00098470746002426460AE0686803685B6904
:1097C0009847C1B22846FFF745FE3043C6B2013480
:1097D000BC42F2D3AB6893F913203AB12A6E042A43
:1097E00007D193F90E30022B00F0B880304603B059
:1097F000F0BD09F065FD0446EB6D8342F6D2AB6E19
:1098000003F5FA63834211D2E86EF7F7C1FC07460D
:10981000686803681B6A9847B842E7D368680368BA
:10982000DB683A46E96E9847AC66DFE795F8903119
:10983000002BDBD06B6EABB1686E0028D6D0F7F78B
:10984000A7FC0446686803681B6A9847A042CDD30A
:1098500068680368DB682246696E9847002385F8CC
:109860009031C3E72B6E042BE6D8DFE803F0032228
:1098700034446F0005F16404AB68EA68127813445D
:1098800093F92270686803681B6E984701280ED010
:10989000434B00934FF461333A464249204606F069
:1098A000ABFCB0F1FF3FC7D100236B66C4E73E4B72
:1098B000EFE7AB68EA681278134493F9223001228B
:1098C0003A4905F1640006F097FCB0F1FF3FB3D1CF
:1098D00000236B66B0E795F85A20354B53F82220E9
:1098E000344905F1640006F087FCB0F1FF3FA3D1D5
:1098F00000236B66A0E7AB6893F90C30012B0FD007
:10990000022B1ED0002B97D12B4A2A4905F1640067
:1099100006F072FCB0F1FF3F8ED100236B668BE73F
:1099200095F85A20254B53F82220224905F164006E
:1099300006F062FCB0F1FF3F7FF47EAF00236B6660
:109940007AE700236B6604232B6675E702F0AEFA14
:1099500093224FF4801102F093FA6DE7184B1B68C5
:109960005B6D93F89C301BB1012385F87C303DE79B
:1099700095F87C30002B3FF439AF6B6F13F4007F08
:109980003FF434AF09F09CFC0446EB6D8342BFF416
:109990002DAF2846FFF7F6FE04F57A74EC6525E74F
:1099A000706C0608786C0608686C06089C6C0608E3
:1099B000006E0608F86C0608FC6C0608DC6D0608EC
:1099C0002C2A003006207047836893F913302BB19E
:1099D000D0F8B804B0FA80F0400970470120704711
:1099E00000487047686E0608024A0260024A026038
:1099F000704700BF8C7006082C71060890F8BC34C4
:109A0000812B09D8802B16D2033BDBB2012B0ED859
:109A10000B4B0B6001207047FF2B08D1094B0B60EB
:109A2000836893F91300B0FA80F040097047054B42
:109A30000B6001207047024B0B600120704700BF94
:109A40008FC2F53DAE47613E704700BF00207047B2
:109A5000704700BF0120704710B50446FFF7C4FFF0
:109A60002046FAF78FFA204610BD00BF0022122AC6
:109A700016D808B5D0F8B8349446012191400B426D
:109A800004D10132D2B2122AF4D908E0C2681178A6
:109A9000044A52F82C2001310348F9F731FF08BD80
:109AA000704700BF38700608706E0608C1F3027078
:109AB000431E042B08D8DFE803F00303090A05005E
:109AC000012070470820704700207047022070472F
:109AD00010B4019C0BE011F8012B93F800C0624414
:109AE000D2B21A7094F800C0624422700246501E2E
:109AF00080B2002AEFD15DF8044B70472DE9F041A8
:109B000086B004460F4616461D46BDF830804068B4
:109B100003681B6A984708F10803984203D20020A3
:109B200006B0BDE8F08100238DF80F308DF80E30BF
:109B3000B5238DF8103062238DF811308DF8127036
:109B40008DF81360ADF814800DF10E0600960DF13E
:109B50000F0304220DF112012046FFF7B9FF009612
:109B60000DF10F03424629462046FFF7B1FF60681A
:109B70000368DB68062204A9984760680368DB680D
:109B800042462946984760680368DB6801220DF168
:109B90000F01984760680368DB68012231469847E7
:109BA0000120BDE710B582B00446406803681B6A17
:109BB0009847072801D802B010BD00220092134632
:109BC00006212046FFF79AFFF5E700BF00B585B0F4
:109BD00090F88B34052B0DD88DF80C108DF80D20D6
:109BE0000223009303AB01220621FFF787FF05B094
:109BF0005DF804FBFFF7D6FF0020F8E7F0B585B06D
:109C000004460F4616461D46406803681B6A98477F
:109C10000A2802D8002005B0F0BD8DF80C708DF830
:109C20000D608DF80E500323009303AB0122062133
:109C30002046FFF763FFEEE708B590F8CE34013316
:109C4000DBB280F8CE3403B108BD90F86D2490F8F3
:109C50007214FFF7D3FFF7E738B50446481E0C2807
:109C600053D8DFE800F00753525252525252523E3C
:109C700052526100901E1E2847D8DFE800F0141BE6
:109C80002F46221046464646464646464646294602
:109C90004646464646464646464646465B000846D3
:109CA0004FF4005523E094F8D204002846D0022552
:109CB00000201CE094F8D204002842D004250020A3
:109CC00015E094F8D20400283ED0082500200EE0CC
:109CD00094F8D204D8B31025002008E008462025C7
:109CE00005E0092A36D00B2A0FD18025052098429D
:109CF00033D003462046FFF781FFD4F8B8342B4316
:109D0000C4F8B834012384F8D03438BD102A06D002
:109D1000152AFAD1A068807B4FF48075E7E7A06828
:109D2000807B4FF48075E2E7032AEED14FF4802563
:109D30000120DCE74FF400450520D8E7084602255E
:109D4000D5E708460425D2E708460825CFE70846A8
:109D50001025CCE740250520C9E7D4F8B83423EA1C
:109D60000503C4F8B834D0E710B582B004460C231C
:109D700000930B4B09220621FFF7C0FE09F0A0FA61
:109D8000C4F87C0494F88034013384F88034E368A8
:109D9000197801310348F9F7B3FD02B010BD00BFD7
:109DA000DC700608986E06088378082B64D8DFE814
:109DB00003F00905161C273340545C00622905D0C6
:109DC00000238370B52905D00020704701338370CC
:109DD000002070478378013383700020704701337F
:109DE0008370C17001710020704701338370C378A4
:109DF0001944C9B2C1700379194401710020704738
:109E000001338370C3780B44DBB2C370027913440F
:109E1000037101700020704701338370C3781944C7
:109E2000C9B2C17003791944017100234370184607
:109E30007047C2781144C9B2C170027911440171EE
:109E400042780132D2B2427001788A4201D00020B9
:109E50007047013383700020704701338370C378EB
:109E60008B420BD0002383709EE70023837003791D
:109E70008B4299D101207047002070470020704725
:109E800000B583B00023009304220A21FFF736FEB9
:109E900003B05DF804FB00BF10B584B00446C3688E
:109EA00019788068FEF76EF9ADF808000123ADF867
:109EB0000A300023ADF80C300621009102AB0822D5
:109EC0002046FFF71BFE04B010BD00BF08B5B0F878
:109ED0006E24083201F07AFA08BD00BF90F8BC0485
:109EE000802814BF00200120704700BF2DE9F047F3
:109EF00084B002AF04460D469046FFF7EFFFD8B19D
:109F000029462046FFF7D2FD064600233B607B60D2
:109F100000F10F0323F00703ADEB030D0DF1080A69
:109F2000606803681B6A98471FFA86F909F11003F5
:109F30009BB2984204D200200837BD46BDE8F087A6
:109F400001233B7007237B707D603B4603CB02906F
:109F500003913246414604A816F060FD09F1080954
:109F60001FFA89F3009353468A2206212046FFF701
:109F7000C5FDE1E7F0B52DED028B93B0044690F8F6
:109F80007234052B4AD0062B00F0A48094F872346A
:109F90000A2B00F0C182022B00F00F83022B00F08D
:109FA00019830D2B00F02383012B40F02A8394F8B2
:109FB0006D24931E2E2B00F20586DFE813F0270395
:109FC0007603AD030306DA033B0403060306030628
:109FD00003060306030603060306030603064405F9
:109FE0000306030603060306030603060306030629
:109FF00003060306030603060306340503060306E9
:10A000000306030603060306030603060306030608
:10A0100003060306030603060306C40590F86D3421
:10A02000012B04D0002013B0BDEC028BF0BD90F8E2
:10A030005A30062B0ED00A2BF4D190F85B30092B46
:10A0400041D00B2BEED1D0F8B83423F08003C0F808
:10A05000B834E7E790F85B30312B2DD013D8162BAE
:10A0600023D0242B06D1D0F8B83423F48063C0F871
:10A07000B834D7E7092BD5D1012380F873340023F6
:10A0800080F8D034CEE73E2B08D0712BCAD1D0F85F
:10A09000B83423F48033C0F8B834C3E7D0F8B83408
:10A0A00023F40063C0F8B834BCE7D0F8B83423F424
:10A0B0008053C0F8B834B5E7D0F8B83423F48043FF
:10A0C000C0F8B834AEE7D0F8B83423F04003C0F895
:10A0D000B834A7E790F86D34242B4FD8242B3FF6E3
:10A0E00055AF01A252F823F021A40408E1A304080B
:10A0F0008D9F04088D9F04088D9F04088D9F040880
:10A100008D9F04088D9F04082DA404088D9F0408CA
:10A110008D9F04088D9F04088D9F04088D9F04085F
:10A120008D9F04088D9F04088D9F04088D9F04084F
:10A130008D9F04088D9F04088D9F04088D9F04083F
:10A140008BA304088D9F04088D9F04088D9F04082D
:10A150008D9F04088D9F04088D9F04088D9F04081F
:10A160008D9F04088D9F04088D9F04088D9F04080F
:10A170008D9F04088D9F0408D9A10408712B00F05D
:10A1800077818B2B06D190F86E34043BDBB200F163
:10A190005E06ACE13E2B7FF4F9AE8368C2681278AC
:10A1A000134493F90F30002B00F0E78000F15A05BB
:10A1B00003AF00F18A0C3E4628686968AA68EB681C
:10A1C0000FC6103537466545F5D128686968AA6815
:10A1D00007C70023184640E00023A0F85A308268E1
:10A1E00092F90130B3F1FF3F08D090F85C1099422A
:10A1F00004D080F85C300123A0F85A3092F90D3079
:10A2000013F1640F0BD094F96620934207D084F8C1
:10A210006630B4F85A3043F00203A4F85A30B4F868
:10A220005A303BB9D4F8B83423F48063C4F8B83456
:10A230000020F8E62422009204F15A030621204669
:10A24000FFF75CFCD4F8B83443F48063C4F8B83446
:10A25000012384F8D034EBE70133062B0EDCA2682F
:10A26000E16809780A4492F90F201A4112F0010FAF
:10A27000F2D0012BF0D00130C0B2EDE7002316E0A0
:10A2800094F85B50E91E420091FBF2F103F10B02DE
:10A2900004EBC202D171157203F10B0204EBC2028E
:10A2A000D2F80A1041F00101C2F80A10013394F803
:10A2B0005D509D423FDDA268E1680D7803F10B011E
:10A2C00004EBC10189792A4492F90F200A4112F066
:10A2D000010F22D0012905D094F8BC24042ACFD83C
:10A2E0000229CDD101290FD00229D5D194F85B20C4
:10A2F000033A410092FBF1F203F10B0104EBC101BF
:10A30000CA7108220A72C7E703F10B0204EBC2020A
:10A310000125D57103251572E6E703F10B0204EB65
:10A32000C2020021D1711172D2F80A1021F001018C
:10A33000C2F80A10BAE704F15A063C22314603A8D3
:10A3400016F05CFB30B9D4F8B83423F40063C4F8D9
:10A35000B83418E0EB000433009333463E22062164
:10A360002046FFF7CBFBD4F8B83443F40063C4F8BD
:10A37000B834012384F8D03405E0D0F8B83423F49D
:10A380000063C0F8B83400204DE6836893F90C20D0
:10A39000022A1DD090F85A30934206D1D0F8B83432
:10A3A00023F48053C0F8B83418E0034603F85A2F5A
:10A3B0000822009216220621FFF7A0FBD4F8B83439
:10A3C00043F48053C4F8B834012384F8D03405E052
:10A3D000D0F8B83423F48053C0F8B834002022E613
:10A3E000B0F86E34082B12D190F88B34052B03D9BA
:10A3F000FFF7D8FB002016E6034493F85C3090F892
:10A400005B2090F85A10FFF727FC00200BE690F82D
:10A410005C3090F85B2090F85A10FFF71DFCF4E7D1
:10A4200090F85A3080F88B340020FCE5B0F85A20C0
:10A430008168C3681B78083331F913309A4202D11E
:10A44000C36D012B0DD02046FFF726FDD4F8B8349C
:10A4500043F00103C4F8B834012384F8D034002059
:10A46000E1E5D0F8B83423F00103C0F8B834F6E7DA
:10A47000B0F85C3013F0010F07D1D0F8B83423F4F2
:10A480008033C0F8B8340020CDE50023A0F85C305C
:10A490002823009300F15A0371220621FFF72EFBB7
:10A4A000D4F8B83443F48033C4F8B834012384F8C2
:10A4B000D034E8E700238DF80C3003AAC2492046C7
:10A4C000FFF714FD012384F8D034D4F8B83443F4F2
:10A4D0008033C4F8B83439462046FFF7E7FA02461D
:10A4E000002800F0A4832B1ADBB204321644042B9C
:10A4F0007FF64CAD3768043BDDB2B34B9F42EAD1E7
:10A5000033798DF80C30002BD4D1D4F8B83423F43F
:10A510008033C4F8B834DEE794F86D34092B4AD0A0
:10A520000B2B48D0042B03D02046FFF785FB42E0DD
:10A53000012384F88C3404F2AB450A2204F178013B
:10A54000284616F0EDFD04F28D461E2204F15A0154
:10A55000304616F0E5FDE368197833462A460131A6
:10A560009A48F9F7CDF908229949284616F0C4FD12
:10A57000D8B90A229749304616F0BEFD60B994F862
:10A58000BC34802B05D0D4F8B83443F48033C4F8FD
:10A59000B834802384F8BC340A228F49304616F040
:10A5A000ABFD10B9812384F8BC34D4F8B83423F05F
:10A5B0000803C4F8B834002035E594F86D24102A57
:10A5C0007FF4ECACA26892F90E20002A3FF4E6ACCE
:10A5D000002028E594F86D24152A7FF4E2ACA268E7
:10A5E00092F90E20002A3FF4DCAC00201BE5D4F8E1
:10A5F0006C2422F0FF0279498A427FF4D5AC002016
:10A6000011E52046FFF718FB00200CE594F8D23442
:10A6100033B1D4F8B83443F00203C4F8B8348BE053
:10A62000D4F85A102046FFF751FCD4F85A30C4F839
:10A630007834E368D4F85E209A61E368D4F8622045
:10A640005A61D4F86A30E168654A82FB0302DB177D
:10A65000C3EBA2030B61E36894F8CF245A7094F81B
:10A66000CD3443F0010384F8CD34D4F86E3007EED6
:10A67000903AE368F8EE677A9FED5A7A67EE877A48
:10A68000C3ED117AD4F8723007EE903AE368F8EE31
:10A69000677A67EE877AC3ED127AE268012382F85F
:10A6A0005230E26882F8533046E0D4F85A1020461F
:10A6B000FFF70CFC94F8D23433B1D4F8B83443F03B
:10A6C0000403C4F8B83437E094F85F3013F0010F96
:10A6D0001CD094F85E20032A09D0032A0ED0022A47
:10A6E00010D0012384F8CF34E268537024E013F0D3
:10A6F000020FF2D0042384F8CF341DE0032384F842
:10A70000CF3419E0022384F8CF3415E0012384F814
:10A71000CF34E26853700FE0002384F8D134D4F8CA
:10A720005A102046FFF7D2FBE368B4F86620DA85BA
:10A73000E368B4F864201A86E36893F85430002B79
:10A7400040F0518294F8CD0410F001003FF46BAC5E
:10A7500094F8CD34C3F3400013F0020F3FF463AC20
:10A76000D4F87424D4F878349A4200F0538200204C
:10A7700059E4D4F85A102046FFF7A8FB94F8D234D5
:10A7800023B1E368B4F862201A81D5E794F8653004
:10A7900013F0010F2CD094F86420032A09D0032A67
:10A7A0000ED0022A20D0012384F8CF34E2685370FF
:10A7B00023E013F0020FF2D0042384F8CF341CE01E
:10A7C000032384F8CF3418E001000320B86E060894
:10A7D000D06E0608DC6E0608E86E060800031C0052
:10A7E000676666666F12833A022384F8CF3404E00A
:10A7F000012384F8CF34E268537094F8D1341BB14C
:10A80000E368B4F88620DA85E36894F8892083F851
:10A81000322094F8CF34012B8ED9E56808F050FD32
:10A82000A865E368D4F85A205A60E368B4F8622057
:10A830001A8181E7012384F8D234D4F85A102046D3
:10A84000FFF744FBD4F85A30C4F8C034C4F8783465
:10A85000E368D4F872209A61E368D4F876205A61EC
:10A86000D4F87E30E168C34A82FB0302DB17C3EBF6
:10A87000A2030B6194F86E30052B00F2D080DFE864
:10A8800003F0039DA1A5C1CAE36801225A70E268E2
:10A89000537884F8CF3494F8CD3443F0010384F82E
:10A8A000CD34D4F8823007EE903AF8EE677A9FED17
:10A8B000B28A67EE887AC2ED117AD4F8863007EE54
:10A8C000903AE368F8EE677A67EE887AC3ED127A19
:10A8D000E368012583F85250E36883F85350E36836
:10A8E00094F8712083F83220D4F85A30C4F87434C4
:10A8F000D4F8963007EE903AE368F8EEE77A67EE20
:10A90000887AC3ED077AD4F89A3007EE903AE66871
:10A91000F8EEE77A9FED990A27EE800AFAF7E6FA51
:10A9200086ED080AE36883F85050D4F88A3007EEC1
:10A93000903AE368F8EEE77A67EE887AC3ED0D7A2D
:10A94000D4F88E3007EE903AE368F8EEE77A67EED7
:10A95000887AC3ED0E7AD4F8923007EE903AE36825
:10A96000F8EEE77A67EE887AC3ED0F7AE36883F84A
:10A970005150D4F89E3007EE903AE368F8EE677ACB
:10A9800027EE888A83ED108A94F8CD3443F00203D1
:10A9900084F8CD3494F8D1343BB1E368B4F8A62000
:10A9A000DA85E368B4F8A6201A86E56808F088FC22
:10A9B000A865E368D4F85A205A60BDE6E36801222E
:10A9C0005A7064E7E36802225A7060E7E368032282
:10A9D0005A7094F86F3013F0020F02D0E36804222B
:10A9E0005A7094F86F3013F0400F02D0E3680522DC
:10A9F0005A7094F96F30002BBFF649AFE368062216
:10AA00005A7044E794F86F105D48F8F779FFE368EF
:10AA100003225A703BE7E36801225A7037E7E36884
:10AA200001225A7033E7D4F85A102046FFF74EFA45
:10AA300094F8653013F0020F3FF47EAEE368B4F88B
:10AA400062201A8178E694F8D23433B1D4F8B8345D
:10AA500043F01003C4F8B8346EE6D4F85A10204618
:10AA6000FFF734FAD4F85A30C4F87434D4F86E309E
:10AA700007EE903AE368F8EE677A9FED428A67EE58
:10AA8000887AC3ED077AD4F8723007EE903AE56819
:10AA9000F8EEE77A9FED390A27EE800AFAF726FAF0
:10AAA00085ED080AE368012583F85050D4F85E303C
:10AAB00007EE903AE368F8EEE77A67EE887AC3ED3E
:10AAC0000D7AD4F8623007EE903AE368F8EEE77A50
:10AAD00067EE887AC3ED0E7AD4F8663007EE903AC6
:10AAE000E368F8EEE77A67EE887AC3ED0F7AE368F9
:10AAF000D3ED0D0A93ED0E0A15F0E4FCE668DFEDE8
:10AB0000227A20EE270AFAF7F1F986ED080AE668BC
:10AB100006F1340009F03AFA86ED070AE36883F893
:10AB20005150D4F8763007EE903AE368F8EE677A41
:10AB300067EE887AC3ED107A94F8CD3443F00203BF
:10AB400084F8CD34F8E5D4F85A102046FFF7BEF962
:10AB500094F85F2002F0070284F8BC24022A19D876
:10AB600053B243BB094B1B68186C03681B68084948
:10AB7000984713E0676666666F12833AACC527375D
:10AB8000F46E06080AD7233CE02E65422C2A0030DA
:10AB9000086F0608D31EDBB2012BE3D8D4F8B83413
:10ABA00023F40073C4F8B834002330220121204676
:10ABB000FFF724F8C0E5D4F8B83423F40063C4F8F0
:10ABC000B834EBE794F8CE340133DBB284F8CE34FA
:10ABD00013B10020FFF727BA01212046FFF70EF836
:10ABE0000020FFF720BA08F06BFBD4F8C834C01A75
:10ABF000B0F5C87F04D9E368002283F85420A1E5AA
:10AC0000D4F8C424D4F8C0349A423FF49BAD002059
:10AC1000FFF709BA94F8CD346FF3000384F8CD340C
:10AC2000DBB26FF3410384F8CD34FFF7FCB90020A9
:10AC3000FFF7F9B930B585B005460C46FFF74EF978
:10AC400048B1002302930393686803681B6A98471E
:10AC50000F2802D8002005B030BD00238DF8083041
:10AC60008DF809300394082300936B448B2206214E
:10AC70002846FEF743FFEEE7836893F91330002B75
:10AC800000F07F8110B582B00446406803681B6AFB
:10AC900098470D2847D9D4F8B834082B1FD094F81A
:10ACA0008A345A1C84F88A24152B00F26681DFE866
:10ACB00013F01F008100AA0037009D009000B7002C
:10ACC0002B003C004F00630072003A003501C500C4
:10ACD000D300E100EF00080121013A00560194F889
:10ACE000D224002ADBD023F00803C4F8B834D6E716
:10ACF000072201212046FEF769FFA0B994F88A34A3
:10AD0000013B84F88A340EE0202201212046FEF720
:10AD10005DFF40B994F88A34013B84F88A3402E03C
:10AD20002046FEF73FFF02B010BD94F8BC34FF2B65
:10AD3000F9D100230093302201212046FEF7DEFEE8
:10AD40000028F0D194F88A34013B84F88A34EAE789
:10AD5000A36893F90C30022B06D1D4F8B83423F44D
:10AD60008053C4F8B834DEE700230093162206218E
:10AD70002046FEF7C3FED6E70023009324220621D7
:10AD80002046FEF7BBFE0028CDD194F88A34013B63
:10AD900084F88A34C7E7002300933E220621204628
:10ADA000FEF7ACFE0028BED194F88A34013B84F84B
:10ADB0008A34B8E700230093082206212046FEF7D4
:10ADC0009DFE0028AFD194F88A34013B84F88A3480
:10ADD000A9E7022201212046FEF7F8FE0028A2D1B1
:10ADE00094F88A34013B84F88A349CE703220121D9
:10ADF0002046FEF7EBFE002895D194F88A34013BFB
:10AE000084F88A348FE7062201212046FEF7DEFE11
:10AE1000002888D194F88A34013B84F88A3482E788
:10AE2000122201212046FEF7D1FE00287FF47BAFDD
:10AE300094F88A34013B84F88A3474E704220121AF
:10AE40002046FEF7C3FE00287FF46DAF94F88A34E5
:10AE5000013B84F88A3466E709220A212046FEF77E
:10AE6000B5FE00287FF45FAF94F88A34013B84F884
:10AE70008A3458E70B220A212046FEF7A7FE002855
:10AE80007FF451AF94F88A34013B84F88A344AE75E
:10AE9000A36893F90E3033B9D4F8B83423F480732F
:10AEA000C4F8B8343FE7102202212046FEF78EFE98
:10AEB00000287FF438AF94F88A34013B84F88A3450
:10AEC00031E7A36893F90E3033B9D4F8B83423F4DA
:10AED0008073C4F8B83426E7152202212046FEF715
:10AEE00075FE00287FF41FAF94F88A34013B84F884
:10AEF0008A3418E794F88C342BB9224B1B685B6DAD
:10AF000093F89C3033B1D4F8B83423F40073C4F808
:10AF1000B83408E72046FEF7B3FF04E72046FEF703
:10AF2000DDFF60B118492046FFF784FE00287FF45A
:10AF3000FAAE94F88A34013B84F88A34F3E60023AD
:10AF40000093712206212046FEF7D8FD00287FF4E9
:10AF5000EAAE94F88A34013B84F88A34E3E60322AB
:10AF60000D212046FEF732FE00287FF4DCAE94F877
:10AF70008A34013B84F88A34D5E6002384F88A3485
:10AF8000D1E670472C2A00300100032010B504469A
:10AF900000F06CF9114B2360002284F88A24FF230F
:10AFA00084F88B3441F6FF71C4F8B81484F8BC34CB
:10AFB0009DF8083084F8CC34012384F8CF3484F829
:10AFC000D13484F8D334E16813460978A068FCF7DB
:10AFD0000DFD2046FFF750FE204610BD8C70060880
:10AFE000F8B5044608F06CF90546D4F88434C31A61
:10AFF000B4F8882493422BD2D4F8B834DBB9A368D0
:10B0000093F91230BBB194F87324A2B994F8802458
:10B01000042A10D8D4F87C24AD1A41F28832954223
:10B0200009D9854A1268526D92F89C201AB9012BF1
:10B030002FD0022B29D0606803681B699847B0F5B0
:10B04000005F01D34FF4005086B200252F462DE05B
:10B050002046FFF711FEC4F88454D4F8B8347BB10D
:10B0600094F8D2243AB913F0170F04D04FF4967322
:10B07000A4F88834C0E740F2EE23A4F88834BBE794
:10B080004FF4FA63A4F88834B6E794F8D034002B70
:10B09000D1D02046FEF768FECDE7622A2AD00023F1
:10B0A00084F86C34B52A29D00135ADB2B54280F0B0
:10B0B000C180606803685B6998470028C0F2BA8065
:10B0C000C2B294F86C34082BEED801A151F823F0E9
:10B0D000A5B004089BB0040809B104081DB1040818
:10B0E0003FB1040863B10408B5B10408FDB1040818
:10B0F00015B20408013384F86C34D5E794F86C3445
:10B10000013384F86C34CFE7013384F86C3484F86D
:10B11000722484F86A2484F86B24C5E7013384F828
:10B120006C3494F86A341344DBB284F86A3494F8CB
:10B130006B140B4484F86B3484F86D24B4E701334A
:10B1400084F86C3494F86A341A44D2B284F86A24CD
:10B1500094F86B341A4484F86B24C0B2A4F86E04DB
:10B16000A2E70133DBB284F86C3494F86A1411441A
:10B17000C9B284F86A1494F86BC4614484F86B14FF
:10B18000B4F86E1401EB002189B2A4F86E14B1F585
:10B19000826F05D90023A4F86E3484F86C3490E7EC
:10B1A0000022A4F8702400297FF47EAF013384F8D4
:10B1B0006C3479E794F86A341344DBB284F86A3467
:10B1C00094F86B140B4484F86B34B4F87034B3F512
:10B1D000826F02D204F15A01CA54B4F870340133B8
:10B1E0009BB2A4F87034B4F86E2493427FF45CAF41
:10B1F00094F86C34013384F86C3455E7013384F8E7
:10B200006C3494F86A3493423FF44EAF002384F8D0
:10B210006C3456E7002384F86C3494F86B34934212
:10B220007FF442AF2046FEF7A5FE00283FF43CAF76
:10B23000074639E73846F8BD2C2A0030032070470E
:10B2400070B50446406860B10E46154603681B6A37
:10B250009847A84205D960680368DB682A463146EA
:10B26000984770BD704700BF704700BF10B50446D7
:10B270000B4820606360A160E26064224FF4FA71C1
:10B2800004F1180000F01EFCE268002382F851303F
:10B29000E26882F85230E26882F85330204610BDEE
:10B2A0002C71060838B52DED028B0446C56895ED66
:10B2B000088ADFED117A28EE278AD5ED078AB0EEED
:10B2C000480A14F0F5FD68EE808AC5ED0D8AE56840
:10B2D000D5ED078AB0EE480A14F0C4FF68EE808A04
:10B2E000C5ED0E8AE3680022DA63E368002283F882
:10B2F0005020BDEC028B38BD35FA8E3C2DE9F04173
:10B3000092B004460E461746C3681D788368C5EBA5
:10B31000C50C03EBCC030DF1100E03F5867CBCE8E5
:10B320000F00AEE80F00BCE80F00AEE80F00BCE86D
:10B330000F00AEE80F009CE803008EE803009DF8C4
:10B340001530CBB1154B1B68D3F8548023685B6B69
:10B35000204698479DF81420114B53F82230029351
:10B360000190013500950F4B3A4631464046F9F7BA
:10B3700077F812B0BDE8F081084B1B68D3F8548011
:10B3800023685B6B20469847019001350095064B7A
:10B390003A4631464046F9F763F8EAE72C2A00308E
:10B3A00010680608E87006080C71060800B58FB032
:10B3B000332201A9FFF7A2FF01A90348F8F7A0FA79
:10B3C0000FB05DF804FB00BFC4D50608836B8B4249
:10B3D00000F0BD802DE9F04385B004460E46816340
:10B3E000D0F81090D0F8148059EA080308D0C36848
:10B3F0005B78012B04D900220023C0E9042309E073
:10B400006068002800F0828003689B6F91B29847C3
:10B410008146884607F054FF0746E36CC51AE0648E
:10B4200019354B4BA3FB05352D09322303FB05F5DD
:10B43000636DAB426FD00023A4F858306565216D71
:10B4400041B12368DA6C4FF47A73B3FBF1F1C9B2FE
:10B4500020469047236D002B6AD0226D05EB5205E4
:10B46000B5FBF2F505FB02F24FF47A7505FB02F22B
:10B47000216C636C521843F1000322646364CDF8BD
:10B480000090CDF8048004F1180000F01FFBE36881
:10B49000C3E91801E368012283F86820E36803AA7E
:10B4A0001978A068FCF734FE00B3E5684FF47A72AF
:10B4B0000023D5E91801F5F799F8381A61EB410135
:10B4C000F4F7FEFF07EE900A9FED227A67EE877A87
:10B4D0009DED037ADFED206A37EE267AB4EEE77A47
:10B4E000F1EE10FA30D5EB6E0133EB66E3685B7872
:10B4F000012B08D94FF47A720023D4E91001F5F733
:10B5000075F8361AA66405B0BDE8F08307F0DCFED6
:10B51000814688467EE7B4F85830042B03D80133BF
:10B52000A4F8583096E7236DAB4293D0256591E798
:10B53000E3681978A068FCF725FEC822322100B222
:10B54000F9F71EFD206588E70023EB66CEE770471C
:10B550001F85EB516F12833ACDCC4C3D10B504469C
:10B56000032300E0013B002BFCDA044B1C60044980
:10B570002046FBF77FFD204610BD00BF083F00308E
:10B580003472060890F8233003B1704710B50123D8
:10B5900080F823300021064B1868F8F71FFE036877
:10B5A000DC6A4FF4007380224FF4E131A04710BDF4
:10B5B0002C2A003000285BDD6F285CD024DC262894
:10B5C0001CDC00284CDD431E252B49D8DFE803F0A6
:10B5D0001355483C484848483F4848484848484828
:10B5E00048484248484848484848484848484848E1
:10B5F0004848484848454FF49660704739283FD03E
:10B6000064282DD124487047B0F5E67F3BD009DD92
:10B6100040F2993398423CD040F2DC5398420ED12C
:10B620001E487047E62831D0B0F5807F02D14FF434
:10B630007A307047732813D14FF4E1307047B0F57A
:10B64000FA7F0DD1164870474FF4965070474FF46B
:10B65000165070474FF4964070474FF416407047AD
:10B66000B0F5FA6FEFDC4FF47A7303FB00F070472C
:10B670004FF4614070470B4870474FF416607047B5
:10B680004FF4614070474FF4E12070474FF4613050
:10B6900070474FF461207047A086010060E31600F8
:10B6A00020A10700FCB1010091421BD0CBB2581E73
:10B6B000C0B22B2918BF012808D8501EC0B22B2AAF
:10B6C00018BF012894BF012000200ED9053BDBB232
:10B6D000012B01D900207047053AD2B2012A03D9C3
:10B6E0000020704701207047012070472DE9F84382
:10B6F00005460F4690460024264604E005EBC400AC
:10B7000013E00134E4B2032C0ED805EBC40393F923
:10B71000062039462846FFF7C7FF0028F1D04645E6
:10B72000ECD00136F6B2ECE70020BDE8F88300BFAC
:10B7300038B50446FFF7DAFF054670B1011BC1F3C7
:10B74000C701074B1868F8F749FD044618B10368AC
:10B750005B6DA9889847204638BD0446FBE700BFCB
:10B760002C2A003070B504460D460A4B1E68C9B23B
:10B770003046F8F733FD03685B6D04EBC504A18820
:10B78000984728B9306C03681B682A4602499847D5
:10B7900070BD00BF2C2A00307C7106082DE9F041F5
:10B7A000064690F92130B3F1FF3F06D02130FF2348
:10B7B00086F821300121FAF789FE3046FFF7E2FED4
:10B7C00001240DE02B68DF6A56F83400FFF7F2FE23
:10B7D00001464FF4807380222846B8470134E4B212
:10B7E000032C00F268812146B44B1868F8F7F6FC88
:10B7F00005460028F2D021463046FFF7B3FF274622
:10B8000006EBC40393F9063001332C2B00F2498177
:10B8100001A252F823F000BFDDB70408C5B7040841
:10B82000C5B70408C5B70408CDB80408D5B80408DE
:10B83000DDB80408DDB80408F7B804080FB9040837
:10B84000A3BA0408D5B80408A3BA040829B904089F
:10B85000A3BA04085FB904088DB90408CFB9040875
:10B86000A3BA0408A3BA0408F3B90408A3BA0408E5
:10B87000A3BA04081FBA0408A3BA040837BA040814
:10B88000A3BA0408A3BA0408A3BA0408A3BA040814
:10B89000A3BA0408DDB70408A3BA04086DBA040803
:10B8A0006DBA0408A3BA0408A3BA0408A3BA04082A
:10B8B000A3BA0408A3BA0408A3BA0408A3BA0408E4
:10B8C000A3BA04086DBA0408C5B70408092346F8EA
:10B8D000343083E7392346F834307FE72B68DF6A5A
:10B8E00056F83400FFF766FE014610234FF48072CD
:10B8F0002846B84772E7732346F834302B68DF6A6E
:10B9000080231A464FF4E1312846B84766E7732092
:10B9100046F834002B68DF6AFFF74CFE01468023AF
:10B920001A462846B84759E706EBC40090F9063096
:10B93000093B07EE903AF8EEE77AF0EEE77A9FEDF2
:10B94000607AF4EEC77AF1EE10FA4FF009038371D2
:10B950004CBF012100210630FAF7B8FD3EE7732005
:10B9600046F834002B68DF6AFFF724FE0146802387
:10B970001A462846B8472B68DB6E012128469847AF
:10B980002B68DB6D00212846984727E7642046F89E
:10B9900034002B68DF6AFFF70DFE014620231022DA
:10B9A0002846B8472B685B6E0221284698472B68CB
:10B9B0009B6E0221284698472B68DB6E01212846A2
:10B9C00098472B68DB6D00212846984706E77320CF
:10B9D00046F834002B68DF6AFFF7ECFD01461E23B2
:10B9E0001A462846B8472B68DB6D00212846984741
:10B9F000F4E62B68DF6A56F83400FFF7DBFD0146FA
:10BA000080231A462846B8472B68DB6E012128465A
:10BA100098472B68DB6D002128469847DEE62B68A7
:10BA2000DF6A56F83400FFF7C5FD014680231A4649
:10BA30002846B847D2E606EBC400FAF755FE10B91F
:10BA4000732346F834302B68D3F82C8056F837002F
:10BA5000FFF7B0FD014610234FF400722846C0479F
:10BA60002B68DB6D002128469847B7E606EBC4003B
:10BA7000FAF73AFE10B9732346F834302B68D3F83E
:10BA80002C8056F83700FFF795FD01464FF4807380
:10BA900080222846C0472B68DB6D00212846984746
:10BAA0009CE62B685F6A56F83400FFF783FD014679
:10BAB0002846B84792E6BDE8F08100BF2C2A003046
:10BAC0000000003401804280704700BF2DE9F04340
:10BAD0008446079C089FA61A67EB0305017E31B1D7
:10BAE0008068DCF80C10864275EB010106DACCF8B0
:10BAF0000860CCF80C5001218CF81810DCF8080014
:10BB0000DCF80C10801841EB03084146BCF800E05B
:10BB10004FF47A7909FB0EFE1EEB000948F100088C
:10BB2000A14578EB07080ADAB4EB0E0067F10001D3
:10BB3000821A61EB0303CCF80820CCF80C30BCF877
:10BB40001A301BB9CCF81060CCF8145001339BB2FA
:10BB5000ACF81A30DCF81040DCF81420A64275EB83
:10BB6000020203DACCF81060CCF81450BCF80220C2
:10BB7000934201D0BDE8F083DCE90423CCE9022341
:10BB80000023ACF81A30F5E710B50446024604234A
:10BB900003E0002102F8011B013B002BF9DA621DD2
:10BBA000042303E0002102F8011B013B002BF9DA1A
:10BBB000002363764FF0FF33636204F13003012109
:10BBC00000291ADB0022DA7000229A60DA601A611A
:10BBD0005A619A61DA611A625A629A62DA631A6485
:10BBE0005A649A64DA641A655A659A65DA65DA669F
:10BBF0001A675A677C330139E2E70023002B01DB27
:10BC0000013BFBE7054B1B680BB1204610BD034B06
:10BC10001C6003492046FBF72DFAF6E70C3F003085
:10BC2000D473060890F832304BB9012380F83230D3
:10BC3000002180F83310117083751846704700207A
:10BC4000704700BF4FF00000704700BF0A4649B17F
:10BC5000037D012B08D0591C0175043340F82320C3
:10BC600001207047002070470020704701238B405F
:10BC7000D0F834211A420CBF01200020704700BFC9
:10BC800010B584B004461021FFF7F0FF28B3194B1C
:10BC90001B68196B0B681B68174A03A89847039B1E
:10BCA0000021039102930291019304220DEB020003
:10BCB00009F0AEF801462046FFF7C8FF019810B121
:10BCC00003685B689847029810B103685B689847FF
:10BCD000039810B103685B689847237D0BB1A37D7F
:10BCE00033B9044B1B68186C03681B6803499847F9
:10BCF00004B010BD2C2A00300C44060860730608FE
:10BD000038B590F91530002B45D0044690F8430122
:10BD1000002841D00025237DAB4208D92B1D54F8C3
:10BD2000230003689B6898470135EDB2F3E707F0FD
:10BD3000C7FA4FF00003DBB29BB9C3EB431204EB2D
:10BD40008202D2F89020821AB2F5FA7F2CBF00222C
:10BD50000122C3EB431104EB810181F8312001334F
:10BD6000E9E74FF0000300E00133DBB233B9E2183A
:10BD700092F92821002AF7D084F8443194F844112C
:10BD80002046FFF75FFFC0B2C0EB401004EB800419
:10BD900094F8310000E0002038BD00BF90F9153064
:10BDA000002B38D010B504464FF00003DBB23BB98E
:10BDB000C3EB431204EB8202116E91660133F5E787
:10BDC000A37D73B1A37D4BB1134B1B68186D036842
:10BDD0005B68642198472046FFF792FF4FF000030D
:10BDE00004E02046FFF74CFFECE70133DBB273B908
:10BDF000C3EB431204EB820292F83220002AF4D102
:10BE0000C3EB431204EB820200211166EDE701232C
:10BE100084F8433110BD70472C2A003038B590F9B2
:10BE20001530EBB1044690F84351D5B1FFF70AFF46
:10BE3000C0B2C0B9C0EB401004EB8004D4ED177A57
:10BE40009FED0B7AF4EEC77AF1EE10FA0DD4B7EE4F
:10BE5000087AF4EEC77AF1EE10FA02DD002500E070
:10BE60000025284638BD0025FBE70025F9E700BF7F
:10BE7000ABAA2A3F014B1868704700BF0C3F003047
:10BE800010B40368194301604368013343600281C1
:10BE9000054B1B685C6DA1624068596D88855B6DC0
:10BEA000DA855DF8044B70472C2A00300048704753
:10BEB000103F003010B50446FFF7F8FF73224FF42F
:10BEC0000001FFF7DDFF0F4B1B7853B10E4B1B68D2
:10BED0005A6D2A2182F846105B6D93F89C3063B14D
:10BEE00010BD094B1B68586D04222146483007F0ED
:10BEF000F7F9044B01221A70E8E72146034807F0DE
:10BF0000ABF900BF1C3F00302C2A0030C474060877
:10BF100010B50446FFF7CAFF83224FF08061FFF798
:10BF2000AFFF074B1B685B6D93F89C3003B110BDEE
:10BF30002146044804F078F92146034807F08CF9BB
:10BF40002C2A0030D8740608F47406080346417B96
:10BF500001228A4006480068024208D110B5054A0D
:10BF60001268D06C026854695A89A04710BD7047A6
:10BF70002C3F00302C2A003010B5002409E004EBDF
:10BF800084029300044A10681844FFF7DFFF01346D
:10BF9000E4B2012CF3D910BD543F0030012801D97F
:10BFA0000020704700EB8000034B1B6803EB800010
:10BFB000B0F90800704700BF543F003008B5037B5C
:10BFC00013F0020F48D1B0F90830023B7D2B43D863
:10BFD000DFE803F03F3F484242424242423F424292
:10BFE00042424848484848484242484848424242FB
:10BFF0004243434242424242424242434242424818
:10C000004848424242424242424242424242424204
:10C0100042424242424242424D42424D4D484848CD
:10C0200048484843424242424848424242424242D1
:10C030004848484848484848484848484848484880
:10C040004D424242424242424242424242424848B9
:10C050004348642109F022F808BD4FF47A7109F0D1
:10C060001DF8F9E741F2941109F00EF8F4E76421A4
:10C0700009F014F8F0E700BF38B52B4B1B68002B14
:10C0800051D02A48428892000021043014F0D4FC98
:10C09000002305E0264A002142F8331001339BB209
:10C0A0008B2BF7D90024234B1C601CE0FFF786FF85
:10C0B0001E4B1B889D422BD26B0905F01F010122EC
:10C0C00002FA01F1194A02EB83035A680A435A60E3
:10C0D000012303FA04F2164951F83530134341F8AD
:10C0E00035300134E4B2012C1AD804EB84029300F9
:10C0F0000D4A10681844B0F90850ADB28B2DD5D94F
:10C10000012303FA04F20B490B6813430B60E8E7C1
:10C11000FFF7CCFE2E224FF40031FFF7B1FED7E738
:10C12000054B01221A7038BD543F0030303F0030BB
:10C13000583F0030283F0030243F00302DE9F041C7
